:020000040800F2
:1000000000800120C1A4000807A5000809A5000878
:100010000BA500080DA500080FA5000800000000B2
:1000200000000000000000000000000011A5000812
:1000300013A500080000000015A50008011800081D
:100040001BA500081DA500081FA5000821A5000884
:1000500023A5000825A5000827A5000829A5000854
:100060002BA500082DA500082FA5000831A5000824
:1000700033A5000835A5000837A5000851AA0008D7
:100080003BA500083DA500083FA5000841A50008C4
:1000900043A5000845A5000847A5000849A5000894
:1000A0004BA500084DA500084FA5000851A5000864
:1000B000C184000855A5000857A5000859A50008E7
:1000C0005BA500085DA500085FA5000861A5000804
:1000D00063A5000865A500083183000869A500082C
:1000E0006BA500086DA500086FA5000871A50008A4
:1000F00073A5000875A5000877A5000879A5000874
:100100007BA500087DA500087FA5000881A5000843
:1001100083A5000885A5000887A5000889A5000813
:100120008BA500088DA500088FA5000891A50008E3
:1001300093A5000895A5000897A5000899A50008B3
:100140009BA500089DA500089FA50008A1A5000883
:10015000A3A50008A5A50008A7A500081947000841
:10016000ABA50008ADA50008AFA50008B1A5000823
:10017000B3A50008B5A50008B7A50008B9A50008F3
:10018000BBA50008BDA5000810B5054C237833B900
:10019000044B13B10448AFF300800123237010BD5A
:1001A000B402002000000000ACE4000808B5064BD3
:1001B0001BB106480649AFF300800648036813B137
:1001C000054B03B1984708BD00000000ACE40008EF
:1001D000B8020020B402002000000000154B002BE4
:1001E00008BF134B9D46A3F5803A00218B460F466E
:1001F0001348144A121A0AF048FE0F4B002B00D085
:1002000098470E4B002B00D0984700200021040097
:100210000D000D48002802D00C48AFF300800AF012
:10022000E7FD2000290008F07BFA0AF0CDFD00BFB1
:100230000000080000800120000000000000000015
:10024000B4020020EC3E002000000000000000008E
:1002500030B4C3787BB902784FF461435109CEF2D0
:10026000000302F01F022031012000FA02F243F8DD
:10027000212030BC70474FF46D43CEF20003457827
:10028000DA6884780378D243C2F30222C2F104010F
:10029000C9B205FA01F10F2545FA02F2C9B22240AE
:1002A0000A4303F1604303F561431201D2B283F8BC
:1002B000002302784FF461435109CEF2000302F0AB
:1002C0001F02012000FA02F243F82120D1E700BF0B
:1002D000F0B444680B680A7924F0407424F4807404
:1002E000234343EA02234360CD680C6987688A6828
:1002F0004E794FF2FD732C43CCF2FF0322433B4077
:10030000134343EA460383600B7DC26A013B22F438
:100310007002DBB242EA0353C362F0BC704700BF15
:1003200000230360037143718360C3600361012391
:100330000375704770B44FF40C5290E84200C4F259
:10034000010285685468C06843F2E0033143CFF688
:10035000FC732943234001430B43536070BC704737
:100360000023036043608360C3607047836819B9EA
:1003700023F001038360704743F0010383607047FB
:10038000092970B421D901EB41041E3CC668072538
:1003900005FA04F526EA050503FA04F445EA040320
:1003A000062AC36020D90C2A02EB82022BD9413ADB
:1003B000C46A1F2303FA02F324EA030301FA02F1D9
:1003C00043EA0102C26270BC7047066901EB410456
:1003D000072505FA04F526EA050503FA04F445EABB
:1003E0000403062A0361DED8013A02EB8202446B61
:1003F0001F2303FA02F324EA030301FA02F143EA9A
:1004000001024263DFE7233A046B1F2303FA02F37E
:1004100024EA030301FA02F143EA01020263D2E78C
:10042000836843F080438360704700BFC06C80B234
:10043000704700BF036819420CBF002001207047BD
:10044000016846F21002002321F00101C4F2020209
:100450000160036043608360C360036121239042B5
:1004600043616BD046F22803C4F2020398426CD079
:1004700046F24003C4F2020398426ED046F258039B
:10048000C4F20203984270D046F27003C4F2020331
:10049000984272D046F28803C4F20203984275D0A3
:1004A00046F2A003C4F2020398423ED046F2B803DB
:1004B000C4F20203984273D046F21043C4F202031E
:1004C000984275D046F22843C4F20203984276D08F
:1004D00046F24043C4F20203984278D046F25843B1
:1004E000C4F2020398427AD046F27043C4F2020387
:1004F00098427CD046F28843C4F2020398427FD0EF
:1005000046F2A043C4F20203984200F0838046F210
:10051000B843C4F20203984201BF4FF4C843C4F287
:1005200002034FF03D52DA6070474FF4C043C4F20B
:1005300002030022C2F23D02DA6070474FF4C0436A
:10054000C4F202033D229A6070474FF4C043C4F2E4
:1005500002034FF474629A6070474FF4C043C4F2D0
:1005600002034FF474129A6070474FF4C043C4F210
:1005700002034FF074629A6070474FF4C043C4F2B4
:1005800002033D22C2F20002DA6070474FF4C0431A
:10059000C4F202034FF47462C2F20002DA607047E0
:1005A0004FF4C043C4F202034FF03D52DA6070478B
:1005B0004FF4C843C4F202033D229A6070474FF4DF
:1005C000C843C4F202034FF474629A6070474FF458
:1005D000C843C4F202034FF474129A6070474FF498
:1005E000C843C4F202034FF074629A6070474FF43C
:1005F000C843C4F202033D22C2F20002DA6070472F
:100600004FF4C843C4F202034FF47462C2F2000212
:10061000DA6070474FF4C843C4F202030022C2F20A
:100620003D02DA60704700BFCA680B68D0F800C0AE
:100630002DE9F0014F698E69CD690C6A42EA030821
:1006400048EA07073E434B6A35432C4344EA03021A
:100650008C6A42EA04034A6B8C6B48F23F071343EF
:10066000CFF21C0723430CEA07071F4307604469C6
:100670000A6BCB6A24F007041343234343610B69DD
:1006800043604B6883608B68C360BDE8F0017047CE
:100690000023036043608360C3600361436183613F
:1006A000C361036243628362C36203634363836320
:1006B000704700BF036819B923F001030360704756
:1006C00043F0010303607047416070470B060CD58F
:1006D0004369AAB143F08003802943610FD00368C6
:1006E00001F01E01194301607047802907D0002ADC
:1006F000F5D1036801F01E0123EA01010160704792
:1007000023F0800380294361F3D1704770B44FF424
:10071000C04246F20F454FF4C84421F0F023C4F222
:100720000205C4F20204C4F2020223F0C316A84276
:1007300088BF224696B1046804F01E0404EAD1245E
:1007400089004CBF5268126823F0821313EA02003A
:1007500002D0201C18BF012070BC7047446904F00F
:100760008004EDE710B44FF4C84246F20F444FF452
:10077000C043C4F20204C4F20202C4F20203A04263
:100780008CBF1046184611F0005F21F0F02121F0D7
:10079000821114BFC160816010BC704700222DE936
:1007A000F00113460126032703E001330232102B28
:1007B0002CD00D6806FA03F42540A542F5D1D0F8F7
:1007C00000C007FA02F4E44304EA0C0CC0F800C0CD
:1007D00091F804C0D0F800800CFA02FC4CEA080C36
:1007E000C0F800C091F804C00CF1FF3CBCF1010F4F
:1007F0000FD9C5682C40C460CC79C56804FA02F4EE
:1008000001332C430232102BC460D2D1BDE8F00179
:100810007047D0F808C004EA0C0CC0F808C091F882
:1008200005C0D0F808800CFA02FC4CEA080CC0F8AD
:1008300008C0D0F804C02CEA0505456091F806C050
:1008400045680CFA03FC1FFA8CFC4CEA0505456070
:10085000CFE700BF00234FF6FF72026003714371C0
:100860008371C371704700BF036919420CBF002038
:10087000012070470AB9418370470183704700BF68
:10088000CB08083301F0070130B4890050F8235039
:100890000F2404FA01F425EA040440F8234050F838
:1008A000234002FA01F2144340F8234030BC704761
:1008B00008B54FF4A843C4F20003984218D04FF48F
:1008C000B043C4F2000398421ED04FF4B843C4F2C0
:1008D0000003984200D008BD01214FF4000000F051
:1008E00091F94FF400000021BDE8084000F08AB9FA
:1008F00001214FF4001000F085F94FF400100021A1
:10090000BDE8084000F07EB901214FF4800000F0FE
:1009100079F94FF480000021BDE8084000F072B979
:10092000F0B5044685B068460D46A68800F0E8F8A4
:10093000029A4DF68363C4F21B33A3FB021326F025
:100940003F06980C3604360C87B23E43A6802388B7
:1009500023F001031B041B0C238048F2A0612B68C9
:10096000C0F201018B4222D85B00B2FBF3F292B2DB
:1009700001372784032A98BF0422A28323889BB2CD
:1009800043F00103238023886989AA8823F48163C3
:1009900023F002031B040A431B0C13439BB2238066
:1009A0002A89AB8913439BB2238105B0F0BDEE8841
:1009B0004BF6FF718E421DBF03EB830303EB8303F2
:1009C000B2FBF3F203EB43030CBFB2FBF3F242F4CE
:1009D000804292B213051B0D0BB942F001024FF495
:1009E000967344F6D35103FB00F0C1F2620181FB20
:1009F00000318909013142F400422184BDE700BF82
:100A0000002341F28832026083804BF6FF7203813B
:100A100043814FF48043C28083817047038829B9A2
:100A200023F001031B041B0C038070479BB243F0AF
:100A300001030380704700BF038829B923F4807342
:100A40001B041B0C038070479BB243F4807303802C
:100A5000704700BF038829B923F400731B041B0CE3
:100A6000038070479BB243F400730380704700BF5C
:100A70001AB901F0FE010182704741F001010182C3
:100A8000704700BF038829B923F480631B041B0C43
:100A9000038070479BB243F480630380704700BFBC
:100AA000038819B95B045B0C038070476FEA43430A
:100AB0006FEA53439BB20380704700BF01827047C7
:100AC000008AC0B2704700BF82B000230A0F0093B3
:100AD000019301900092009B21F07F4153B1019B53
:100AE00014330193019B1B6819420CBF00200120A5
:100AF00002B07047019B1833090C0193F2E700BF65
:100B000010B44FF46053C4F202039A6802F00C026E
:100B1000042A22D0082A26D04FF41052C0F2F40240
:100B200002604FF46053C4F2020320499C68C4F38E
:100B300003140C5D22FA04F242609C68C4F3822420
:100B40000C5D22FA04F484609B68C3F34233CB5CEF
:100B500022FA03F2C26010BC70474FF49052C0F208
:100B60007A020260DDE75C68596814F4800F5C6803
:100B700015BF4FF490534FF41053C0F27A03C0F2F4
:100B8000F40301F03F01B3FBF1F24FF46053C4F200
:100B90000203C4F388145B68C3F30143013302FB0F
:100BA00004F25B00B2FBF3F20260BAE7000000203F
:100BB0004FF46053C4F202031A6B19B922EA000021
:100BC0001863704710431863704700BF4FF46053B9
:100BD000C4F202031A6C19B922EA000018647047C3
:100BE00010431864704700BF4FF46053C4F202030F
:100BF0005A6C19B922EA00005864704710435864CF
:100C0000704700BF4FF46053C4F202031A6A19B967
:100C100022EA00001862704710431862704700BF54
:100C2000002270B44FF48064C4F201020388C4F25D
:100C30000104904218BFA0429BB214BF00220122BF
:100C400008D04FF48064C4F20004B0F1804F18BFA4
:100C5000A04223D14FF68F754C881D4045EA04030E
:100C60004FF4A0564FF48055C4F20005C4F20006BC
:100C7000B04218BFA8421FBF0D894FF6FF441C4069
:100C800044EA050303804B68C3620B8803850AB1FD
:100C90008B7A03860123838270BC70474FF44065D2
:100CA0004FF40064C4F20005C4F20004A04218BF6F
:100CB000A842D5D1CEE700BF00234FF0FF314160FD
:100CC0000380038143808372704700BF038829B982
:100CD00023F080031B041B0C038070479BB243F07E
:100CE00080030380704700BF038829B923F0010304
:100CF0001B041B0C038070479BB243F0010303806D
:100D0000704700BF038C23F001031B041B0C0384FA
:100D10002DE9F001038C8D8984884F88028BB1F80E
:100D200000C02F4322F07302002523F002034FF48A
:100D3000806612041B04C4F20106C4F20105120C01
:100D40001B0CBFB2A84218BFB042A4B242EA0C02C8
:100D500047EA030316D14FF6F775B1F80EC0B1F8A4
:100D600012800F8A8E881D4045EA0C0C4FF6FB73EB
:100D70004FF6FF4548EA070725400CEA0303BCB2DB
:100D800033432C43848002838A6842630384BDE832
:100D9000F001704700230380438083808360838158
:100DA000C381038243827047038B23F008031B0433
:100DB0001B0C194301837047B0F8443021B95B0420
:100DC0005B0CA0F8443070476FEA43436FEA53432B
:100DD0009BB2A0F84430704783899BB21AB923EACA
:100DE000010181817047194381817047C94389B2EC
:100DF0000182704783899BB21AB923EA010181817C
:100E0000704719438181704770B5038ACA8823F4FB
:100E100040531B041B0C1343038283898A880446B6
:100E200008890D4623F4B0534989024323F00C038B
:100E30001B040A431B0C92B21343A381A38AAA8901
:100E400023F440731B041B0C84B01343A382684635
:100E5000FFF756FE4FF4A0524FF48053C4F2010343
:100E6000C4F201029C4218BF9442A2890CBF039BAA
:100E7000029B12B2002A21DB286803EB830303EBF9
:100E800083038000B3FBF0F148F21F53A089C5F241
:100E9000EB13A3FB0152520900B21601642500288E
:100EA00002FB151213DB12013232A3FB0253C3F310
:100EB000431333439BB2238104B070BD2A6803EB14
:100EC000830303EB83035200B3FBF2F1DCE7D200B0
:100ED0003232A3FB0213C3F342133343EAE700BFEA
:100EE0004FF41652002302600C228380C3800381DA
:100EF00042818381704700BF838929B923F400535D
:100F00001B041B0C838170479BB243F40053838105
:100F1000704700BF838919B95B045B0C83817047FC
:100F20006FEA43436FEA53439BB28381704700BF2C
:100F3000C905C90D818070478088C005C00D704704
:100F400001F01F0310B4C1F342110124A14204FABD
:100F500003F30DD002290DD014302AB9026822EA19
:100F60000303036010BC7047026813430360F9E792
:100F70000C30F2E71030F0E7C1F3421310B401F087
:100F80001F020124012B04FA02F416D0022B0CBF1D
:100F9000028A828A92B2224003880124090A04FA52
:100FA00001F19BB219420CBF00200120002A0CBFA6
:100FB000002000F0010010BC7047828992B22240EC
:100FC000EAE700BF090A012303FA01F1C94389B224
:100FD0000180704770B52A4D2C688CB0002C4BD125
:100FE0006846FFF737FC06A8FFF79AF904200121AD
:100FF000FFF7DEFD10234FF40060C4F202006946E3
:10100000009303238DF804308DF80740FFF7C6FBEB
:1010100001214FF48070FFF7E7FD02A8FFF7A0F968
:101020004FF4803302A80393029404940594FFF7CD
:1010300081F94FF400500126C4F2010006A906947C
:101040008DF81C408DF81D4008940A948DF82C6092
:10105000FFF73EF94FF400502346C4F201000E2181
:101060003246FFF78DF94FF40050C4F201003146CB
:10107000FFF77CF9034B1E6001232B600CB070BDA1
:10108000D4020020003E00204FF4005008B5C4F206
:101090000100FFF7C5F940F2D023C2F2000301229C
:1010A0001A6008BD38B50D4C236805460BB9002001
:1010B00038BD4FF40050C4F201000221FFF7BAF925
:1010C0000028F4D04FF40050C4F20100FFF7AEF94D
:1010D000002328802360012038BD00BFD0020020FB
:1010E00030B448F6396301EB4105941EC3F6E303BF
:1010F0000229C1EBC501D8BF144683FB0153D8BFF9
:10110000013AC917C1EB6301201848F21F54D51CDE
:101110000818C5F2EB1484FB02340430D31732EA0A
:10112000220228BF2A46A3EB641100EBA202C3EB04
:10113000E413521842F29340D218C9F2492080FBBE
:1011400002508018D317C3EBA000C0EBC000101AE8
:1011500030BC704770B40646002922D00078F0B148
:1011600000231846F25CA2F13004E4B2092CA2F18B
:1011700041050DD9052DA2F161049CBFA2F13704F0
:10118000E4B205D9052C9ABFA2F15704E4B20024B9
:101190000133DDB204EB0010A94280B2E2D870BC8A
:1011A00070470846FBE700BF0020C4F20200202180
:1011B0000122FFF75FBB00BF0020C4F20200202124
:1011C0000022FFF757BB00BF00B583B06846FFF7AA
:1011D00041FB01200146FFF7EBFC002020220346E3
:1011E0006946C4F20200009201228DF805308DF8A4
:1011F00004208DF806308DF80730FFF7CFFAFFF79F
:10120000DBFF03B000BD00BF00B583B06846FFF749
:1012100021FB04200121FFF7CBFC4FF400600023E9
:101220004FF40052C4F20200694600928DF8043077
:101230008DF80730FFF7B2FA03B000BD4FF400603D
:1012400008B54FF40051C4F20200FFF70DFBD0F1D6
:10125000010038BF002008BDF0B412490A680346F7
:10126000E2B11148114D066811482D680768114810
:101270009D6004681048114D00682D68D8600020FA
:10128000072C08BF04465D60013F06F164059C61C0
:101290000F245D611F6118621C6008601046F0BC7D
:1012A000704700BF00030020D80200200803002080
:1012B00010030020EC020020DC020020E4020020E9
:1012C000F0B583B068464FF40065FFF7C3FAC4F287
:1012D000020504200121FFF76BFC00244FF400639A
:1012E0006946284600938DF805408DF804408DF836
:1012F0000740FFF753FA6846FFF7ACFA04200121D4
:10130000FFF756FC4FF480570126284669460097A0
:101310008DF805408DF804608DF806408DF8074083
:10132000FFF73CFA284639463246FFF7A3FA03B0E6
:10133000F0BD00BFF8B5A44C2368FF2B56D04FF486
:101340000060C4F202004FF40061FFF78DFA054619
:10135000002833D0FFF728FF23689B4D0120012B85
:1013600033D04AD3022B4DD0984B1A68904200F0EC
:101370008680974E186033689A1F0221122A2960CE
:1013800063D9052B94BF93489348944F06F09AFF76
:10139000934806F097FF002323603B680F2B00F073
:1013A000CC81102B6ED0FF2B3AD001333B2B3B600E
:1013B00000F0CE8134D90023236031E0FFF7FCFE3A
:1013C0002368012B2846804DCBD1804B1A6882427E
:1013D00029D01860814BFF221A607D4B002814BF72
:1013E00003200220002220601A60F8BD7D4B1A689D
:1013F000642A19D001321A60F8BD01232B60734BA7
:101400001860F8BD714B1A68904238D0704E186061
:1014100033680322782B2A6012D9704B00221A609D
:1014200000233360F8BDF8BD4FF40060C4F2020041
:101430004FF480510022FFF71DFA00232360F8BD0E
:101440004A2BEDD800232B60EAE7644F0F2B3B6853
:1014500034D8232B00F097813A2B00F085811C2B88
:101460009CD1614A1268D0079FD5604806F02AFFD8
:101470005B4806F027FF002323603B688EE7544B50
:101480001A68B7E75A4A002313605A4A1360564A4B
:101490001360594A1360594A1360594A1360594AF4
:1014A0001360594A1360594A1360594A1360594AE4
:1014B0001360594A136011233B60B1E7A3F1110295
:1014C000292A3FF66BAF01A151F822F0331700082B
:1014D0009D1300089D1300089D1300082D17000898
:1014E00027170008211700081B1700081517000808
:1014F0000F17000809170008F9160008F31600086E
:10150000ED160008E7160008E1160008DB160008D3
:10151000D5160008C5160008BF160008B916000841
:10152000B3160008AF160008AB160008A71600088F
:10153000A11600089B160008951600088F160008D3
:1015400089160008831600087F1600087B1600081D
:1015500069160008571600084516000833160008DB
:1015600021160008B7150008A515000893150008F6
:1015700075150008214A126812F001057FF415AFB5
:10158000264806F09FFE164806F09CFE25603B6844
:1015900004E72149194A0D681068503501300D6083
:1015A0001060FEE61C49154A0D68106828350130A8
:1015B0000D601060F5E61849104A0D681068143582
:1015C00001300D601060ECE630000020F0020020D9
:1015D0000403002030BF000850BF00082C0000208A
:1015E00068C900080C030020E002002070BF00085A
:1015F00000030020F802002014030020E80200206D
:10160000FC020020E402002008030020EC0200207D
:10161000DC02002010030020D8020020B8BF000820
:101620006549664A0D6810680A3501300D60106022
:10163000B7E66149614A0D681068083501300D60F0
:101640001060AEE65C495D4A0D68106804350130F3
:101650000D601060A5E65849584A0D6810680235BB
:1016600001300D6010609CE65349544A0D681068C3
:10167000013501300D60106093E65149D1E75049C2
:10168000D8E74F494D4ADFE74D494C4AE5E74C4919
:101690004A4AEBE74B49494AD6E74A49474ADCE719
:1016A0004849464AE2E7484986E74749B9E7464993
:1016B000C0E74549414AC7E74349404ACDE7424967
:1016C0003E4AD3E7414A126812F001057FF46DAE3D
:1016D0003F4856E73F493D4A6FE73E493B4AA1E74D
:1016E0003C493A4AA7E73B49384AADE73949374AC6
:1016F000B3E73849354AB9E7374A126812F00105AD
:101700007FF453AE35483CE73549334A4CE734491A
:10171000314A52E73249304A84E731492E4A8AE752
:101720002F492D4A90E72E492B4A96E72C492A4A01
:101730009CE72C4A0121116033E62B4B1A6822B139
:101740002A4A0121116000221A6010233B6067E6DB
:10175000274B204A196812689142264922D0204816
:1017600000681A6008605BE6144A1268D2077FF5C9
:101770001CAE214806F0A6FD204806F0A3FD00227D
:101780003B682A600AE6114A1268D1077FF50DAE60
:101790000F4806F097FD194806F094FD00232B60D2
:1017A0003B68FBE50E480C68006801348442D8D1E0
:1017B0000D4C01252560D4E7D8020020E802002066
:1017C00010030020EC020020DC02002014030020A3
:1017D00094BF000808030020E002002070BF00084A
:1017E000E4020020FC020020F80200200003002098
:1017F00018030020F4020020B8BF000868C90008E0
:10180000034B1A6812B11A68013A1A60704700BF98
:10181000043E0020064B074A1B68012B1EBF064BE7
:101820001B68B0FBF3F010601368002BFCD170470D
:101830001C030020043E002038000020044B054A11
:101840001B6803FB00F010601368002BFCD170478D
:1018500034000020043E0020084B094A1B684FF466
:101860007A7110F1FF3001FB03F106D311601368A8
:10187000002BFCD110F1FF30F8D27047340000206B
:10188000043E0020012810B423D002282CD01C4B89
:1018900064221A601B4B0A221A6042F21071032064
:1018A000194B1C684EF21003CEF200034FF46D4248
:1018B000B4FBF1F1CEF2000201395960F02182F857
:1018C000231000229A6007221A60104B186010BC87
:1018D00070470B4B18600B4B44F240214FF47A7267
:1018E0001A60C0F20F01DBE7054B0A221A60054BB4
:1018F00048F2A06164221A60C0F20101D0E700BF83
:101900003800002034000020E80100201C030020E3
:101910002DE9F00140F26C1040F2A81540F24C01A4
:10192000C2F20000C2F20001C2F2000540F2A014AF
:1019300040F2400240F24403C2F20002C2F200034D
:1019400090F8008090F801C087780E7848782D686C
:10195000897882F80080C2F2000482F801C0256014
:1019600097701E7058709970BDE8F001704700BF05
:10197000722009F089B800BF70B5214A82B01160A9
:10198000204A002310608DF804308DF805308DF862
:10199000063000282AD01C481C4A857804784678EE
:1019A00032F8144032F8160032F815208DF8004055
:1019B0004CF6CD45CCF6CC45A5FB0145AD0805EB75
:1019C00085058DF801008DF802204D1B1C46A542AF
:1019D000204601A988BF6946013409F0F5F8042CB6
:1019E000F5D1042009F050F802B070BD044620463D
:1019F00001A9013409F0E8F8042CF8D1F1E700BF9F
:101A0000E8030020200300204C000020DCC3000875
:101A1000D62009F039B800BF70B505460E467224CD
:101A200020462946013409F0CFF8D62CF8D106B962
:101A300070BDBDE87040FFF7EBBF00BF30B540F2AE
:101A40004402C2F200024CF2DC33C0F6000311780B
:101A50009478557833F8111033F8152033F8143092
:101A600083B08DF80410014601A88DF805208DF88B
:101A70000630FFF7D1FF03B030BD00BF00B583B023
:101A80000023014601A88DF804308DF805308DF84B
:101A90000630FFF7C1FF03B000BD00BF0E2A30B40F
:101AA00036D81F4B0C789B5C48F6890213FB04F474
:101AB000C8F68802A2FB0452C2F3C70202700C7877
:101AC00014B10AB9012202704C7848F6890213FB5E
:101AD00004F4C8F68802A2FB0452C2F3C7024270A3
:101AE0004C7814B10AB9012242708C7848F6890208
:101AF00013FB04F3C8F68802A2FB0342C2F3C70239
:101B000082708B7813B10AB90123837030BC70479F
:101B10000B7803704B7843708B788370F6E700BFC7
:101B2000D4C4000810B5104B104C1A68104982B08C
:101B30002046FFF7B3FF0F4B1B689BB10E4B21787C
:101B4000A078627833F8111033F8122033F810308F
:101B50008DF8041001A801218DF805208DF80630BC
:101B6000FFF75AFF02B010BDA00100204400002082
:101B70004000002070010020DCC300080E4B1B68F1
:101B8000032B18D8DFE803F013100A020B4B0022D6
:101B90003F2119705A709A70FFF7C4BF084B012299
:101BA00000201A60FFF76ABF0020FFF767BF054BF0
:101BB0001868FFF743BF7047F4030020400000207F
:101BC000280400207001002030B5244B1B688DB024
:101BD000002B22D0224D00242A462346116911F001
:101BE000020F02F1140205D00CA800EB84010134AD
:101BF00041F82C3C01330B2BF0D1002C1FD1194A9A
:101C00002346146003EB830305EB83056B68984759
:101C1000154B00221A600DB030BD124A10481168F1
:101C2000114A01EB810100EB8100116884680131E8
:101C3000A1421160EFD3416813608847EBE709F0D8
:101C4000B9FBB0FBF4F30CAA03FB140002EB800316
:101C5000044A53F82C3C1360D4E700BF240400204E
:101C600050000020D8030020DC0300202DE9F00FF5
:101C70000C0682B04DD4DFF810C1424C01276FEA48
:101C8000020904EBC10BC2F1040A3D46CDF80490F1
:101C9000ACF10B060021042A1AD854460BEB0708B6
:101CA00001460A290DD818F8019C49FA04F933B302
:101CB00019F0010F05D01CF8019049F002090CF849
:101CC0000190013C0131B4F1FF3FEAD101990631A5
:101CD00063B909180A2909D807EB870807EB4808F0
:101CE00008EB010401310A293555F9D90137092FCB
:101CF0000CF10B0CCED102B0BDE8F00F704719F01B
:101D0000010F1ABF4FF004090CF801900CF80150B4
:101D1000D7E7B0394C292AD8DFE801F02B29292947
:101D20002929292929292929292929292929292923
:101D30002D2929292929292929292929292929290F
:101D400029292F29292929293129292729292929F7
:101D50002D292929292929292929292929292929EF
:101D600029292F29292929293100052183E7202123
:101D700081E701217FE702217DE703217BE7042141
:101D800079E700BFDCBF0008173E00206D2812D89D
:101D900048F6A333CBF62E23A3FB0023DB08DA0798
:101DA00041BF03EB830203EB4203C0EB43000A3065
:101DB000043008F009BF704770B52B4B1A6882B029
:101DC00006460AB901261E60284A294B1178547824
:101DD000907833F8111033F8142033F81030254D73
:101DE0008DF8001000248DF801208DF802308DF858
:101DF00004408DF805408DF806400AE0FFF7C6FF65
:101E000015F8013C013443F001036E2C05F8013C48
:101E100015D015F8013B03F00203DBB220466946FA
:101E2000002BEBD1204601A9FFF7B0FF15F8013CCC
:101E3000013423F001036E2C05F8013CE9D10E4B6F
:101E400018680E4B1968FFF797FD16B10C4B1B680D
:101E500033B1FFF78DFD0B4B01221A6002B070BD4C
:101E60000120FFF7EBFDF6E7FC0300204C0000200B
:101E7000DCC300080C3E002020030020E803002003
:101E8000F4030020083E002008B5064B1A6822B172
:101E9000002210461A60FFF78FFF034B01221A60E1
:101EA00008BD00BF24040020083E002008B50D4BEB
:101EB0000D481A680D49FFF7F1FD0D4B1B68032B08
:101EC00003D00C4B1B68990708D40B4B1B6803B954
:101ED00008BD0120BDE80840FFF76EBFFFF718FD01
:101EE000F3E700BFA80100204C0000206C01002097
:101EF000F403002048000020700100202DE9F0418B
:101F0000854B1A6884B03AB984490B68002B00F0FD
:101F1000E28004B0BDE8F081814A80491678DFF89C
:101F200018824CF6CD40CCF6CC40A0FB06500024E5
:101F300000091C600C6000F0B380C8F80000557800
:101F4000DFF8F8C14CF6CD43CCF6CC43A3FB050338
:101F50001B0902D1002D40F0BC80CCF800309478F1
:101F6000704F4CF6CD43CCF6CC43A3FB04231B09A6
:101F700002D1002C40F0AB806B4A3B606B4B0020E1
:101F80001070507090701E705D709C70D8F80030AA
:101F90001C4693B1654A1478A34240F2948014B170
:101FA000002010700124604A5D4815780078EB1815
:101FB000834200F2A08013700124DCF800308BB162
:101FC0005A48427893427AD912B1002242700124D1
:101FD000554A534855784078EB18834200F2908078
:101FE000537001243868002861D0504B9A78904291
:101FF00061D912B100229A7001244B4D484AAF7842
:1020000096783818B0429CBFC0B2A87003D9B742C6
:102010004DD0AE703046464992F800C092F801E0CB
:102020006C782F785A781D789B7831F81C8031F8BD
:10203000177031F81EC031F8122031F816E031F86F
:10204000133031F8146031F8104031F815008DF874
:102050000A40384D8DF804808DF805C08DF806E0F3
:102060008DF808708DF809608DF80C008DF80D2042
:102070008DF80E30002406E0012B32D0032B35D032
:1020800001346E2C09D0635D022BF5D1204602A9E4
:102090000134FFF77BFE6E2CF5D1FFF769FC38E7C2
:1020A000002E3FF44AAF0123C8F8003047E764BB75
:1020B00001230B602DE7121A9A7001249DE7D21AB2
:1020C0004270012484E7E41A147001246BE70123B1
:1020D00052E7012341E7DFF86080DFF860C0114F6D
:1020E00054E7204603A9FFF751FEC9E7204601A99E
:1020F000FFF74CFEC4E785421CBF107001245CE76B
:1021000085421CBF507001246CE7054A064D967845
:10211000A878064B7FE700BF24040020083E00207B
:102120004C00002034040020400300204403002021
:10213000DCC300080C3E0020CC030020B0030020CC
:1021400070B5154A154B94781178557833F81110FD
:1021500033F8152033F81430114E82B000248DF876
:10216000001005468DF801208DF802308DF80440EE
:102170008DF805408DF80640A35D2B42204601A94D
:1021800018BF69460134FFF701FE6E2CF4D1FFF74A
:10219000EFFB02B070BD00BF4C000020DCC30008A4
:1021A0000C3E00202DE9F843584B594D1A682AB9C6
:1021B0002E68002E00F09B80BDE8F883DFF8588180
:1021C00000221A602A60C8F80020524C4FF0000E1E
:1021D0007646A4460EEB8E000EEB40000B230CEB74
:1021E00000095A1E81186718615C11F0010F46D072
:1021F0000A2A00EB03064BD01CF80660F60742D40F
:1022000021F001013970002A47D0023B0126002B42
:10221000E7D10EF1010EBEF10A0FDBD10120FFF76D
:102220008FFF002E5FD0D8F800300126012B08BFA9
:10223000384CC1D1374F4FF0000EB8460EEB8E0030
:102240000EEB4000002308EB000CC21804EB02095F
:10225000A25C02F00601022926D001330A2BF4D930
:102260000EF1010E0B37BEF10A0FE7D10420FFF784
:1022700067FF002EA0D101232B60BDE8F883134631
:10228000002BAED1C5E713460126002BA9D1C0E72C
:1022900021F0010189F80A10B7E70EF1010E0126BD
:1022A000BEF10A0F96D1B9E743B302F00401C9B2F7
:1022B0000029D2D142F004020A2B89F8002022D052
:1022C0000133C218A25C02F00202D2B24AB10A2B58
:1022D00003F1010317D0FA5C02F00202D2B2002A25
:1022E000F5D10126BAE70123C8F80030A2E7DFF8EC
:1022F0002880D8F80030002B98D166E742F004021D
:102300008CF80020DCE70126AAE700BF24040020A7
:10231000083E00200C3E0020300400202DE9F00F84
:102320006C4B1A6832B96C4A1368002B6BD0BDE84D
:10233000F00F704700201860674A684E684B1060C5
:1023400001213160196033688BB166480A256C1E23
:102350000023C25C02F00301012938D001330B2BAA
:10236000F7D10B382546002CF1D1346043E0DFF87B
:1023700070A1DAF80010002942D0DFF87CB1DBF858
:102380000020002A41D0584D58492A680868584909
:10239000584E02EB820402EB4404241801320F5D14
:1023A0002A6002EB820502EB450527F00407281896
:1023B0000F5536680C5CB24244F0040508BF44F087
:1023C00005040D5404BFCBF800300C5413E004EBAB
:1023D000840004EB40004649C01822F00102092C99
:1023E0000A5408D005EB850205EB4205EB18CA5CE0
:1023F00042F00102CA540520BDE8F00FFFF7A0BE6D
:102400000123136093E7354E9DE740F2C831C2F2D5
:10241000000140F234330F68324840F25C31C2F2BE
:102420000003C2F20001D3F80090D1F80080944676
:102430000A25A0F163066C1ED30749D40023C25CB1
:1024400002F00301022905D001330B2BF7D14B46D3
:10245000002211E0ACB112F0010217D005EB8502A9
:1024600005EB4202D218A846B15C41F00401B15418
:102470004FF0010C2746012225460B388CB19946B6
:10248000D9E7F25C42F00502F254F3E7BCF1000F29
:10249000F0D1F15C41F00401F1544FF0010C904691
:1024A000E8E740F2C831C2F20001CBF800C00F608B
:1024B00040F23431C2F200010B6040F25C33C2F2F0
:1024C0000003C3F80080002A95D1CAF8002092E7E3
:1024D0004B46D1E724040020083E002024030020BE
:1024E000E40300206F3E00205C0300203403002042
:1024F0000C3E0020C8030020040400202DE9F8430E
:102500006B4B1A6832B96B4D2B68002B00F0A6801C
:10251000BDE8F88300201860674C664B20601860A7
:102520004FEA8008654B08EB0007C0F10B0600EB93
:10253000400200EB470703EB8202F7191D4699465C
:10254000DF191346197841F0040103F8011BBB425F
:10255000F8D1C0F1090E431C73454FEA8E0C18D216
:1025600008EB000300EB09070CEB0E0105EB43033E
:102570000B3F0EEB41010A337F18D17A41F0040181
:1025800002F80B1FD97ABA4241F0040103F80B1F7D
:10259000F3D10CEB0E020EEB420252190346D15C52
:1025A00041F00401D1540133B342F8D300284DD097
:1025B000421EC0F10C07BA4210D202EB820102EBBC
:1025C00041010B185B197E19013B761813F8011BAA
:1025D00021F00401B34203F8011CF7D1C0F10A084D
:1025E000404528BF4FEA880920D200EB80034FEA1C
:1025F000880900EB430309EB08019B1802EB050C6B
:1026000008EB4101C0F10B065B198C4493F800E024
:10261000991A2EF0040E83F800E011F806E00B334F
:102620002EF0040E634501F806E0EFD109EB080334
:1026300008EB43031B185B19013B13F8011B013224
:1026400021F00401BA4203F8011CF6D30420FFF77D
:1026500077FD236801332360BDE8F883164C2068BA
:1026600004287FF65DAF05281CBF144B03F16E04F0
:1026700004D119E0A34203F8010C0ED013F8012B8A
:1026800002F00201C9B242F0040022F00402002963
:10269000F0D1A34203F8012CF0D10420FFF750FD44
:1026A00001232B60BDE8F88304220727034D84E74C
:1026B00024040020083E0020580300200C3E002087
:1026C00070B5254A254813681BB90368002B39D01B
:1026D00070BD00231360224D224A03602B601360FB
:1026E0002E6886B9204B03F16E011A7822F004029D
:1026F00003F8012B8B42F8D10420FFF721FD2B6852
:1027000001332B6070BD174A136801331360DA0779
:10271000DED5741EA4B26D2C0FD813490B5D03F0E7
:102720000202D2B22AB10FE00B5D03F00202D2B274
:1027300052B90134A4B26E2CF6D1012303600136E4
:102740002E6070BD064DCBE743F0040304200B550B
:10275000661CFFF7F5FCF2E724040020083E002089
:102760000C0400202C0400200C3E00202DE9F00F6A
:102770008F4B1A6886B042B98E4B1A68002A00F057
:102780000D8106B0BDE8F00F704700221A608A4C38
:10279000884B22601A600292DFF820C2002000EB12
:1027A000800200EB4202624400231178013321F0E1
:1027B00004010B2B02F8011BF7D101300A28EED1DE
:1027C000029A029B0132C3F1040305922260009336
:1027D000002000EB0C0200231178013321F00801E6
:1027E0000B2B02F8011BF7D10B306E28F1D1009FA3
:1027F000724CDDF800B07F420197BA460027BAF16B
:10280000050F2CBFD1464FF005099DE806000023B7
:10281000BBF1040F34BFD8464FF004081AE0042976
:1028200034BF0D460425042B404603D9052A2CBF8E
:102830001546052500EB800600EB460040191CF804
:10284000005045F008050CF8005001330131013209
:102850000B2B15D0E05C00F00200C0B20028F4D0D1
:10286000042FDCD9042B05D8042934BF0D460425D8
:102870004846DFE7042A8CBF154605254846D9E7B8
:1028800001370B340A2F0AF1010A0BF1010BB6D103
:10289000029ADDF808A0DDF814B06FF015036FF0B0
:1028A000090909FB02F903FB02F253460020DB434E
:1028B0000190049280460393CDF800B0039F0298E4
:1028C00007EB080303EB83050AEB8A020AEB4202DB
:1028D00003EB4505019B16182D18D21903EB0C01CB
:1028E0006644624465445C4600231EE0042B30D8F5
:1028F000C34509D89B4507D8049FD01910F80B7C15
:1029000047F0040700F80B7C11F8010B00F00807F2
:10291000FFB21FB140F0040001F8010C0133013691
:102920000132013501340B2B25D002EB0900407830
:10293000C007E9D5B8F1040FD8D9042B009811D8F5
:102940000928E1D89B45DFD8D07A40F00400D07246
:10295000DAE7C345D8D80A2CD6D8687840F0040006
:102960006870D1E70928CFD80A2C9EBF307B40F091
:1029700004003073C8E7019A009B08F101080B328C
:102980000133B8F10A0F01920AF1010A009395D1BF
:10299000042006B0BDE8F00FFFF7D2BB064C20685C
:1029A000042802907FF6F8AE01221A60E9E600BF23
:1029B00024040020083E0020D00300200C3E00200C
:1029C000F8B59B4C2368002B40F0A280994B1B6804
:1029D000032B11D8DFE803F0724211022368002BA9
:1029E00040F0C280944A136833B994490B686D2B48
:1029F00040F2C18001231360F8BD2368002B00F072
:102A00009D808B498E4B00220A608B491A600A60B8
:102A10008C4802F10B0500F10B071D600021BF1A65
:102A20008B1A1B187C180DE013F80B6C16F0010FB5
:102A30009E5C00F0EC8046F004069E5401339C42FC
:102A400000F0EC808D42EFD993F8636006F0020647
:102A5000F6B2002E00F0DA809E5CECE72368002BD3
:102A600076D07349784A00230B60734913600B607A
:102A70005F1C744817601E4603F16E0C594203F147
:102A80000C0433183A460DE05D7815F0010F5D5CDB
:102A900000F0AF8045F0040501325D540133A242DD
:102AA00000F0AF800A2AEFD913F80A5C05F002059E
:102AB000EDB2002D00F09C805D5CEBE72368002BFD
:102AC00031D05B4A614B002111605B4A1960116093
:102AD0004C1C5C481C604E42C1F16E07331800224A
:102AE0000CE013F8015C15F0010F5D5C74D045F04B
:102AF000040501325D5401330B2A74D09442F0D99D
:102B00009D7A05F00205EDB2002D64D05D5CEEE724
:102B100008F050FCC217920F831803F003039B1AAE
:102B2000444A136054E7444A1368002B7FF464AFAF
:102B3000464B19680A293FF65DAFC9E73E490B6865
:102B4000002B7FF459AF3E4B1A686D2A09D85FE716
:102B500039490B68002B7FF44FAF3B4A13680A2BAF
:102B600086D901230B60F8BD314A34490023136034
:102B7000314A0B601360334803F10B021B180A60E3
:102B800003F1160C002113180CEB01040CE01F7864
:102B90009E1A17F0010F354611D0755C013345F0D0
:102BA00004059C42755411D06D2AF0D913F86E7C3F
:102BB00007F002079D1AFFB22E46002FEDD16E5C82
:102BC000013326F004069C426E54EDD10B310B32DA
:102BD0006E29D8D126E05D5C25F0040501325D54F4
:102BE00001330B2A8AD10B36BE427FF477AF19E04E
:102BF0005D5C25F0040501325D540133A2427FF48F
:102C000051AF0B3666457FF43CAF0BE09E5C26F07F
:102C100004069E5401339C427FF414AF0B316E299D
:102C20007FF4FEAE0420BDE8F840FFF789BA00BF8C
:102C30002404002014040020083E0020200400206A
:102C4000600300200C3E00201004002050030020F0
:102C50002DE9F04FB54AB64E136885B033B93368E5
:102C6000002B00F0978005B0BDE8F08F00231360C3
:102C7000B04AB14C1360B14AB14D1360B14A3360F0
:102C800023602B6013602368002B44D1AE4A117877
:102C90001F2960D951781F2900F2C8803F228DF882
:102CA00008308DF809208DF80A30A84BA84E1A6814
:102CB000A04F03A802A9FEF7F1FE29689DF80C8039
:102CC0009DF80DC09DF80EE0A24B36F8188036F83E
:102CD0001CC036F81EE038689F4A83F8008001EB7C
:102CE000810601EB460108180026194683F801C049
:102CF00083F802E0167056709670FFF747F8236865
:102D00002968964A3868D15495495A1CC85422609B
:102D1000FEF72EFEA7E72A680F2A24D9914B03F16C
:102D20006E0403E0A34203F8010C0ED013F8012B4C
:102D300002F00201C9B242F0040022F004020029AC
:102D4000F0D1A34203F8012CF0D10420FFF7F8F9E9
:102D50000123336087E73F228DF808208DF8093082
:102D60008DF80A30A1E7DFF8D4C1724FDCF80030EB
:102D7000D7F800809A4279D0724B1B6802F00109A3
:102D8000B9F1000F4BD143452ED908F101033B6047
:102D90002A6830E0684C6A4D75E7BBF10A0F1AD813
:102DA0005B460EEB8E000EEB400043F60C68C0183D
:102DB000C2F2000818F8008018F0010FDDF800805A
:102DC00004D0E5E0C85CC00700F1E28001330B2BC2
:102DD000F8D1CDF800800EF1010E0B31BEF10A0FD3
:102DE00067D11023CCF80030DCF800309A4228D3A9
:102DF00001232A683360092A2ED92368DFF85C8111
:102E0000062B7BD0564E29683A6808F80310052B2C
:102E1000F25401D801332360FEF7AAFD23E74345AE
:102E2000E2D208F1FF333B602A68E4E792781F2A78
:102E30000AD88DF808308DF809303F238DF80A3014
:102E400033E701322A60D6E73F228DF808308DF84B
:102E500009208DF80A2028E702EB82003B683D49F3
:102E600002EB4000C018FEF791FFC6E740F20840B1
:102E7000C2F200000368984580D112F0010900F009
:102E80008F8008F1FF3B9246B8F1000F02D102F1AA
:102E9000010AC346BAF1090FA3D80AEB8A0143F627
:102EA0000C630AEB4101C2F200035918D646CDF873
:102EB0000080D64562D01EF001033FF472AF0A23B2
:102EC0000EEB8E000EEB400043F60C68C2F20008D9
:102ED000C01818F80000DDF80080C00706D4002BE9
:102EE0003FF477AF013BC85CC007F8D540F208401B
:102EF000C2F20000CCF800E0036041E798F800302F
:102F0000174E092B30D90023013308EB030218F8C0
:102F10000300F15C02F8010CF218052B02F8011C09
:102F2000F2D12368013B23606DE700BF2404002039
:102F3000083E00201C040020F8030020C0030020ED
:102F4000F0030020080400206C010020A8010020EC
:102F5000DCC30008000400204803002038030020E0
:102F6000280300200C3E00203278124903EB830036
:102F700003EB40008018FEF709FFC4E71EF0010FC5
:102F80003FF40BAFBBF1FF3F18BF5B4698D122E780
:102F900040F20841C2F20001CCF800E00B60EFE61D
:102FA000B8F1090F9CBF08F1010B92467FF672AF92
:102FB0006DE700BF480300202DE9F04F874B884D97
:102FC0001A6885B0002A40F09B802B68002B58D1EE
:102FD000DFF820A2DAF800201D2A55D8DFF80CB25D
:102FE000DFF818829BF800009BF801109BF8022084
:102FF0008DF80C008DF80D108DF80E209946D8F83C
:1030000004400F2C2ED9A4F10F05012D64D0A4F19A
:103010001103092B69D9092D5ED904EB840304EB54
:103020004303103CA9F1BB070126A51E092C1F4430
:1030300009D9082D45D90136163F6B1C2C460FD0F7
:10304000A51E092CF5D89BF8013007F10B00B3FB46
:10305000F6F303A98DF80D30FEF798FE002CE8D1A9
:10306000D8F8044009F101090134B9F10B0F48F80F
:10307000044FC4D1FEF77CFCDAF800300133CAF803
:10308000003005B0BDE8F08F564B03F16E0403E04D
:10309000A34203F8010C0ED013F8012B02F0020139
:1030A000C9B242F0040022F004020029F0D1A34288
:1030B00003F8012CF0D10420FFF742F801232B6024
:1030C000DFE79BF801303846B3FBF6F303A98DF830
:1030D0000D30FEF75BFEAEE705EB850005EB40002B
:1030E00048444149FEF752FE97E705EB850005EBA2
:1030F0004000A9F11603C0183C49FEF747FE8AE7D5
:103100003B4ADFF8FC80176800261E60394B2E60B2
:103110003F243A4602A869461E6010238DF8063007
:103120008DF800408DF801408DF805408DF8026063
:103130008DF80460FEF7B2FC3A4603A801A9FEF739
:10314000ADFC2D4B9DF808709DF809C09DF80AE074
:103150009DF80C409DF80D009DF80E90224933F823
:103160001770224A33F8144033F81CC033F81EE0BD
:1031700033F8100033F819300F7046F26767147097
:1031800081F801C081F802E0507093703446C6F2B5
:10319000666711E008F00EF987FB0032C317C3EB36
:1031A000A20303EB8303A0EB430048F806000134BD
:1031B00004360B2C3FF409AFE207EBD408F0FAF821
:1031C00087FB0032C317C3EBA20303EB8303A0EB1F
:1031D0004300053048F80600E9E700BF240400205A
:1031E000083E00200C3E002038040020B8030020D8
:1031F000A8010020B4030020DCC3000880030020E5
:1032000084030020704700BF074B012003F16E01CB
:1032100013F8012B12F0020214BF03F8010C03F89B
:10322000012C8B42F4D170470C3E00202DE9F84F61
:103230009246814688460AB9BDE8F88F0020FEF71D
:10324000BBFD1AF0080F40F095801AF0100F40F007
:103250008D80DFF87CB14146DBF80000FEF78CFB87
:10326000524A534B11784CF6CD42CCF6CC42A2FBDD
:103270000802920801EBC101C90002EB420201EB16
:1032800042021AF0040F02EB0301D05CD4D0494A89
:10329000494F00249460D4601461146054615460F8
:1032A000148394763B4607F16E05012613F8014B13
:1032B00014F0020414BF03F8016C03F8014CAB4294
:1032C000F4D1DBF80030002B62D03C4B1B68DC07EC
:1032D00062D501235370937000230125CC1801336C
:1032E000A47814B1042B1555F8D1B9F10B0F4B7814
:1032F00088BFA9F10C099944B9F10B0F88BFA9F156
:103300000C0900EB400009EB80092D4B13F8191054
:1033100003EB490329B15B78012050540BB1254AD6
:10332000D054284CDFF8ACC004F11B06002514F87B
:10333000013F9BB105EB0C0315F80C2098785B78E6
:1033400060B102EB820102EB41021818D219D15C84
:1033500041F00201D15401338342F8D10335B44224
:10336000E5D1194B01221A60BDE8F88F0120FEF764
:1033700085FB6EE706F01CFDC820FEF75FFA134BD5
:103380001B68002B7FF465AF0120FEF757FB60E759
:103390001AF0100FE5D14FE7B8F1040F99D9A8F151
:1033A0001E08B8F1040F97D893E700BFC4030020AC
:1033B000E4C40008640300200C3E00204800002004
:1033C000F8C600086303002024040020F403002052
:1033D00070010020A4C6000840F24803C2F20003B6
:1033E0001868704738B50B4B0B4D1B68032B044610
:1033F00004D0820702D52B689B0707D5FEF7BEFBDA
:10340000064B2C6001221A60204638BDFEF780FA78
:10341000F4E700BFF403002048000020240400204B
:1034200040F2F433C2F2000318687047032810B565
:1034300009D8074C2368834203D02060FEF79EFB27
:103440002368184610BD024B1B68184610BD00BF0C
:10345000F403002040F23C03C2F2000318687047F6
:103460006328024B88BF6420186070473C0000202E
:1034700040F29C13C2F20003186870476228024BA6
:1034800088BF0020186070479C01002040F2C433C0
:10349000C2F20003186870470328044B04D8186070
:1034A000034B01221A60704718687047C40300205C
:1034B00024040020064B1868022805D90020186053
:1034C000044B01221A60704701301860F8E700BF12
:1034D000C403002024040020054B186828B10138DB
:1034E0001860044B01221A60704703201860F8E747
:1034F000C40300202404002040F21843C2F2000359
:1035000018687047074B10B5186000B110BD064B26
:103510000F241C60FEF7CAFC044B1C60BDE8104081
:10352000FEF700BB18040020A8010020A001002025
:1035300040F2A413C2F2000318687047024B0A2835
:103540008CBF186818607047A4010020044B1868ED
:10355000092802D9002018607047013018607047B0
:10356000A4010020044B186810B10138186070479E
:103570000A201860704700BFA4010020064B1B689A
:10358000012B00D07047054B00223F2119705A7063
:103590009A70FEF78BBC00BFD40300206C010020A2
:1035A00040F2D433C2F2000318687047012810B506
:1035B000034602D9054B186810BD044C2068984298
:1035C00003D02360FFF7DAFF206810BDD40300208A
:1035D000F0B5574B1B68012B83B0044641D0022B3A
:1035E00001D003B0F0BD20B9524B1A68002A78D040
:1035F00018600020FEF742FA4F4B1B683B2B2DD87A
:103600001D2B71D967081E254C4A4D4B10785178F7
:10361000927833F8100033F8111033F81220454B2C
:103620008DF804001B688DF805108DF80620002B1E
:1036300045D1AF423CBF434E3C4605D338E07230E3
:1036400007F0C2FAAC4233D2306820180134A842E5
:1036500001A9F4D33C386328F4D8F0E727463C2589
:10366000D2E70020FEF70AFA334B1B683B2B47D901
:10367000344B1A683C23A418304AA34298BFC3EBCA
:10368000040411782E4B9078557833F8111033F8E4
:10369000152033F810308DF80410632C8DF80520B8
:1036A0008DF8063004D804F1720001A907F08CFAF5
:1036B000254B1B68002B94D0FEF7AAF991E7214E09
:1036C000002404E0723007F07FFABC42F0D833687F
:1036D000E0180134A84201A9F4D33C386328F4D897
:1036E000F0E701221A6084E7132B7FF67AAF4AF6DF
:1036F000AB27CAF6AA27A7FB04377F08142583E760
:103700001D2B0ED8132B7FF66CAF0E4A4AF6AB2357
:10371000CAF6AA231268A3FB041402EB5404142370
:10372000AAE7084B1A681E2302EB5404A4E700BF63
:10373000F4030020280400203C0000204400002066
:10374000DCC300089C0100207001002038B5874BC5
:103750001B680A2B1DD8864A864C126892B9864D82
:103760002A68DAB9042B00F0E2808449844A03EB2A
:10377000830301EB83031168986801318142116072
:1037800045D238BD7D4A03EB830302EB83035B68BC
:103790009847794B1B68002BF3D0764C794B1B680C
:1037A000012B1FD0784B1B68032B06D02368002BFE
:1037B000E7D1BDE8384006F019BB744B74491A686C
:1037C000496B0132B2EB411F1A60EFD371490A68AD
:1037D0000020013A1860052A3AD8DFE802F050A12B
:1037E0009A938C856C4B6D491A6849690132B2EB2A
:1037F000411F1A60D6D36A490A680020013A18604E
:10380000052A0CD8DFE802F069625B544D440021C0
:103810005B68116098472B68002BBED1B1E7614A05
:1038200013680133072B00F09E805F481360026825
:103830000B6001320D2A5A49026000F08B800E2A7B
:10384000B0D1013B08BF06230B6000230360A9E74A
:10385000564A13680133072B7AD055481360026823
:103860000B6001320D2A4B49026068D00E2A9DD1AF
:10387000013B08BF06230B600023036096E74D4B16
:103880005A783E2AE4D801325A70FEF74BF98DE798
:10389000494B9A78002AC2D0013A9A70FEF706FB8B
:1038A00080E7454B1A783E2AB9D801321A70F5E7FD
:1038B000414B5A78002AB2D0013A5A70EEE73E4B9B
:1038C0009A783E2AABD801329A70E7E73A4B1A78D9
:1038D000002AA4D0013A1A70E0E7374B5A783E2A02
:1038E0009DD801325A70D9E7324B9A78002AAFD06E
:1038F000013A9A70C9E72F4B1A783E2AA8D80132AC
:103900001A70C2E72B4B5A78002AA1D0013A5A709C
:10391000BBE7284B9A783E2A9AD801329A70B4E7CE
:10392000244B1A78002A93D0013A1A70ADE7134B52
:103930005B6D98472B68002B7FF42FAF21E7013395
:10394000072B18BF0B607FF431AF01230B602DE70D
:10395000012382E70133072B18BF0B607FF422AFEE
:1039600001230B601EE701235FE700BFA4010020D5
:103970002404002070010020083E00205000002098
:10398000EC030020D4030020F4030020E003002017
:103990002C0100204C030020300300207C0100207B
:1039A000800300203C040020740100205403002008
:1039B00078010020400000206C010020064B1A789E
:1039C0003E2A07D803D13F221A70FEF76FBA02329F
:1039D0001A70FAE7704700BF6C010020064A13789E
:1039E00043B1012B03D100231370FEF75FBA023BF2
:1039F0001370FAE7704700BF6C010020064B5A783D
:103A00003E2A07D803D13F225A70FEF74FBA02323E
:103A10005A70FAE7704700BF6C010020064A5378DD
:103A200043B1012B03D100235370FEF73FBA023B91
:103A30005370FAE7704700BF6C010020064B9A787C
:103A40003E2A07D803D13F229A70FEF72FBA0232DE
:103A50009A70FAE7704700BF6C010020064A93781D
:103A600043B1012B03D100239370FEF71FBA023B31
:103A70009370FAE7704700BF6C01002040F26C13AE
:103A8000C2F200031A7802705A7842709B788370F1
:103A9000704700BF10B440F26C130478417882780C
:103AA000C2F200033F2C34BF20463F203F2928BFED
:103AB0003F213F2A28BF3F22187059709A7010BCCE
:103AC000FEF7F4B940F24003C2F200031A78027024
:103AD0005A7842709B788370704700BF10B440F2F0
:103AE0004003047841788278C2F200033F2C34BF4F
:103AF00020463F203F2928BF3F213F2A28BF3F22A1
:103B0000187059709A7010BCFEF70CB840F2A813E8
:103B1000C2F20003186870470F2803D8034B1860DF
:103B2000FEF7C4B9014B0F221A60F9E7A801002083
:103B3000034B1A6802B97047013A1A60FEF7B6B92A
:103B4000A8010020044B1A680E2A00D970470132E0
:103B50001A60FEF7ABB900BFA801002040F2A01325
:103B6000C2F20003186870470F2803D8034B18608F
:103B7000FDF7D8BF014B0F221A60F9E7A001002022
:103B800030B5012583B015F0010F0CBF002139219C
:103B900015F0020F0CBF0022392215F0040F0CBFE4
:103BA000002339238DF804108DF805208DF8063098
:103BB0000024204601A9013407F006F8D62CF8D1DC
:103BC000204606F061FF01350320FDF745FE082D74
:103BD000D9D10020FEF7F0F803B030BD284B2DE915
:103BE000F04103F16E01012413F8012B12F00202DF
:103BF00014BF03F8014C03F8012C8B42F4D1017877
:103C000000293AD080460746013705260020C6F134
:103C100005020346FEF72AF898F8011059B30A2E58
:103C200018D83D46344601E00A2C13D8002220461D
:103C30001346FEF71BF815F8011F06340029F3D1CF
:103C400006E000222046202113460634FEF70EF837
:103C50000A2CF6D90420FEF773FA3220FDF7EEFDA8
:103C6000013E02D017F8011CD0E718F8011F002907
:103C7000CAD1BDE8F0813446EAE7BDE8F08100BF73
:103C80000C3E002070B51B4D2B6882B004460BB96A
:103C900002B070BD4208184901A807F0D7FB002008
:103CA000FEF78AF8154B04F0010603F16E000124BB
:103CB00013F8012B12F0020214BF03F8014C03F8B1
:103CC000012C8342F4D1002002469DF80410012308
:103CD000FDF7CCFF0022012306209DF80510FDF71B
:103CE000C5FF28687100FDF747FE054B01221A60E9
:103CF000CEE700BF700100205CC400080C3E00202D
:103D0000240400202DE9F04FB94B1B68044693B002
:103D1000184613B913B0BDE8F08F3F268DF8346014
:103D20003C2603258DF82360162600230CA92A467D
:103D3000A4208DF824600F268DF835308DF83630AC
:103D40008DF825308DF826308DF82B308DF82750E2
:103D50008DF8296000F0AEFB01220DF12101A720B2
:103D600000F0A8FB01220DF12501A82000F0A2FB24
:103D700001220AA9BD2000F09DFBBE2001220DF109
:103D80002A0100F097FBB4F5843F80F0A3809DF8F2
:103D900021809DF822C09DF825E09DF82610B8F1FD
:103DA000030F84BF4FF000088DF82180BCF1030F92
:103DB00084BF4FF0000C8DF822C0BEF10A0F84BF03
:103DC0004FF0000E8DF825E0012902D900218DF871
:103DD00026109DF828700F2F02D90F278DF8287014
:103DE0009DF829600F2E71D89DF82A00012802D075
:103DF00000208DF82A009DF82320642A009203D920
:103E000064258DF8235000959DF82430632B02D94A
:103E100016238DF82430774C07932568764B01954F
:103E20009DF827509DF834B002959DF830509DF8CC
:103E300035A003959DF831509DF8369004959DF876
:103E4000325083F800B005959DF82B5083F801A0FF
:103E5000069540F2C435C2F2000583F80290C5F819
:103E60000080DFF8C081029DC8F800C0DFF8B8C14B
:103E7000624BCCF80050DFF8B4C1614ACCF800E0E6
:103E8000DFF8ACE11F60CEF800105E4B0399049D93
:103E900011701E6005995C4B557091701860009A06
:103EA0005A4B079D1A605A4B06991D60594B196071
:103EB00000232360FDF736FEFDF7F8FF019A22602C
:103EC000FFF75CFBFDF75AFE012023E70F268DF874
:103ED000296089E7A92001220DF1260100F0EAFA04
:103EE00040F6FF03C0F201039C427FF650AF01226F
:103EF0000DF12701BC2000F0DDFA0DA92A46D720DC
:103F000000F0D8FA01220DF12901DA2000F0D2FAEE
:103F1000DB2001220DF1220100F0CCFAB4F5003FC4
:103F2000FFF435AF01220DF12301DC2000F0C2FACD
:103F3000DD20012209A900F0BDFAFF23C0F202032F
:103F40009C427FF624AF0DF12B010122E02000F00E
:103F5000B1FA0FA90B22E52000F0ACFA0EAE0BA9C6
:103F6000022240F2251000F0A5FA40F23510314649
:103F7000042200F09FFA0DF14605274B0DF13B009E
:103F800005E042F002021A611433A84212D010F880
:103F9000012FFF2AF8D002F01001C9B202F00F027F
:103FA0009A601A690029ECD122F002021A611433D6
:103FB000A842ECD19DF82C301848FF2B1EBF184AA0
:103FC00003F00F0353609DF82D30FF2B1EBF144AE2
:103FD00003F00F0353610023F25CFF2A1EBF00EBC6
:103FE000031102F00F024A600133042BF4D1CEE634
:103FF000600400207001002040000020A801002083
:104000006C010020A0010020180400203C000020CA
:104010009C010020BC030020500000202C01002047
:104020007C010020F403002048000020A4010020AF
:10403000D40300202DE9F04F854B1B68A3B0002B63
:1040400000F08B80834B844A93F8008093F801C082
:1040500093F802E0814B92F800B01F68804B92F811
:1040600001A01E687F4B92F802901D687E4B8DF870
:1040700019501C687D4B8DF81A401B688DF820B0D4
:1040800000937B4B009C1B688DF81B400193794B80
:10409000019C1B688DF821A00293774B8DF822902C
:1040A0001B688DF824800393744B8DF825C0186825
:1040B000734B8DF826E01968724B8DF815701A68ED
:1040C0008DF816608DF81C40029C6F4B8DF81D40DA
:1040D000039C8DF817008DF81E408DF818100020F5
:1040E0008DF81F2012ACFF250A2888BF255409D857
:1040F0009A68196902F00F028907225444BF42F0FE
:1041000010022254013014334028EDD15F480023BF
:104110000AAEFF22012B97BF00EB0311F25449684E
:1041200001F00F0198BFF1540133102BF2D158491F
:1041300000230EADFF2001EB0312032B97BF526843
:10414000E85402F00F02EA540133102BF3D1A420FB
:1041500008A9032200F0C8F918B9002023B0BDE86F
:10416000F08FA7200DF11501012200F0BDF9002804
:10417000F3D0BC200DF11901012200F0B5F900289F
:10418000EBD0A8200DF11A01012200F0ADF90028B2
:10419000E3D0A9200DF11B01012200F0A5F90028B0
:1041A000DBD0BD2007A9012200F09EF90028D4D061
:1041B000BE200DF11E01012200F096F90028CCD09E
:1041C000D72009A9032200F08FF90028C5D0DA20F2
:1041D0000DF11D01012200F087F90028BDD0DB2080
:1041E0000DF11601012200F07FF90028B5D0DC2086
:1041F0000DF11701012200F077F90028ADD0DD2084
:1042000006A9012200F070F90028A6D0E0200DF1E7
:104210001F01012200F068F900289ED0E520214608
:10422000402200F061F9002897D040F22510314675
:10423000102200F059F900288FD0102240F23510DA
:10424000294600F051F9003018BF012086E700BF71
:1042500060040020400000206C010020C403002006
:10426000F403002048000020A4010020D403002013
:10427000A8010020A0010020180400203C0000201C
:104280009C010020BC030020500000207C01002085
:104290002C01002006F0C4BC2DE9F8438146884675
:1042A000174605F041FC10B90020BDE8F883552001
:1042B00005F0D2FC2E48082105F0F6FC442005F05C
:1042C000CBFC002443F2144505F090FC0134AC42D1
:1042D00098BF002814BF00260126F5D043F21443EE
:1042E0009C4227D805F020FC0028DDD0552005F0A1
:1042F000B3FC204C1E48082105F0D6FCBE2005F07A
:10430000ABFC0921204605F099FC05F00DFC1A4B89
:104310001B68222B13D0282B11D00923C9F8003099
:1043200094F90130DB0FC8F80030237801203B609E
:10433000BDE8F88305F0F8FB3046BDE8F883237943
:1043400062782578C3F34113093302F00704C3F1FF
:104350000C00191F45FA00F004FA01F10143D209DB
:10436000C9F800300120C8F800203960BDE8F883A2
:10437000540400204004002050040020F8B5A0F1AF
:104380000905032D044602D900263046F8BD05F084
:10439000BBFC05F0C9FB0028F6D02E4F384605F0CF
:1043A00091FC3B782C4A13602C4A0121222B0646B3
:1043B000116001D0282BE8D105F0B6FB0028E4D02D
:1043C000552005F049FC264F2248082105F06CFCD9
:1043D000BE2005F041FC0921384605F02FFC3B7951
:1043E000C3F341130933A342CFD005F09DFB00284E
:1043F000CBD0552005F030FC0821164805F054FCC0
:104400004E2005F029FC7F2005F026FC802005F0D9
:1044100023FC680100F0E00005F01EFC05F084FBC1
:1044200005F082FB0028B0D0552005F015FC0948A6
:10443000082105F039FC482005F00EFC002405F0A9
:10444000D5FB0134F92C98BF0028F8D005F06CFB9F
:104450009BE700BF54040020500400204C040020BF
:10446000400400202DE9F04184B003F035F8DFF876
:10447000408000240127650045F0A0050126009733
:104480002846002132460DF10F03A419C8F8005048
:1044900003F076F830B1082CEDD1044B186804B065
:1044A000BDE8F081014B30461E60F8E76004002053
:1044B0005C04002010B50A4B1C6882B00B4614B98E
:1044C000204602B010BD0092064A1268014610460E
:1044D000012203F055F8D0F1010038BF0020F0E7C9
:1044E000600400205C0400202DE9F047144B1B6899
:1044F00082B0174603B3EAB1DFF84CA0114C064670
:10450000C0EB01094FF001080025DAF80000CDF8F2
:1045100000803146012209EB060303F0AFF858B9D9
:1045200010202368002BFCD001382560F9D101361A
:10453000013FEAD1012000E0002002B0BDE8F08791
:10454000600400207C3E00205C04002070B53E4BDF
:104550001A68824288B0064674D002A81E60FCF732
:1045600079F904A8FCF7BCFC01200146FCF720FB0C
:1045700001200146FCF71CFB20200121FCF734FB45
:104580000020C4F202000B210822FCF779F9002078
:104590000822C4F202000C21FCF772F90223002069
:1045A0008DF80C30032304460125C4F2020002A951
:1045B0008DF80D304FF4006302938DF80E408DF8A6
:1045C0000F50FCF7EBF820464FF48053C4F2020082
:1045D00002A90293FCF7E2F84FF4A050C4F20100E4
:1045E0002946FCF797FC4FF4A0500C23C4F20100BD
:1045F00004A9ADF81A300496ADF81440ADF8164091
:10460000ADF81840ADF81C40FCF7FEFB4FF4A0508D
:10461000C4F201002946FCF76FFC4FF4A050C4F22D
:10462000010040F225512A46FCF78AFC472301A8E5
:104630008DF804308DF805408DF806408DF8075050
:10464000FBF706FE08B070BD7C06002030B40F4AB0
:1046500013687F2BFCD80E490E4D0B685C1C7F2C19
:1046600045F8230098BF0C6001D900230B6072B697
:1046700013680133136062B64FF4A050C4F2010016
:1046800040F22771012230BCFCF75ABC78060020AA
:10469000740600206C04002010B50446007828B190
:1046A000FFF7D4FF14F8010F0028F9D110BD00BFA7
:1046B00040F26843C2F200031868003018BF0120BE
:1046C000704700BF30B40D4B1A6882B10C490D4DD4
:1046D0000A68541C802C55F8225018BF0C6009D071
:1046E00072B61A68013A1A6062B601220560104675
:1046F00030BC704700220A60F2E700BF6804002067
:104700006404002080060020024A1368002BFCD1BC
:10471000704700BF780600204FF4A05038B5C4F2AF
:10472000010040F22551FCF727FC00282BD14FF463
:10473000A050C4F2010040F22771FCF71DFC00B943
:1047400038BD4FF4A050C4F2010040F22771FCF7CD
:1047500039FC234B1A68002A38D0224A224C1168AF
:10476000481C802808BF002054F8211010601A68E7
:104770004FF4A050013AC4F2010089B21A60BDE8BA
:104780003840FCF7D5BB4FF4A050C4F2010040F212
:104790002551FCF717FC4FF4A050C4F20100FCF7C0
:1047A000CBFB124B1A687F2AC1D81149114D0A68F8
:1047B000541CC0B27F2C45F8220098BF0C6001D970
:1047C00000220A601A6801321A60B0E74FF4A05064
:1047D000C4F2010040F22771BDE83840FCF7B0BBDD
:1047E000780600206C0600206C040020680400207D
:1047F00070060020800600202DE9F04383B0684653
:10480000FCF728F800260120C4F202060146012424
:10481000FCF7CEF900254FF0800930466946CDF807
:1048200000908DF805508DF804408DF806508DF8F5
:104830000750FBF7B3FF20462146FCF7B9F94FF0CC
:10484000400830466946CDF800808DF805508DF857
:1048500004408DF806508DF80750FBF79FFF204667
:104860002146FCF7A5F910273046694600978DF8D8
:1048700005508DF804408DF806508DF80750FBF771
:104880008DFF304649462246FBF7F4FF304641464D
:104890002246FBF7EFFF304639462246FBF7EAFF98
:1048A00003B0BDE8F08300BFF8B5094D04460F46DC
:1048B000002601E02B6833B92046FFF703FF0028EC
:1048C000F8D00120F8BD0136BE422860F4D3F8BD0F
:1048D000803E00202DE9F04F85B0054603F020FD15
:1048E000FFF712FFFFF7E4FE002843D00024624FD9
:1048F000DFF888A10126A346294603A8FFF7D4FFC5
:10490000DFF874914FF001080346002835D0039B6F
:104910003E600A2B07D00D2BEED0FF2CECD80AF806
:1049200004300134E8E70AF804B0002C32D103F077
:10493000F7FCE1E7514852491A4606F0D2FD00283B
:104940004CD04E484F49032206F0CBFD00284FD0F3
:104950004A484D49052206F0C4FD002855D14B4870
:104960004B49022206F0BDFD002849D10123C9F8B8
:104970000830062005B0BDE8F08F4648019303F0EB
:10498000A1FC454803F09EFC444803F09BFC019BBE
:104990001846EFE73F48019303F094FC374803F0D3
:1049A00091FC3E4803F08EFC34483D49022206F05B
:1049B00098FD38B131483B49052206F092FD18B9FF
:1049C0000220D7E74046D5E72C483749022206F0B7
:1049D00088FD019B0028ADD10320CBE709F13C0005
:1049E00032490F2206F096FDC9F804800420C1E781
:1049F00009F11C002E491F2206F08CFD0520B9E7A5
:104A00000023C9F808300620B4E71C4829490522CC
:104A100006F067FD98B119482749092206F061FDA3
:104A200010B316482549042206F05BFDA8B11348CF
:104A30002349092206F055FD40B1FF209AE721489D
:104A400012490F2206F066FD072093E71E481F4912
:104A5000FF2206F05FFD0A208CE71D481D491F223A
:104A600006F058FD092085E71B4818490F2206F07B
:104A700051FD08207EE700BF80080020FC090020CF
:104A800048C7000854C7000858C70008010A00209A
:104A900060C7000828C700082CC7000834C70008F2
:104AA00038C700083CC7000844C70008060A0020B1
:104AB000FF09002064C700086CC7000878C7000819
:104AC00080C70008EC090020CC080020050A00205F
:104AD000CC090020000A00208C080020F0B583B02B
:104AE000074606F0F6FC06461A4803F0EBFBBEB19B
:104AF0003C46F61904E0184603F0BEFBB4420FD062
:104B000014F8013B1449A3F120055E2D68461A46AE
:104B1000F1D906F09BFC684603F0D4FBB442EFD118
:104B20000E4803F0CFFB03F0FBFB3846FFF7B4FD64
:104B30000B48FFF7B1FDFFF7E7FD02E0022807D0C1
:104B400020B10A20FFF7C6FE0128F7D103B0F0BD5F
:104B50000020FBE78CC70008A0C7000894C7000826
:104B600068C9000838B539B10446451814F8010B76
:104B7000FFF76CFDAC42F9D1BDE83840FFF7C4BD8A
:104B800040F68000C2F20000704700BF10B5002060
:104B9000C4F202008021002282B0FBF76BFE0C4AB7
:104BA0000521144600201368002BFCD00139206039
:104BB000F9D10020C4F2020080210122FBF75AFE45
:104BC00001A83221FFF770FE0028F9D102B010BD14
:104BD000803E002008B502460B460748074906F00C
:104BE00035FC0548FFF77AFF20B1054B002283F81A
:104BF0003C205A6008BD00BF000B0020A8C7000879
:104C00008008002008B502460B460748074906F011
:104C10001DFC0548FFF762FF20B1054B002283F819
:104C20003C205A6008BD00BF000B0020B8C7000838
:104C30008008002008B5024608B1037823B9074868
:104C4000BDE80840FFF74ABF0549064806F0FEFBED
:104C50000448BDE80840FFF741BF00BFE4CD0008AD
:104C6000C8C70008000B002030B54FF4E13083B016
:104C700003F0F0FBFFF7C0FD4FF4E130FFF766FCF7
:104C80000020C4F2020010210022FBF7F3FD1E4CAD
:104C900000200022C4F202008021FBF7EBFD052575
:104CA0002246002321680029FCD0013D1360F9D180
:104CB000002080210122C4F20200FBF7DBFD124933
:104CC00032222368002BFCD0013A0D60F9D100207C
:104CD000C4F2020010210122FBF7CCFD03E001A881
:104CE00003F0FCFA60B901A8FFF7ECFC0028F6D04D
:104CF000019803F0C1FA01A803F0F0FA0028F2D0FD
:104D00000198FFF7A3FCEEE7803E002008B50B4BAF
:104D10001A6802B108BD01224FF4E1301A6003F0B5
:104D200099FB074803F0CEFAFFF766FD4FF4E13038
:104D3000FFF70CFCBDE80840FFF728BF500B002030
:104D4000D4C7000810B403781649FBB100220860EC
:104D50001446013005E001300E2A14DC10F8013C45
:104D60008BB13D2B02BF01EBC20300F8014C586030
:104D7000F1D0262BEFD1013200F8014C41F832007E
:104D800001300E2AEADD531C0F2B08DC002201EB58
:104D9000C30011460133815008320F2BFADD10BCDD
:104DA000704700BFA80B0020F8B50A4D0646002446
:104DB00055F83430E70031461846013423B106F087
:104DC00076FB18B1102CF3D10348F8BD014BDF1965
:104DD0007868F8BDA80B0020F0C8000808B5FFF7F8
:104DE000E3FF4CF6CC01C0F6000106F060FBD0F109
:104DF000010038BF002008BD00B50B4685B04CF659
:104E0000D4010246C0F60001684606F01FFB684662
:104E1000FFF7CAFF05B000BD10B5044606F059FB08
:104E2000014600B910BD2046BDE81040FFF79ABE0C
:104E300010B504464CF6DC00C0F60000FFF7ECFFAE
:104E40004CF6EC00C0F60000FFF7E6FF4CF6F4006D
:104E5000C0F60000FFF7E0FF4CF60010C0F60000BF
:104E6000FFF7DAFF4CF60C10C0F60000FFF7D4FF96
:104E70002046FFF7D1FF4CF61410C0F60000FFF7F4
:104E8000CBFF4CF62010C0F60000FFF7C5FF4CF634
:104E90002C10C0F60000FFF7BFFF4CF63810C0F62C
:104EA0000000FFF7B9FF2046FFF7B6FF4CF64010B1
:104EB000C0F60000BDE81040FFF7AEBF38B50446AD
:104EC0004CF64810C0F600000D46FFF7A5FF20463F
:104ED000FFF7A2FF4CF65410C0F60000FFF79CFF4E
:104EE0002846FFF799FF4CF65810C0F60000BDE8C1
:104EF0003840FFF791BF00BF4CF6F0004CF66C1144
:104F000008B5C0F60000C0F60001FFF7D7FF4CF669
:104F100074104CF67C11C0F60000C0F60001FFF7DB
:104F2000CDFF4DF288104CF68411C0F60000C0F69B
:104F30000001FFF7C3FF4CF690104CF69411C0F639
:104F40000000C0F60001FFF7B9FF4DF200304CF64B
:104F50009811C0F60000C0F60001FFF7AFFF4CF655
:104F6000A0104CF6AC11C0F60000C0F60001FFF72F
:104F7000A5FF4CF6B8104CF6C411C0F60000C0F600
:104F80000001FFF79BFF4CF6D0104CF6D811C0F68D
:104F90000000C0F60001FFF791FF4CF6E010C0F6EC
:104FA0000000BDE80840FFF737BF00BF054A13689F
:104FB00001331360DB0702D40348FFF72DBF03481A
:104FC000FFF72ABF340C0020FCC90008E4C9000820
:104FD00010B504464CF60420C0F60000FFF71CFF95
:104FE0002046FFF719FF4CF60C20C0F60000BDE884
:104FF0001040FFF711BF00BF70B584B00C460546E6
:105000001B49164668461A4606F020FA02A81849B7
:10501000089A06F01BFA3CB123782BB12046FFF723
:10502000FBFE1448FFF7F8FE1348FFF7F5FE28468D
:10503000FFF7F2FE1148FFF7EFFE2846FFF7ECFE00
:105040000F48FFF7E9FE3046FFF7E6FE0D48FFF791
:10505000E3FE6846FFF7E0FE0B48FFF7DDFE02A81F
:10506000FFF7DAFE0948FFF7D7FE04B070BD00BFB6
:105070001CD50008B4D0000814CA00082CCA0008C7
:1050800038CA000844CA000854CA000854C90008B5
:1050900010B504464CF66020C0F60000FFF7BCFED9
:1050A0002046FFF7B9FE4CF69420C0F60000FFF74B
:1050B000B3FE4CF6A420C0F60000BDE81040FFF798
:1050C000ABBE00BF70B505460F480E46FFF7A4FE05
:1050D0000E48FFF7A1FE002E0EDD043D00240C4813
:1050E000FFF79AFE55F8040FFFF796FE01340948C2
:1050F000FFF792FEB442F2D10748FFF78DFE074B4F
:1051000000221A6070BD00BFACCA0008FCC90008CC
:10511000C8CA0008E0CA0008C0CA0008340C002051
:105120004CF6F020C0F60000FFF776BE38B5044616
:105130004CF60030C0F600000D46FFF76DFE20462D
:10514000FFF76AFE4CF65410C0F60000FFF764FE4D
:105150002846FFF761FE4CF62C30C0F60000BDE893
:105160003840FFF759BE00BF08B54CF63C30C0F6DA
:105170000000FFF751FE4CF64830C0F60000BDE8D5
:105180000840FFF749BE00BFF0B5044683B01F4892
:105190001E460D461746FFF73FFE2046FFF73CFE32
:1051A0001B48FFF739FE2046FFF736FE1948FFF788
:1051B00033FE002E24DD043D00240BE01648FFF7EB
:1051C0002BFE55F8040FFFF727FE1448FFF724FEC7
:1051D000B44215D02246124901A806F037F9114809
:1051E000FFF71AFE01A8FFF717FE0F48FFF714FE9E
:1051F000BC4204F10104E1D10C48FFF70DFEDDE7EC
:105200000B48FFF709FE03B0F0BD00BF54CB000808
:105210002CCA000864CB000860CC000894CB0008BE
:105220001CD5000878CB000840CA000888CB0008CD
:105230006CCB000870B50E4605460E481446FFF7C5
:10524000EBFD3046FFF7E8FD0B48FFF7E5FD28468C
:10525000FFF7E2FD0948FFF7DFFD14B10848FFF74B
:10526000DBFD0848FFF7D8FD0748BDE87040FFF7B1
:10527000D3BD00BF04CA0008A0CB0008C4CB0008FF
:10528000D8CB000860CC00080CCA00082DE9F0411A
:10529000069F079D04461646984611B10B78002BD1
:1052A00049D12848FFF7B8FD2046FFF7B5FD26484D
:1052B000FFF7B2FD2046FFF7AFFD2448FFF7ACFD36
:1052C0003046FFF7A9FD2248FFF7A6FD4046FFF74D
:1052D000A3FD2048FFF7A0FD3846FFF79DFD55B11F
:1052E0002B7843B11C48FFF797FD2846FFF794FD44
:1052F0001A48FFF791FD1A48FFF78EFD2046FFF789
:105300008BFD1848FFF788FD2046FFF785FD1648FE
:10531000FFF782FD1548FFF77FFD2046FFF77CFD74
:105320001348FFF779FD3046FFF776FD1148BDE8D9
:10533000F041FFF771BD0846FFF76EFD0E48FFF71D
:105340006BFDAEE7E0CB00082CCA000838CA0008A5
:10535000FCCB000804CC00080CCC00081CCC0008D6
:1053600020CC00082CCC00083CCC000848CC00081D
:1053700058CC000864CC0008B4D000084CF670404B
:10538000C0F600000321FFF7EDBB00BF10B50446D7
:105390004CF60420C0F60000FFF73EFD4CF67441C9
:1053A0002046C0F60001FFF7C1FE4CF6A420C0F66F
:1053B0000000BDE81040FFF72FBD00BF70B50646E6
:1053C0004CF6042082B0C0F600000D461446FFF7EC
:1053D00023FD4CF6F0014CF67C43C0F60001C0F60C
:1053E00000033046009301912A462346FFF74EFF03
:1053F0004CF6A420C0F6000002B0BDE87040FFF7F4
:105400000BBD00BF38B505460C46FFF7CFFD28465B
:10541000FFF7DEFD2046FFF7DBFD4CF6F000C0F69F
:105420000000FFF7D5FD4CF6C020C0F60000BDE837
:105430003840FFF7F1BC00BF10B504464CF6804081
:10544000C0F60000FFF7E8FC2046FFF7E5FC4CF64D
:105450006430C0F60000BDE81040FFF7DDBC00BFBF
:1054600010B50446FFF7A2FD2046BDE81040FFF747
:10547000E3BF00BF4CF6A040C0F60000FFF7CCBC75
:1054800008B5FFF7F7FF4CF6C020C0F60000BDE8F6
:105490000840FFF7C1BC00BFF0B583B00E4614460C
:1054A0001F46089DFFF7DCFF3046FFF791FD4CF6E5
:1054B0000420C0F60000FFF7AFFC4CF6F001C0F688
:1054C00000013A462B4620460095FFF795FD4CF625
:1054D0000C20C0F60000FFF79FFC2046FFF7D8FD28
:1054E00003B0BDE8F040FFF7CBBF00BFF8B5069DA5
:1054F0000E4614461F46FFF7B3FF3046FFF768FD20
:10550000204639462A46FFF795FE2046FFF7C0FDA4
:10551000BDE8F840FFF7B4BF2DE9F0410F4614464F
:105520009846069E079DFFF79BFF3846FFF750FD04
:105530004CF60420C0F60000FFF76EFC41463246F0
:105540002B462046FFF720FE4CF60C20C0F600004C
:10555000FFF762FC2046FFF79BFDBDE8F041FFF737
:105560008FBF00BF2DE9F04F83B08B46924699461E
:10557000DDF830800D9F124EFFF772FF1148FFF7E4
:1055800027FD1148FFF748FC00243D595BF8040053
:105590005AF8041059F8042058F804308DE86000D7
:1055A000FFF774FE04340948FFF736FC0C2CECD1ED
:1055B0000748FFF76DFD03B0BDE8F04FFFF760BF90
:1055C000BCCC0008ACCC0008B4CC0008C0CC0008AF
:1055D00068D300082DE9F04F05460E46C7B0A7482E
:1055E0002946924602F026FF33781BB3741C4FF015
:1055F0002008002706E02B2B08BF04F8018C14F8C4
:10560000013BBBB1252BF6D120460221FBF7A2FDC1
:10561000A27804F8010C002A00F03F85234603F825
:10562000012B9A781946002AF9D10F7014F8013B22
:10563000002BE7D13146924802F0FCFE3046FFF7DE
:1056400081FB28468F4905F032FF002842D02846CA
:105650008D4905F02CFF0446002800F0CB83284636
:105660008A4905F024FF002800F06F842846884905
:1056700005F01DFF0446002800F093812846854967
:1056800005F015FF002800F069852846824905F0DD
:105690000EFF002800F0E2872846804905F007FF4A
:1056A000002800F04D8228467D4905F000FF0028C3
:1056B00000F0F8867B48FFF7AFFB7B48FFF7ACFBB9
:1056C0007A48FFF7A9FB0026FFF758FE304647B09F
:1056D000BDE8F08F764C94E803001AAD04F108069B
:1056E00085E803000FCE3EAF07953D460FC596E80F
:1056F0000300059704F1200785E803000FCF25ADCF
:1057000004F1340E2E460FC6BEE80F003F68089520
:1057100004F1480C2AAD069537600FC5BCE80F00B0
:105720002FAF48343E460FC60FCC0DF1D00844468B
:105730000FC4DCF80030DEF800203360236015A9C8
:105740002A6014A816AA1CAC0DF1600B13AE3C9194
:105750003D920994CDF8E4B03A963B9002F0BCFF3C
:10576000814602F0BFFF5349C0F30742C0F307234D
:10577000099805F06BFE02F0BBFF4269002A04465F
:1057800032DB0369002B2FDBC16800292CDB80682A
:10579000002829DB6568002D26DBB2F5966F23DC37
:1057A0000C2B21DC1F291FDC17281DDC3B2D1BDCEB
:1057B00002F26C725846404905F048FE22693F49A2
:1057C0000132304605F042FEE2683C4914A805F07B
:1057D0003DFEA268394915A805F038FE16A83749DC
:1057E000626805F033FE0AE000238DF860308DF822
:1057F0004C308DF850308DF854308DF8583030489A
:10580000FFF7D2FA0546002801F080802D4905F007
:105810004EFE002841F041802B4C49262B48DFF8F2
:10582000C4A0FFF705FBFFF767FB07980221FFF70E
:1058300049FC27484946FFF7E5FDDAF80030254ADC
:1058400025492648002B18BF1146FFF7DBFDDAF883
:105850000030002B41F01B80FFF762FC0598062109
:10586000FFF730FC1E48FFF7FBFDDA4609954FF0C5
:1058700000090594089DDDF818B038E054CE000802
:1058800068CE000880CE0008A8CF00081CD1000810
:1058900000D2000884D20008BCD3000878D40008E5
:1058A00020D500086CD50008ECC8000884D5000895
:1058B000E8C7000884CE000890CE000894CE000807
:1058C0009CCE0008A4CE0008D8CC0008F4CE000876
:1058D00000CF000888DD000828CD000808CF0008A8
:1058E000F0C800086004002039AB59F803A07548DF
:1058F000FFF792FA58F8094055F809005BF80910CB
:1059000057F8093000945246FFF776FB09F1040975
:105910006D48FFF781FAB9F1140FE5D16B48059C8A
:10592000099DFFF7B5FBFFF7ABFDFFF7F9FB079804
:105930000221FFF7C7FB6648664A67491E270346F0
:105940000097FFF7A9FDFFF7EBFB6148FFF774FD38
:1059500062486349FFF7EAFB62486349FFF7E6FBE9
:1059600062486349FFF7E2FB62486349FFF7DEFBE9
:10597000FFF780FD44B16148FFF74EFA2046FFF77C
:105980004BFA5F48FFF748FA28465A4905F08FFD61
:105990000446002800F0DA84FFF7E6FBFFF7EEFC90
:1059A00094E6584B93E803003EAD85E80300059567
:1059B000FDF7A2FD80465448FFF7F6F9054600289A
:1059C00001F0F881514905F072FD0646002801F00A
:1059D0003F8128464E4905F06AFD0646002801F041
:1059E000158028464B4905F062FD0546002841F028
:1059F000DD814948FFF7F2F910F1000818BF4FF0B8
:105A00000108CAF800804C2600238DF8BC300A2417
:105A1000FBF73AFB0DF13A00FBF744FB002841F09D
:105A200001810A20FBF70AFF013CF3D146AF3F2377
:105A300027F85C3D02F06CFA384982B234A805F0D0
:105A400005FD02F06BFA354982B239A805F0FEFC7B
:105A50003348FFF7EDF9FFF74FFA05980221FFF7FA
:105A600031FB30483946FFF7CDFC2F4834A9FFF70A
:105A7000C9FC2E4839A9FFF7C5FC274A2C4B2949F8
:105A80002C48CDF80080FFF731FDFFF749FB29488E
:105A9000FFF7D2FC1D482849FFF748FB1C4827495F
:105AA000FFF744FBFFF7E6FC002D3FF475AF13480A
:105AB000FFF7B2F92846FFF7AFF91148FFF7ACF945
:105AC0006AE700BF04CA00080CCA0008C4CE000878
:105AD000F0C80008ECCE000820CF0008ACCE0008CB
:105AE00028CF0008B4CE000834CF0008A4CE0008A8
:105AF00040CF000858CF000864CF000870CF0008DE
:105B000010D10008E8C700089CCE000808D20008A1
:105B100010D2000818D200081CD200085CC400088B
:105B200024D2000894C9000834D2000838D20008F2
:105B30003CD2000890C9000854D200086CD200087A
:105B4000914E924D96E8070006F1500320AC84E890
:105B500007000FCB3EAF06F10C0E87E80F009EE862
:105B6000070025AB08930597089F06F1180387E8FF
:105B7000070093E807002AAB0693069F06F124036B
:105B800087E8070093E807000DF1D008303688E871
:105B9000070096E807002B687D4F0DF1E40989E8BE
:105BA00007004BB97B4E3B6A39683A69386B86E827
:105BB0000E000123F0602B60FDF732FC0790FDF72B
:105BC00049FC0A90FDF754FC0B90FDF705FC00F032
:105BD00002000C90FDF7C2FF0990FDF78DFC0D90BF
:105BE0000FA8FDF76FFF6C48FFF7DEF805460028A9
:105BF00000F01187694905F05AFC8346002801F03E
:105C000083802846664905F052FC8346002801F04F
:105C1000FB802846634905F04AFC8346002801F0D2
:105C2000BB812846604905F042FC0646002801F089
:105C30004F8328465D4905F03AFC0646002801F0EE
:105C4000F08228465A49072205F04BFC06460028F8
:105C500001F0DE8228465749042205F042FC064640
:105C6000002801F052832846534905F020FC002605
:105C7000B34610B9DFF878B153267A6B4F4915A8AF
:105C800005F0E4FB4D490A9A16A805F0DFFB4B49E5
:105C90000B9A18A805F0DAFB11AD4849099A10A82B
:105CA00005F0D4FB0DF1480A44499DF83C202846F4
:105CB00005F0CCFB13AF41499DF83D20504605F05F
:105CC000C5FB9DF83E203D49384605F0BFFB3C48EA
:105CD0002F950325CDF8C0A03197FFF7A9F8FFF75E
:105CE0000BF920462946FFF7EDF936483649374A81
:105CF000009516ABFFF7D0FB009532483449354A82
:105D000018ABFFF7C9FB0C9C5CB90D9D002D01F091
:105D10001D818DE800032B480899069A2FABFFF7E9
:105D200021FC079F2C4A1B4B26482C490097042432
:105D30000194FFF7F1FBFFF7F3F921460598284D91
:105D4000FFF7C0F900242B68DA0700F190860134D0
:105D50001035042CF7D1FFF7E3F91A48FFF76CFB75
:105D600015482049FFF7E2F9FFF784FBBBF1000F6C
:105D70003FF412AE1C48FFF74FF85846FFF74CF8B7
:105D80001A48FFF749F807E64CC800082C0C002019
:105D90002C010020980B00209CCE0008ACD20008FB
:105DA000BCD2000884D4000894D40008A4D400080D
:105DB000B4D40008C4D4000808D300081CD50008D7
:105DC000CCD40008B8C90008E0D4000898D4000872
:105DD000E8D40008A8D4000888D4000800D500083A
:105DE00038010020B0D3000870CF000810D100089F
:105DF00034CE0008AB4B93E803000DF1E4090833FF
:105E000089E8030093E807003EAD85E807000595A3
:105E1000FEF7B6FE0546A448AF68FEF7C5FF05F1DC
:105E20000C088246002800F0EA87A04905F03FFBF5
:105E30000646002800F0468650469D4905F037FB8F
:105E40000646002800F0F78650469A4905F02FFBD9
:105E50000646002800F00E875046974905F027FBBC
:105E6000002800F057852646B24604F063FD9349AA
:105E7000024634A805F0EAFA9148FEF7D9FFFFF789
:105E80003BF805980321FFF71DF98E4805F13C0109
:105E9000FFF7B8FA41468C48FFF7B4FA8B48FFF792
:105EA000DFFA8B48FFF794F88A48FEF7B5FF4FF00A
:105EB0000F08894849463A460223FFF765F98749A2
:105EC0008748CDF8008005F11C022023FFF794F8E5
:105ED0008448FEF7A1FF14238349844A8448009331
:105EE0004023FFF789F88348FEF796FF8248FFF7C3
:105EF000CFF8FFF7C5FA04F03FFD8049804ACDF89E
:105F0000008003467148FFF7C7FA03237D497E4AA4
:105F10006E48009334ABFFF7BFFAFFF701F96B4807
:105F2000FFF78AFA64487949FFF700F9FFF7A2FA08
:105F3000002C00F0FC817648FEF76EFF2046FEF74D
:105F40006BFF7448FEF768FF26E5734B93E8030088
:105F50000DF1D00888E803005348FEF725FF0446FA
:105F6000002800F0EA846D4905F0A1FA06460028F1
:105F700000F04E8620466A4905F099FA0646002848
:105F800000F0A5862046674905F091FA002840F008
:105F9000D484654D5726654B1B68002B00F05E8549
:105FA00004F06EFA0DF1E4090446620848464349DC
:105FB00005F04CFAE70700F1B286484605F089FA89
:105FC0005B4B09EB000201469C8818689B7949F8F5
:105FD000010094809371574B1B68002B00F03585AE
:105FE00004F0E4FB3EAF04466208384633490597A7
:105FF00005F02CFAE40700F19F86059805F069FA90
:10600000059C4B4B059F221801469C8818689B797C
:1060100078509480937104F023FA0246002840F0EF
:10602000738546AF07F85C0D04F010FC02460028AB
:1060300040F0628546AC04F8700D06943E48FEF7C9
:10604000F7FEFEF759FF40460221FFF73BF83B48B9
:106050004946FFF7D7F9022439480599FFF7D2F9E5
:1060600038483949394A00943B46FFF715FA384910
:10607000384A069B33480094FFF70EFAFFF750F8B2
:106080003048FFF7D9F927483349FFF74FF8FFF7B2
:10609000F1F9002D7FF40BAD7EE421460F70FFF780
:1060A000C5BA00BF44C800089CCE0008B4CF0008A1
:1060B00050D0000860D0000870D000081CD500083F
:1060C000D4CF000878D0000884D0000874C9000834
:1060D00098D0000804CA0008C0CF0008A0D000086B
:1060E000CCCF0008A8D00008BCD00008F0C8000839
:1060F00094DE00080CCA0008B8CF0008C0D0000821
:1061000054D00008CCD0000864D00008E0D00008CB
:10611000F0D000080CD10008E8C700082CD1000816
:106120003CD100084CD10008ECCD0008D81200206A
:1061300064D100084C0400206CD1000884D1000810
:1061400094D1000888D100089CD1000830D1000803
:10615000C4D1000840D10008ECD10008A94B93E855
:10616000070003F10C0425AE86E8070094E8070059
:106170002AAD03F1180485E8070094E807002FAF63
:1061800003F1240487E8070094E8070030330DF199
:10619000E40989E8070093E8070008963EAE86E820
:1061A000070006950596FDF771F90B90FDF714F9B8
:1061B0000546FDF7F5F90C90FDF7A8FC8046FDF7C4
:1061C0009BF9914C0D9016A8FDF758FC236805F03B
:1061D0000102C5F3400B0792002B00F06B838B4844
:1061E000FEF7E2FD0446002800F00186884905F02C
:1061F0005EF9002800F066832046864905F057F9CD
:10620000002840F0A4858448FEF7E8FD002800F04F
:106210001C86012645F002050996CAF8005047265B
:1062200020467E4905F043F90546002800F06085C8
:1062300020467B4905F03BF9002840F0A685794DC2
:10624000DFF85CA20A9558260DF1600B42467649AC
:106250000DF16808584605F0F9F81CAD72499DF833
:106260005820404605F0F2F81EAC6F499DF85920C1
:10627000284605F0EBF89DF85A206B49204605F0BA
:10628000E5F80A9BCDF8D0801A6835953694002A37
:1062900040F0278546AC04F8982D6448FEF7C8FD09
:1062A000FEF72AFE08980321FEF70CFF079D6048C1
:1062B0006049614A614B0095FFF718F90B9D5C48F6
:1062C000009504255E495F4A5F4B0195FFF724F96D
:1062D000099D574800955D494F4A5D4BFFF706F908
:1062E0000D9D002D00F0D5840C9D002D00F0E38461
:1062F0000223584A58494E4800932346FFF7CCF8EA
:10630000FEF70EFF4A48FFF797F854485449FEF746
:106310000DFF54485449FEF709FF41485349FEF721
:1063200005FF53485349FEF701FFFFF7A3F8BAF101
:10633000000F3FF431AB5048FEF76EFD5046FEF7BC
:106340006BFD4E48FEF768FDFFF726BB4C48FEF795
:1063500063FDA0461EAD20AC42464A49284605F0E2
:1063600075F82846FEF758FD4748FEF755FD4046AC
:1063700021461022FEF79EF800283DD000270CE0B1
:10638000E25D284605F062F82846FEF745FD013734
:106390003E48FEF741FD102F0BD007EB0803B3F585
:1063A000A27F3B493B48EBD90137FEF735FD102F63
:1063B000F3D13648FEF730FD002320212E2003EBD9
:1063C0000802B2F5A27F88BFE15404D8E25C203A0B
:1063D0005E2A88BFE0540133102BF0D10023204601
:1063E0008DF8903008F11008FEF716FD2A48FEF7E8
:1063F00013FDB8F5A87FAFD12848FEF70DFDFFF7D4
:10640000CBBA00BF4CC80008280C00209CCE000866
:1064100090D200089CD20008A0D20008ECD200085C
:10642000FCD20008BC0300201CD5000810D30008D3
:1064300000D3000824D3000894D200082CD300080D
:106440004CD30008E0D20008540B0020C4C9000857
:106450005CD30008F0D2000888D30008ACCE000856
:1064600028CF0008B4CE000834CF0008A0D300081D
:1064700008D30008B0D3000870CF000810D100087E
:1064800088CF000890CF000898CF0008D4CB000830
:1064900070DC0008A4CF000868C900089CCF000881
:1064A00020CE0008B34D0FCD3EAC05940FC495E847
:1064B0000F0084E80F00B048FEF776FC044630B1C8
:1064C000AE49062205F00DF8002800F03A82DFF808
:1064D00030B30DF1E409AA48FEF7AAFC25ACFEF79B
:1064E0000BFD05980821FEF7EDFD1AAD08941CACD4
:1064F0004FF0000A079509942AAD20AC0695564640
:106500002FAF0DF1D0081EAD05940BEB0A0C48F629
:106510008904DCF804209B49CDF80CC0C8F6880437
:10652000A4FB02025209099804F090FFDDF80CC0A8
:106530009449DCF80420A4FB02035B09C3EB0313BA
:10654000A2EB8302284604F081FF8F48FEF788FF04
:1065500032468E49079804F079FF32468C490598F7
:1065600004F074FF32468B49089804F06FFF3246FE
:106570008949069804F06AFF32468849384604F093
:1065800065FF32468649404604F060FF0798FEF7F3
:106590001FFD5BF80A2083490898C2F3C012FEF77A
:1065A00049FE5BF80A207F490698C2F38012FEF785
:1065B00041FE32467C49484604F048FF5BF80A2019
:1065C0007A48C2F3C204FEF727FC07232246784923
:1065D0004846FEF7D9FD7748FEF71EFC324676495D
:1065E000484604F033FF5BF80A20704802F00704C5
:1065F000FEF712FC224607236D494846FEF7C4FD0C
:106600006C48FEF709FC02246848FEF705FC654962
:10661000099A009423463846FEF7EEFC6548FEF7DB
:10662000FBFB6248FEF7F8FB5E4900942A462346CE
:106630004046FEF7E1FC5F48FEF7EEFB01360598A9
:10664000FEF726FDFEF71CFF082E0AF1080A7FF46C
:106650005CAFFEF765FD0026FFF79EB9574F584D1A
:1066600097E8070007F13C040DF1D00888E807001F
:106670000FCC3EAE503705960FC697E80F00246842
:106680002F6834600DF1E40989E80F00002F00F055
:106690002981DFF870B1FCF74BFF0746FCF780FF5C
:1066A00005463548FEF780FB0446002800F0CA8303
:1066B000444904F0FCFE0346002800F0CE82204648
:1066C000414904F0F4FE0346002800F07D83204693
:1066D0003E49032204F005FF0646002800F07784B7
:1066E00020463B49062204F0FCFE0646002800F046
:1066F000C48420463749072204F0F3FE06460028EA
:1067000000F0A28420463449042204F0EAFE064642
:10671000002800F064852046304904F0C8FE0026B9
:10672000B24610B9DFF8E0A053262D48DFF8D4B008
:10673000FEF77EFB0B24FEF7DFFB40460321FEF74E
:10674000C1FC28482849294A294B01940097022472
:10675000FEF7E2FE2749284A284B2248019400957B
:10676000FEF7DAFEFEF7DCFC05980521FEF7AAFC31
:10677000002451E0ACC800089CCE000828D50008D1
:1067800040D5000894CE0008D0C900081CD50008E8
:1067900054D500085CD5000860D5000864D5000811
:1067A00068D50008F0C8000838D5000804CA0008F9
:1067B000100000200CCA00083CD500084CC8000896
:1067C000300C0020C8D30008D8D30008ECD3000850
:1067D000F0D3000808D4000818D4000808D3000833
:1067E00020D40008A0C9000838D40008CCD3000881
:1067F0006C0B002044D40008DCD30008640B00209C
:10680000A83E00205000002034CE000801340B2C9C
:106810000BF1140B00F00381DBF81030D807F5D52D
:106820002246BD491AA804F011FE2246BB491CA805
:1068300004F00CFE2246BA491EA804F007FE2246C8
:10684000B84920A804F002FEDBF80820B64918A8D1
:1068500004F0FCFDB548FEF703FEDBF80000FEF790
:10686000B7FB18A91CA8B24AFEF7A8FD1EA8FEF7A0
:106870008DFDDBF81020AF49C2F3400220A8FEF7DF
:10688000D9FC1AA8FEF704FCFEF7FAFDBEE7AA48F9
:106890000999FEF7B7FDFEF7DFBF2846A74904F0C8
:1068A00006FE00283CD10123CAF800305026A44C33
:1068B000FEF7B4BFA34BA44E0FCB86E80F00012315
:1068C00023608CE4A148FEF789FA002800F0598281
:1068D000012645F001050796CAF80050CDF824B00E
:1068E00047269DE49A4ADFF8C8B23B4653F80B109E
:1068F0001433DC2B42F8041FF8D1964B96491A68E2
:106900001B6981E80C0001232B60C4E6064604469F
:10691000FEF784BFDFF89CA24E260446FFF7A5BA17
:1069200028468E4904F0C3FD002840F02183CAF8B0
:10693000000050268A4CFEF771BF00263546FFF74F
:106940002ABBA01D04F03CFA072804463FF6BFAD61
:1069500001468448FEF750FA834904F0A8FD002858
:1069600000F05C83DFF850B25BF8343023F0800332
:106970004BF8343021467D48FEF73EFA7A4904F060
:1069800096FD002800F043835BF8343023F0400389
:106990004BF834300DF1E40922467549484604F0BD
:1069A00055FD4846FEF700FA04F00AFA22467149FE
:1069B0000546484604F04AFD4846FEF7F5F904F05E
:1069C000FFF95BF83430ED0000F0070023F03F03DF
:1069D00040EA030205F0380313434BF834302146F4
:1069E0006548FEF709FA04F0EBF9214605466348CD
:1069F000FEF702FA04F0E4F90BEBC404C5EB05154D
:106A000000EB8500606003F025F864E501F0A8FA6A
:106A10005B4DFEF7F9BF06468346FFF72EB9FEF73A
:106A20007FFB48460421FEF74DFB564D00242B68A2
:106A3000D90700F1C38001341035022CF7D1FEF7DD
:106A40006FFB3A48FEF7F8FC6BE44F4B93E803000A
:106A50003EAC059484E80300FFF7DDBA4A4B93E8A7
:106A600003000DF1E40989E80300FFF7B4BA2246F8
:106A700046491AA804F0EAFC224645491CA804F03D
:106A8000E5FC224643491EA804F0E0FC55F8082C1A
:106A9000254914A804F0DAFC3F48FEF7E1FC55F85C
:106AA0000C0CFEF795FA14A93C4A1CA8FEF786FCCC
:106AB0001EA8FEF76BFC1AA8FEF7EAFAFEF7E0FC48
:106AC000FFF745B93648FEF76FF904F079F9074644
:106AD0003448FEF769F982463348FEF765F9044603
:106AE000002F00F0B78104F0F4FC092800F2CC81FB
:106AF0002E4CB246FFF7B9B92AAC20460A49069493
:106B000004F0A4FCFFF79ABA2FAF3846064904F008
:106B10009DFCFFF789BA00BF54D40008F8D30008E1
:106B20005CD4000800D400081CD50008A0C90008E7
:106B300064D40008F0C8000810CF0008ACCE0008EC
:106B4000F8CC0008AC010020540B002094D20008BF
:106B5000680B00207C010020640B0020B4CE0008EC
:106B600010CD000830D50008CCC8000834D5000886
:106B700038D500083CD50008DCCE00086CD80008E9
:106B800008CE00088801002028CD000810D5000894
:106B9000BCD4000818D50008B8C9000884D3000880
:106BA000C0CF0008CCCF000894DE000830CD00082C
:106BB00050000020D8CD0008A83E00202246BF4942
:106BC00025A804F043FC2246BD492AA804F03EFC57
:106BD0002246BC492FA804F039FC55F8082CBA49C4
:106BE00016A804F033FCB948FEF73AFC55F80C0C33
:106BF000FEF7EEF916A9B64A2AA8FEF7DFFB2FA882
:106C0000FEF7C4FB25A8FEF743FAFEF739FC12E7AE
:106C1000B048FEF7C9F804F0D3F803F027FC354676
:106C2000FFF7B9B92FAF3846AB49BDF83A2004F0A9
:106C30000DFCFEF7FFBEA948FEF7B6F803F0A2FE72
:106C4000002800F0BB803446DFF8ECA2FFF70DB956
:106C500001F06AF9A24DFEF7D7BEA2480493FEF7F1
:106C6000A3F804F0ADF8CAF80000049B07464126DB
:106C70009A465AE59C48FEF797F804F0A1F803F00D
:106C80005FFE002800F0AD803446DFF8B0A2FFF7C9
:106C9000ECB89648FEF7E4FB9548FEF799F98C4A64
:106CA00094485946FEF78AFB9248FEF7F1F9FEF741
:106CB000E7FBFFF719BB059DCDF8009001958B48C8
:106CC00006993A4634ABFEF74DFCFFF711BB8A48F4
:106CD000FEF76AF804F074F803F0BEFD3546FFF7DE
:106CE0005AB920AC2046784904F0B0FBFFF7D5BA7A
:106CF000824B83480A93FEF757F804F061F80A9C28
:106D0000AA462060FFF7A0BA7A48FEF74DF804F0D3
:106D100057F862260990CAF80000FEF7AEBF484651
:106D200004F0D7FB774B09EB000219889B7829F810
:106D300000109370FFF741B9059804F0CAFB714B3E
:106D40003A1819889B7839529370FFF756B9204644
:106D50006D4904F0ACFB002800F04C8120466B49E3
:106D600004F0A5FB002800F0BC812046684904F02F
:106D70009EFB002800F05B81CDF824B00026FFF7D1
:106D80004FBA25F001050790A6E52046614904F0B9
:106D90008EFB002840F00B81584D0123CAF80030CB
:106DA0005026DFF89CA10A95FFF74EBA26462546E5
:106DB000FEF72ABE06460546FEF726BE06460446F0
:106DC000DFF880A1FFF751B853480493FDF7ECFFBB
:106DD00003F0F6FFCAF80000049B054646269A46D3
:106DE000A3E406460446DFF860A1FFF73EB8434B34
:106DF000CDF824B0064682460A93FFF725BA064628
:106E000004468246FFF731B84448FDF7CDFF03F052
:106E1000D7FF8DF83C004248FDF7C6FF03F0D0FFD6
:106E20008DF83D003F48FDF7BFFF03F0C9FF8DF827
:106E30003E000F9B1A0CAAF800308AF80220632645
:106E4000FEF71BBF064682466FE425F00205099057
:106E5000FFF7E3B93448FDF7EBFF3448FDF7DCFFFB
:106E6000FEF782F9FEF78AFA4FF4FA70FAF7E6FCB9
:106E70002F4B6F6085F83C70504621461F603E46A0
:106E8000FDF7A8FEFEF722BC2748FDF7D1FF2948F1
:106E9000FDF7C2FFFEF768F9FEF770FA4FF4FA70DB
:106EA000FAF7CCFC224B6E6085F83C6050462146D8
:106EB0001E60FDF7A7FEFEF709BC00BF68D40008FE
:106EC00010D4000870D400081CD50008A0C9000820
:106ED00084D3000830D100085CC4000854D00008F6
:106EE00008CE0008CCD3000864D0000800D3000806
:106EF00070D30008D8E1000840D10008BC0300208E
:106F0000F0D2000860D10008ACD20008BCD2000862
:106F1000DCD20008ACCE0008DCD30008C8D20008E0
:106F2000CCD20008D4D20008D4CF0008E8CF0008A3
:106F3000F81100201CD0000850CD000898CD0008A2
:106F4000F8CC000874CD0008B8CD0008C248FEF7A0
:106F500087FAC248FEF73CF8C14AC24810A9FEF7BA
:106F60002DFAC048FEF794F8FEF78AFAFEF7D1BE74
:106F70002846BD4904F09BFA0A90002800F0D18011
:106F80002846BA4904F093FA0446002800F03581F7
:106F900000263446FEF742BCB548FDF705FF03F076
:106FA0000FFF64260790CAF80000FEF766BE204671
:106FB000B04904F07CFA002840F03E81AE4BCAF89C
:106FC00000005026DFF800A30A93FFF73DB9E01C4C
:106FD00003F0F6FE0A280AD800EB80000BEB800BCA
:106FE000B246DBF80C30CBF80830FFF79EBBB24658
:106FF000FFF79BBB9B48FDF7D7FE03F0E1FE42265F
:107000008046CAF80000CDF824B0FFF709B95BF854
:10701000343043F040034BF83430BBE4DFF8ACB21B
:107020005BF8343043F080034BF83430A2E49348EB
:10703000FDF7BAFE03F0C4FE44260B90CAF8000028
:10704000CDF824B0FFF7ECB8E01D03F0B9FE01283D
:107050000446CCD802468A492AA804F0F7F92AA89F
:10706000FDF7A2FE03F0ACFE0F28C0D8854B03EB62
:107070000414B2466060FFF758BBA01D03F0A0FEE9
:107080000A288246B3D802467F4920AC1CA804F0E7
:10709000DDF97E495246204604F0D8F91CA8FDF7D8
:1070A00083FE03F08DFE431E0E2B4FEA8A069CBF23
:1070B00006EB0A030BEB8303564498BF9860204607
:1070C000FDF78CFE0BEB860B002800F02A81DBF825
:1070D0001030002643F00203CBF81030B246FFF721
:1070E00024BB6B48FDF760FE03F06AFE8DF8580084
:1070F0006848FDF759FE03F063FE8DF859006648B5
:10710000FDF752FE03F05CFE8DF85A00169BCDF899
:1071100024B01A0CAAF800308AF802204326FFF7A0
:107120007FB85E48FDF740FE03F04AFE03465C4828
:107130000493FDF739FE03F043FE84465948CDF829
:107140000CC0FDF731FE03F03BFE04465648FDF748
:107150002BFE03F035FE0B905448FDF725FE03F09F
:107160002FFE049B0C901A465149584604F06EF9C4
:10717000DDF80CC04F496246304604F067F92246FC
:107180004C4914A804F062F94A490B9A15A804F076
:107190005DF948490C9A16A804F058F90B9E049B17
:1071A000DDF80CC0CAF808600C9ECAF80C40CAF89A
:1071B00004600A9EA3F26C710CF1FF32CAF81C1035
:1071C000CAF81020CAF80060204661461A46F9F74E
:1071D00087FF5426CAF818000A9CFEF71FBB201D23
:1071E00003F0EEFD01283FF602AF264B03EB001340
:1071F000B2469A685A60FFF798BA2F48FDF7D4FD57
:107200001E220146504604F085F97026FEF706BBA3
:10721000E81D03F0D5FD0328054664D9B346FEF703
:107220002CBD2648FDF7C0FD03F0CAFDFCF726F98A
:10723000B3460B90FEF721BD20460F4C20490A941F
:1072400004F035F91F4B00280CBF9A464FF0000A96
:1072500008BF5326FEF7F8BFB8C9000870D300086E
:1072600084D30008D8E10008C0CE0008E8CE0008AA
:1072700088D40008B4CE0008BC030020E0D2000887
:1072800010D400087C010020F8D3000800D40008C6
:10729000C8D20008CCD20008D4D20008D0CE000852
:1072A000D8CE0008E0CE000884E10008E4CE000853
:1072B00090CE000894CE0008ECCE0008A8D40008B8
:1072C00008D3000834CE000810CD0008A83E0020E6
:1072D0001948FDF769FD03F073FDFCF7C1F8B346EB
:1072E0000A90FEF7CABC024614491CA804F0AEF886
:1072F0001CA8FDF759FD03F063FD0F288ED807EB9E
:107300000515B3466860FEF7B8BC281D03F058FDAC
:10731000032883D807EB0013B3469A685A60FEF738
:10732000ACBCDBF8103023F002030646CBF810307B
:107330008246FFF7FAB900BF98D40008BCD4000811
:1073400030B585B04FF480446846F9F759FB002208
:10735000200448F2A063C0F201030121ADF804202B
:10736000ADF8082040F4B8404FF480624BF6FF754A
:10737000ADF80650ADF80A20ADF80C400093F9F7CF
:107380004DFB200440F4B8406946F9F7C9FA05B04E
:1073900030BD00BF10B54FF4B844C4F2000420461D
:1073A0000121F9F757FB20460121F9F779FB204627
:1073B0000021F9F775FB2046F9F77AFABDE810408D
:1073C000FFF7BEBF70B505460E4643F2010401E06B
:1073D000013C13D04FF4B8402946C4F20000F9F73D
:1073E00073FB0028F4D04FF4B840C4F200003146DB
:1073F000F9F76AFB0028EBD0012070BDFFF7CAFF48
:10740000204670BD38B5054619B1BDE83840FFF7D4
:10741000D9BF43F2010401E0013C0AD04FF4B84067
:10742000C4F200002946F9F74FFB0028F4D00120F0
:1074300038BDFFF7AFFF204638BD00BFF8B507469F
:107440004FF4B840C4F200000E46012115461C4618
:10745000F9F7F2FA0120C1F200000021FFF7D2FF94
:10746000002832D04FF4B840C4F2000034BB0121F0
:10747000F9F708FB4FF4B844C4F200042046F9B20F
:107480000022F9F7F5FA0220C1F200000021FFF70F
:10749000B9FFB8B18020C1F200000021238BFFF7B3
:1074A000B1FFA8B125B1C6F307212046F9F706FBC5
:1074B0002046F1B2F9F702FB0020F8BD0021F9F7F0
:1074C000E1FAD7E76FF00100F8BD4FF0FF30F8BDEB
:1074D0006FF00200F8BD00BF30B5284B1C6883B0C8
:1074E0000CB103B030BD012568461D60F9F7B2F953
:1074F00029464FF40000F9F769FB28462946F9F7B9
:1075000057FB04202946F9F753FB29464FF40000A6
:10751000F9F778FB21464FF40000F9F773FB0020E0
:1075200008210422C4F20200F9F7AAF94FF400601E
:1075300004220921C4F20200F9F7A2F90223002073
:1075400069468DF804308DF80530C4F202004FF41E
:10755000807300938DF806508DF80740F9F71EF9F7
:107560004FF400604FF40073C4F2020069460093C8
:10757000F9F714F9FFF7E4FEB3E700BF380C002079
:107580002DE9F041069D6F1E1E467B427B418046E1
:10759000FFF754FF074610B13846BDE8F081802060
:1075A0000421C1F20000C1F20001FFF70BFF002827
:1075B0005BD04FF4B844C4F2000420460121F9F72F
:1075C0003BFA0120C1F200003946FFF71BFF0028FB
:1075D0004ED020465FFA88F10122F9F749FA0220DD
:1075E000C1F200003946FFF70DFF002843D0238B7E
:1075F0008DB33C4611E040200021C1F20000FFF7AE
:1076000001FF18B34FF4B840C4F20000F9F758FA7C
:107610003219AC4202F8010C1DD00134AC42EAD15F
:107620004FF4B840C4F200000021F9F72BFA4FF4F0
:10763000B840C4F200000121F9F70CFA4020002103
:10764000C1F20000FFF7DEFE0028DBD16FF0060775
:107650003846BDE8F0814FF4B840C4F20000012183
:10766000F9F710FA3846BDE8F0816FF0030793E7A9
:107670006FF0040790E76FF005078DE770B51C46C3
:107680000023FFF7DBFE064608B1304670BD8020C0
:10769000C1F200003146FFF7B5FE28B3049BD3B119
:1076A000049BE51801E0AC4215D04FF4B84014F843
:1076B000011BC4F20000F9F701FA80200421C1F295
:1076C0000000C1F20001FFF77DFE0028EBD16FF052
:1076D0000306304670BD4FF4B840C4F200000121EB
:1076E000F9F7B8F9304670BD6FF00206CDE700BF7C
:1076F00070B43A4A3A49546A0B689C4207D8956A72
:10770000AB4204D2D56B002D4FD0364D13E0D46A76
:10771000324DA34208D21268032A15D0052A20D080
:1077200001330B6070BC70472E6BB342F3D2ED6B2C
:10773000002D40D02C4D2E681C1B00FA04F426436B
:107740002E601268032AE9D1102BE9D9142BE7D84F
:10775000264AA3F11105146800FA05F004431460E9
:10776000DEE7A3F11402032A16D9A3F11804032CAF
:1077700027D81F4C256800FA02F215432560DA0865
:1077800010BB1C4803F00704855C012606FA04F4CC
:1077900025EA04048454C3E7134AA3F108051468D6
:1077A00000FA05F52C431460E9E70E4C256840EA21
:1077B00045052560AFE70C4C256840EA4505256086
:1077C000A9E72F2BACD8DAE70A4803F00704855C59
:1077D000012606FA04F42C438454A1E7640C00202B
:1077E0004C0C0020A80C0020C40C0020BC0C002075
:1077F000C00C00203C0C002000B583B06846F9F7AF
:1078000029F804200121F9F7D3F94FF4006000238F
:107810004FF48062C4F20200694600928DF8043091
:107820008DF805308DF806308DF80730F8F7B6FF83
:1078300003B000BD70B4294A1368002B2BD028492F
:107840000B68022B17D0032B264B26D0264C0E6834
:107850002168264DA0F8011019680670A0F80310E1
:107860002E680021196046712160012029600023E3
:10787000136070BC70471B4B1D681C68E443E4B286
:10788000B4EB152F1BD0184C266848F2EE75AE42AB
:107890001AD00020EBE71846EBE71D681C68E443AC
:1078A000E4B2B4EB152FF4D11D680F4CEDB21D609E
:1078B0000F4D2E681D6845EA06251D60C7E71D6847
:1078C000094CEDB21D60C2E70B250D601D68C5F3C4
:1078D000072525601D68EDB21D60B8E7CC0C0020BF
:1078E000440C0020480C0020B00C0020B40C0020F8
:1078F000540C00202DE9F0474FF400609E4CC4F278
:1079000002004FF48061F8F7AFFF236893B99B4EF4
:10791000356895B99A4B002800F0C2801B68002B8F
:1079200040F00C81974B1A684FF6FE718A4201D8DD
:1079300001321A602068BDE8F087934F3A68002A48
:1079400070D0002800F0B280904A11780131C9B29D
:10795000E929117000F206818D4B8E495A6B096836
:107960008A42E7D1996B0029E4D1DFF868828A491D
:10797000D8F800C00D68AC4500F078818748002732
:1079800007601B68012B00F06481052B00F07981F2
:107990000A2B18BF292B03D10068C00700F15581BD
:1079A0000120022B206040F09C81002A40F00282DE
:1079B00074480368B3F5E16F80F01682784D794F13
:1079C000D5F800903B68DFF8F4A1C1F800C049F099
:1079D0000109C5F80090CAF8003002606546724A95
:1079E0003B6002201060714A1360714B1A68714B42
:1079F0001D60714B1A60236863B10B689C4500F0F1
:107A0000BA816E4A5F481568664FC8F80030002397
:107A10003D6003605A4A002313605C4A33600B6088
:107A2000137087E7664F3B68002B00F08180584B4E
:107A3000002840F0D1801A68032A00F05581DFF851
:107A40004C81DFF83C915A68D9F8001050488A42BE
:107A50000BD88268914208D898F800C0C268944553
:107A600003D30269944540F2B3815B69484A994265
:107A70000BD39369994208D898F80010D3699942BA
:107A800003D3136A994240F2A9810025356088F832
:107A900000500123C9F80030002D3FF44BAF5BE7E5
:107AA0001A6801321A602068BDE8F087DFF8D090CC
:107AB000DFF8D880D9F80030A3F11F020A2A17D8BE
:107AC00098F80020052A13D90A2A11D83D493048D0
:107AD000442203F0D1F92F4A002313600122C9F890
:107AE000002088F800303B60002D3FF423AF33E7DF
:107AF000A3F15E02532A08D898F800202D2A00F23C
:107B00009F80162A01D93049E1E7A3F13C020F2AF0
:107B100040F28980283B162B00F28F8098F80030C5
:107B2000122B40F28A801F2B00F287802749CEE774
:107B3000E8B9134B1A6801321A600DE7204B124A5C
:107B40001D6001231360144A336015601B4A1560E1
:107B50001F4A1560164A15600E4AFF2111600B4A34
:107B60001370E7E6064933600B601370E2E6074ADC
:107B700001233B601370EFE6CC0C0020500C00207A
:107B8000C80C0020580C0020AC0C0020600C002019
:107B9000640C00204C0C0020C40C0020B80C002009
:107BA000B40C0020C0010020440C0020B00C0020C8
:107BB000BC0C0020480C0020540C0020A80C002015
:107BC0005C0C002024D60008F0D6000868D6000817
:107BD000C00C0020BC0100208C49D3F83490D1F8AF
:107BE00000C0E14500F09180DFF854821A6898F8EF
:107BF00000A087480AF1010A5FFA8AFA012A88F888
:107C000000A000F09A80BAF1E90F7FF645AF09F1C4
:107C1000FF32944500F0C4807E4A00233360136035
:107C200088F8003086E698F800203B2A7FF672AF8D
:107C30004B2A3FF66FAF784949E7002535604AE7A0
:107C4000592A3FF662AF754941E775480023036042
:107C5000D1E60268013A012A88BF2360F5D9714A4A
:107C6000714812680360714B1A60BEE66C48006888
:107C7000B0F5966FBFF482AE6D48076801370760B4
:107C80007FE60368012BE0D001232360694B1F7856
:107C900058789A7887EA000909F00F0989EA1717D6
:107CA00087EA101002F00F09814501D00020206002
:107CB00093F803901F79587982EA09037B40984230
:107CC00001D0002323605C4B5C4A1F681068554A52
:107CD00038431860544B126805201860534B1A60E3
:107CE00083E6052BD2D0BAE748490A68102A7FF408
:107CF000A6AEDFF82091D9F80020053A072A79D9F5
:107D00004F4B306018700546C3E6986B01287FF42E
:107D10006BAFDFF800915869D9F80010884205D898
:107D20009869814298BF9A637FF6B6AE444A0023B1
:107D30003360C9F800301370FCE5BAF10B0F7FF621
:107D4000ABAEBCF10A0F7FF65EAFDFF8D890C16A28
:107D5000D9F80020ACF10B0A614442EA0A220CF186
:107D6000010C0131C9F800200A22C0F834C00163B7
:107D700088F8002065E62B48324F05683A682848A5
:107D8000AA427FF442AE026840F6C90C62459FBF2A
:107D9000294AD2F800C04CF0010CC2F800C034E609
:107DA0009B6B002B7FF438AFC1F80090002D3FF49F
:107DB000C1ADD1E51B4B234F1B6810E60A200F3ADB
:107DC0002021186010200F2AD8621963596305D842
:107DD0000120FFF78DFC00233B605AE60020FFF7EF
:107DE00087FC00233B6054E6174B164F1A600D4B7F
:107DF0001B68F4E5124A12783B2ADFD94B2ADDD8FA
:107E000000233B6011230B6043E600BF4C0C0020B5
:107E1000640C0020C80C002034D70008ACD6000841
:107E2000580C0020A80C0020440C0020B00C0020AE
:107E3000B80C00203C0C0020B40C0020C00C00202A
:107E4000600C0020C0010020CC0C0020F9F71CB908
:107E500010B582B004460DF10600F9F723F978B1A8
:107E6000084B09491B88BDF806200988D21AC2EBC5
:107E70000212CB1A92FBF3F30F2B28BF0F232360C0
:107E800002B010BDD00C0020D20C002008B50F4B62
:107E90001B686BB1FF23C0F2020398420AD80C4B57
:107EA00000221A800B4B40F2FF321A80012008BDDD
:107EB000184608BD02220649E120FCF7FBFAE32040
:107EC00004490222FCF7F6FA012008BD60040020F4
:107ED000D00C0020D20C002008B50A4B1B680BB94F
:107EE000002008BDE12008490222FCF7FDFA002825
:107EF000F6D00222E3200549FCF7F6FA003018BF5D
:107F0000012008BD60040020D00C0020D20C00200D
:107F100040F6D043C2F200031888704740F6D243BF
:107F2000C2F200031888704710B582B0F9F7ACF8B8
:107F30000A240DF10600F9F7B5F840B90A20F9F75F
:107F40007DFC013CF5D1054C208802B010BD034CEE
:107F5000BDF806302380FFF7BFFFF5E7D00C002007
:107F600010B582B0F9F790F80A240DF10600F9F780
:107F700099F840B90A20F9F761FC013CF5D1054CAC
:107F8000208802B010BD034CBDF806302380FFF7F7
:107F9000A3FFF5E7D20C0020F9F71CB8F0B50746AF
:107FA0008DB00A20FCF796FC092828D00A2813D0A7
:107FB000072803D0002420460DB0F0BDFCF7E0FDFB
:107FC0000A2201A900F5B67003F0D2FB014638463B
:107FD00002F0EAFC7424EEE7FCF7D2FD00F14C0459
:107FE0002021204603F056FA014610B1002301F883
:107FF000013B20463A46FDF7EDFA0446DBE7FCF785
:10800000BFFD01AE00F5A674002502E002340A2D82
:1080100012D0237820460221002B7BD06378002BDE
:1080200078D0F9F797F8A37846F8040F0135202B9C
:10803000ECD103340A2DECD1029CA4F141032F2B87
:10804000B8D801A252F823F009810008098100087C
:108050006381000809810008B57F000809810008D4
:1080600009810008B57F0008B57F0008B57F0008CA
:10807000B57F000809810008B57F00081D81000850
:10808000B57F000809810008B57F0008B57F0008AA
:108090001D8100083D810008B57F0008B57F0008FC
:1080A0001D810008B57F0008B57F0008B57F000876
:1080B000B57F0008B57F0008B57F0008B57F0008D0
:1080C000B57F0008B57F0008B57F0008098100086A
:1080D0006381000809810008B57F0008B57F0008AA
:1080E000B57F0008B57F0008B57F0008B57F0008A0
:1080F000B57F0008B57F0008B57F0008B57F000890
:10810000B57F000825810008022D7FF453AF039B43
:108110003B6050E7002D3FF44DAF8DE7012D7FF41C
:1081200049AF48E73846202300F8013B0DF109012B
:108130001E2203F0EFF90023FB773CE7072D7FF4C5
:1081400039AF059BFB60039B03F16402049B7A61DA
:10815000013B3B61069BBB60079B7B60089B3B60D0
:1081600029E7042D7FF426AF039B3B70049B7B70B3
:10817000059BBB701FE700BF70B53E4B1A6882427B
:1081800088B0064673D002A81E60F8F763FB04A807
:10819000F8F7A6FE01200146F8F70AFD0120014686
:1081A000F8F706FD4FF400300121F8F70FFD00202D
:1081B000C4F2020002210722F8F762FB0020072226
:1081C000C4F202000321F8F75BFB022300208DF8C4
:1081D0000C30032304460125C4F2020002A98DF8E5
:1081E0000D30042302938DF80E408DF80F50F8F7F0
:1081F000D5FA20460823C4F2020002A90293F8F738
:10820000CDFA4FF48840C4F200002946F8F782FE08
:108210004FF488400C23C4F2000004A9ADF81A30D2
:108220000496ADF81440ADF81640ADF81840ADF81E
:108230001C40F8F7E9FD4FF48840C4F200002946DD
:10824000F8F75AFE4FF48840C4F2000040F225517E
:108250002A46F8F775FE262301A88DF804308DF81C
:1082600005408DF806408DF80750F7F7F1FF08B08C
:1082700070BD00BFEC0E002030B40F4A13687F2B96
:10828000FCD80E490E4D0B685C1C7F2C45F8230072
:1082900098BF0C6001D900230B6072B613680133DC
:1082A000136062B64FF48840C4F2000040F22771B8
:1082B000012230BCF8F744BEE80E0020E40E002096
:1082C000DC0C002010B50446007828B1FFF7D4FF7D
:1082D00014F8010F0028F9D110BD00BF30B40D4BC8
:1082E0001A6882B10C490D4D0A68541C802C55F84F
:1082F000225018BF0C6009D072B61A68013A1A6091
:1083000062B601220560104630BC704700220A6048
:10831000F2E700BFD80C0020D40C0020F00E0020A3
:10832000024A1368002BFCD1704700BFE80E002002
:108330004FF4884038B5C4F2000040F22551F8F7F8
:108340001BFE00282BD14FF48840C4F2000040F2FD
:108350002771F8F711FE00B938BD4FF48840C4F218
:10836000000040F22771F8F72DFE234B1A68002A0F
:1083700038D0224A224C1168481C802808BF0020AF
:1083800054F8211010601A684FF48840013AC4F282
:10839000000089B21A60BDE83840F8F7C9BD4FF453
:1083A0008840C4F2000040F22551F8F70BFE4FF46C
:1083B0008840C4F20000F8F7BFFD124B1A687F2A0C
:1083C000C1D81149114D0A68541CC0B27F2C45F820
:1083D000220098BF0C6001D900220A601A6801329D
:1083E0001A60B0E74FF48840C4F2000040F22771F1
:1083F000BDE83840F8F7A4BDE80E0020DC0E0020F0
:10840000DC0C0020D80C0020E00E0020F00E002034
:1084100010B541F2F004C2F2000402460B462046B9
:108420004FF4807103F0CEFC2046BDE81040FFF70A
:1084300049BF00BF0FB400B583B004AB53F8040BC1
:1084400019460193FFF7E4FF03B05DF804EB04B0B5
:10845000704700BFFFF790BE10B584B001A8F8F7D1
:108460002BFC01200146F8F7B1FB0023ADF80C30DE
:10847000ADF80630072301A902934FF0804003F5C1
:108480002D73ADF80430F8F7CBFB01210A464FF00D
:108490008040F8F7A1FC01240F2368461C228DF8C8
:1084A00000208DF803408DF801308DF80230F7F789
:1084B000CFFE4FF080402146F8F716FC04B010BD07
:1084C00038B54FF080400121F8F790FC6A4B1C68EA
:1084D000002C34D0694B1A6843F6982101328A4245
:1084E0001A6000D038BD664C6649674A012020609A
:1084F0000C6824180C6011680918116014680021B8
:108500003C2C1960EED1614B11601A6812181A6088
:108510005F4A10601A683C2AE4D15E4A1960136809
:108520001B1813601368182BDCD15B4B11601A68A1
:1085300012181A601A68072AD4D1196038BDFFF7DB
:10854000D9F950490B68012B07D9544B1A6840F6EA
:10855000A660013282421A6043D0514B1A68013240
:10856000EA2A1A6054D04F4B1A680132962A1A60D0
:1085700048D04D4B1A680132962A1A603CD04B4BBA
:108580001A6801320F2A1A6030D03C4B1A6843F641
:108590009820013282421A60A4D1394C3A4A012013
:1085A00020600C6824180C601168091811601168AB
:1085B00000242D291C6031D01268334B3C2A38D05E
:1085C0001B681E2B53D03A4B1A68002A8AD01A68AF
:1085D000013A1A601B68002B84D1364B01221A60C5
:1085E00080E71C60344B01221A60B6E7334A012051
:1085F000106000221A60C8E7314A01201060002292
:108600001A60BCE72F4A0120106000221A60B0E710
:108610002D4A0120106000221A60A4E72B4B1B4951
:108620001C680D68AC421FBF09681960284B1860B0
:10863000C2E7164A00211960136801331360144B16
:108640000120186013683C2BBDD1124B11601A68D1
:1086500012181A601A68182AB5D10F4A19601368DF
:108660001B1813601368072B08BF1160ABE7194B89
:1086700001221A60A7E700BF3C1200200012002070
:10868000FC11002044120020381200204C1200205F
:1086900010120020301200200412002020120020AE
:1086A000F011002014120020501200200C120020A3
:1086B000C4010020F4110020341200207C3E002070
:1086C000803E00202C12002048120020C80100200B
:1086D0001C120020181200204DF27870C0F6000025
:1086E000704700BF40F2D013C2F200031868704711
:1086F00041F2302141F24C2241F23823C2F2000112
:10870000C2F20002C2F2000343F68460C2F200002B
:10871000096812681B68816042600360704700BF8F
:108720002DE9F04F9DB001F04FFF01F0F5FF4FF440
:10873000E130FFF78FFEFFF75FF801F00DFB01F06E
:1087400037FBFFF789FE0120F9F79CF8F8F73CFDAD
:10875000F8F75AFD01F0EAFCFBF784FEF8F76EFD2E
:10876000002841F0D280C048FFF7ACFDBF48FFF7BA
:10877000A9FDBF48FFF7A6FDBC48FFF7A3FDBD4814
:10878000FFF7A0FDBC48FFF79DFDB848FFF79AFD35
:1087900041F2D820C2F200000368002B01F05C8097
:1087A000B648FFF78FFDB148FFF78CFDB44DFBF7DE
:1087B00071FD2B68002B01F04680B248FFF782FD67
:1087C000AA48FFF77FFD2B68002B41F07B80AE4C61
:1087D000AE482168FFF72EFE226822F47F0323F4BF
:1087E0007F43EBB940F2FF43C0F201039A4201F22A
:1087F000AA8040F2FF632268C0F201039A4201F2AC
:108800009880A348FFF75EFD9848FFF75BFD20685E
:1088100001F0E2FF206801F0E9FD2068FFF736FB78
:10882000FFF7BAFBF8F74CFD01F07CF941F23C216F
:10883000C2F2000101230B6002F018F841F23C2261
:10884000C2F2000200261660FAF7DEFCFAF71EFEFE
:1088500041F20823C2F2000341F2282A1860FAF715
:1088600067FEC2F2000ACAF80000FAF799FE41F268
:10887000242EC2F2000ECEF80000FAF73DFE41F2BF
:108880004021C2F200012B68086083B34FF4807569
:1088900023687D4FC0F20205AB4228D07D482946AF
:1088A000FFF7C8FD764B3D601B68002B41F07E80D2
:1088B0007948FFF707FD6D48FFF704FD01F0EEFB77
:1088C000002801F06B80FBF7B5FB002801F05E800B
:1088D00002F002F8002801F0518001F0BBF80028F6
:1088E00001F01F804FF48073C0F20203236041F255
:1088F0001C22C2F2000241F244230120C2F2000312
:1089000010601C68014602460334FAF77BFC41F212
:108910004425C2F2000509A82B689C421ED9FEF727
:1089200089FF0028F3D000210A460120FAF76AFCEB
:108930000120F8F791FF09A8FEF77CFF002001460F
:108940000246FAF75FFC5548FFF7BCFC4748FFF7C3
:10895000B9FC01F0A9FA08B101F0A0FB0020014622
:1089600002468046FAF74EFCFCF7D0F9FCF708F90E
:108970004FF0010ACDF814A0DFF82891484FCDF848
:10898000188000F13C0A834604254446CDF81CA01B
:10899000CDF8108013A8FFF701FB8246002840F0B5
:1089A000E381D9F800303BB141F24022C2F200022B
:1089B0001368002B40F00381B8F1000F40F02381D1
:1089C000DBF80030002B40F009863548F8F744FC0E
:1089D000002840F0478141F21C20C2F200000368E9
:1089E00073B141F2D821C2F200010B68002B40F0B4
:1089F000FF8541F21C2EC2F2000E0023CEF800309B
:108A0000D9F800306BB141F24020C2F20000036897
:108A10003BB141F23421C2F200010B68002B40F05F
:108A2000AB8641F2F412C2F20002136893B1DBF894
:108A30000430002B40F0228641F2F416C2F2000608
:108A400040F2C41A0023C2F2000A336040F6D86331
:108A5000CAF8003041F2102EC2F2000EDEF80030EB
:108A6000002B40F052851FE080D7000868C900083D
:108A7000A0D70008C0D7000878D70008CCD70008D6
:108A800060040020ECD70008D001002000D80008C6
:108A9000B8D80008F4D8000818D90008D8D90008B8
:108AA000843E0020083E002041F21821C2F200015D
:108AB0000B68002B00F0368340F2BC3AC2F2000A89
:108AC0008E4ADAF8003000211160002B00F02A8372
:108AD00041F24C2EC2F2000EDEF80020B2FBF3F1A0
:108AE00003FB1123002B40F01D8340F24C40C2F2E7
:108AF00000000368002B40F0548541F2D82EC2F2EA
:108B0000000EDEF80030002B00F0438501F0B8FCC9
:108B10007B4B7C4A064616F0010F7B484FEA560114
:108B200018BF1A46FFF786FCFF2E09D03046FBF728
:108B3000A9F841F24420C2F200000368063306930C
:108B4000002D40F0038341F24820C2F20000036888
:108B5000002B40F0188341F2FC12C2F200021368AD
:108B6000002B40F0228341F22C25C2F200052B6835
:108B7000002B40F02C8301F055F9FF28054600F04A
:108B80003183002101200A46FAF73CFB132D00F245
:108B90006B86DFE815F0C901BC01AA0145021A0283
:108BA0000802E30194025802AE025C0190018301C5
:108BB000760169019D01470132016906C90008A8D3
:108BC000FFF746F900283FF4F7AE40F2CC13C2F2AB
:108BD0000003089A1968531C8B4203D34B1C9A421A
:108BE0007FF6EAAE4948FFF725FC40F2CC15089B1A
:108BF000C2F2000518462B60FAF78EFF0225B8F185
:108C0000000F3FF4DDAE41F2F816C2F200064FF05D
:108C100001083368002B7FF4D8AEDBF804304FF046
:108C20000108002B3FF4D1AE394B3A48C3F800801D
:108C3000FFF748FB3848FFF745FB41F2F41A374984
:108C4000079A0BA802F002FCC2F2000A0BA8FAF77E
:108C5000C5FF3348CAF800800425F8F7FDFA00285C
:108C60003FF4B9AE012001460022FAF7CBFA41F2F7
:108C7000D82EC2F2000EDEF80030002B40F019852D
:108C800041F23020C2F20000BC680368244A9C42D2
:108C900000F06685D2F804E0042540F21002B969BC
:108CA0003E69D7F800C0F868C2F2000241F2042A17
:108CB00052F821307A69CDF80CC0C2F2000A8DE872
:108CC0001140CAF80010194641F24C2A731C41F2B7
:108CD0003026C2F20006C2F2000A3460CAF800E090
:108CE00041F2382EC2F2000E0E48CEF800C002F259
:108CF0006C72FFF79FFB32246DE600BF1812002054
:108D000060D10008F0C8000838DE000840DD000827
:108D1000F81100207CDD000868C9000890DD00081B
:108D2000843E002098DD0008AC48FFF7CBFAAC4841
:108D3000FFF7C8FA0126322404960025059E18EA9A
:108D4000060F52D1002C3FF425AE013C7FF422AE39
:108D5000204621462246FAF755FA13A8FFF71EF9D6
:108D6000824600283FF41DAE002101200A46AAF1E8
:108D7000410AFAF747FABAF1330F00F24182DFE80D
:108D80001AF0A40391038C0376033F026103560398
:108D90003F0234023F023F0235033F02CA023F0254
:108DA000B2023F023F02A7024B023F023F022A03E8
:108DB0001F033F023F023F023F023F023F023F02CA
:108DC0003F023F02140305039C023F023F023F02A1
:108DD0003F023F023F023F023F023F023F023F028B
:108DE00091023F023F023F024202F8F727FA0028B1
:108DF00040F09C8401260596A4E77A48FFF762FAC2
:108E00007748FFF75FFA41F24026C2F20006336866
:108E1000002B40F0DF840025FAF794FE32240495FD
:108E200002258BE77048FFF74DFA6D48FFF74AFAC5
:108E300041F24026C2F200063368002B40F0BB84AA
:108E40000025FAF775FE32240495022576E7674877
:108E5000FFF738FA6248FFF735FA0025FAF7BEFD4A
:108E600032240495022569E76148FFF72BFA5C4834
:108E7000FFF728FA0025FAF7F1FD322404950225C0
:108E80005CE75C48FFF71EFA5548FFF71BFA00261F
:108E9000FAF7B4FD3224049602254FE75648FFF74F
:108EA00011FA4F48FFF70EFA0025FAF7B7FD322402
:108EB0000495022542E75148FFF704FA4848FFF7B6
:108EC00001FA0026FAF77AFD32240496022535E7E6
:108ED0004B48FFF7F7F94248FFF7F4F90026FAF795
:108EE000ADFD32240496022528E74648FFF7EAF94B
:108EF0003B48FFF7E7F9FAF7EFFA41F20825C2F22B
:108F000000050026286032240496042516E73E4812
:108F1000FFF7D8F93248FFF7D5F900240494FBF79E
:108F200089F83224049D09E73848FFF7CBF92C482B
:108F3000FFF7C8F940F2701EC2F2000EDEF80050D2
:108F4000D5F1010538BF00250026CEF800503224A7
:108F50000496B5420CBF14250C25EFE62C48FFF70C
:108F6000B1F91F48FFF7AEF941F23026C2F2000610
:108F7000284B3268002A00F006841A68013A1A6009
:108F800041F2382AC2F2000A0023CAF8003041F246
:108F9000D82AC2F2000ADAF80060002E73D1322417
:108FA00004960425CAE61C48FFF78CF90C48FFF725
:108FB00089F9FAF7CBFA41F22826C2F20006002519
:108FC0000495322430600425B8E61448FFF77AF996
:108FD0000348FFF777F9FAF7C5FAECE788E00008ED
:108FE00068C900086CE0000850E0000888DF00084D
:108FF00010E00008ECDF0008C8DF0008A8DF000868
:1090000030E00008A8DE000898DE000888DE0008CE
:1090100028DF00083012002008DF0008E8DE000822
:10902000C448FFF74FF9C448FFF74CF9FAF742FA82
:1090300041F2082AC2F2000A002504953224CAF837
:10904000000004257AE6BD48FFF73CF9BA48FFF76F
:1090500039F941F24C21C2F20001B94B0A68002AE9
:1090600000F095831A68013A1A6041F2D82AC2F2D8
:10907000000A41F23822C2F20002DAF8006000234E
:109080001360002E8BD041F2302A41F24C2E41F277
:109090003820C2F2000EC2F20000C2F2000A00251F
:1090A000DAF80010DEF800200368A648B9607A609C
:1090B0003B60322401F096F8049504253EE6A24870
:1090C000FFF700F99C48FFF7FDF841F2302EC2F29D
:1090D000000E9E4BDEF80020162A00F25E831A680E
:1090E00001321A6041F23820C2F20000002303600E
:1090F0004DE79748FFF7E6F88F48FFF7E3F841F2AE
:109100004C23C2F200031A688D4B3A2A00F24283C4
:109110001A6801321A6041F23824C2F200040023B6
:10912000236034E7049E002E7FF4DFAC069E002E01
:109130003FF406AD41F2442AC2F2000ADAF80030E8
:10914000B342FFF4FDAC049E042506968148FFF768
:10915000B9F87948FFF7B6F841F2302A41F24C2EBF
:10916000C2F2000EC2F2000A2A46DAF80000DEF867
:109170000010FAF75BF841F24820C2F200000368E1
:10918000002B3FF4E8AC40F27011C2F20001724BC8
:10919000086800221A60FAF7D9FA41F2FC12C2F20A
:1091A00000021368002B3FF4DEAC6C4B00221A6007
:1091B00041F23823C2F2000341F22C25C2F200052D
:1091C0001868FAF705FA2B68002B3FF4D4AC644B0F
:1091D00000221A60F8F7AEF800F024FEFF280546DA
:1091E0007FF4CFAC00250495A8E55E48FFF76AF848
:1091F0005148FFF767F800F057FE002840F08081E3
:109200003224FFF7CEBB139B40F2C414C3F56E6348
:10921000C2F200040233236041F2D826C2F20006F3
:109220003368002B40F0E58241F2302AC2F2000A96
:10923000159CDAF800309C4200F0DF82DDF850E047
:10924000042540F21000199B169ADDF84CC0C2F2BA
:10925000000041F2302650F82310009241F24C2ACF
:1092600041F20422C2F20002C2F20006C2F2000A77
:109270000194CDF808E0CDF80CC013603460CAF852
:1092800000E041F2382E189A179B3748C2F2000EC0
:1092900002F26C720133CEF800C03224FFF7CAF834
:1092A000FFF77FBB13A8FAF799FC304813A9FFF723
:1092B000C1F804253224FFF774BB1398FAF7B6F807
:1092C00001462B48FFF7B6F804253224FFF769BBA7
:1092D000FAF7B0FE2748FEF7F5FF1748FEF7F2FF52
:1092E0003224FFF75EBB40F27010C2F20000139B05
:1092F0000268934284D0204A20491360002B204BFF
:10930000204808BF194614BF0C2514253224FFF746
:1093100091F8FFF746BB41F2F411C2F200010123BC
:1093200019480B60FEF7CEFF0348FEF7CBFF32244F
:10933000FFF737BBC8DE000868C9000858DF00081F
:109340004C120020843E002040DF00083012002034
:1093500070DF000878DE000848120020FC110020B1
:109360002C120020ECDC000894DC000824DD00084E
:10937000DCDA000804DD000870010020C4E0000809
:10938000D8E00008A0DA0008CCDC000813A8FAF73F
:10939000A5FBCA489DF84C109DF84D209DF84E3015
:1093A000FFF748F83224FFF7FCBA1398FAF7DCFB12
:1093B000C3481399FFF73EF802253224FFF7F1BAAC
:1093C000C048FEF77FFFC048FEF77CFF3224FAF763
:1093D000D7FBFFF7E6BABD48FEF774FF0124BA4891
:1093E000FEF770FF04943224FFF7DBBA139B002BC7
:1093F00000F00F8241F2402AC2F2000AB448012371
:10940000CAF80030FEF75EFFAF48FEF75BFF41F29F
:109410004021C2F2000140F2CC12C2F20002FF234E
:10942000086813603224FAF76DF8FFF7BABA139898
:10943000F9F7D8FFA7481399FEF7FCFF042532245B
:10944000FFF7AFBA41F22426C2F200061398336840
:1094500098423FF4D5AEFAF7A9F89F4A0346014671
:109460009E4813603224FEF7E5FFFFF79ABA41F2F7
:109470000821C2F2000113980B6898423FF4C0AE75
:10948000FAF70AF8964A03460146964813600425FF
:10949000FEF7D0FF3224FFF784BA13A8FAF7FAFADE
:1094A000914877E741F24025C2F200052B68002B76
:1094B00040F0BC811398FAF72FFB8C481399FEF704
:1094C000B9FF02253224FFF76CBA41F22822C2F21A
:1094D00000021398136898423FF492AEFAF72EF800
:1094E00041F24824824B0146C2F2000419608148CF
:1094F000002323600425FEF79DFF3224FFF751BAB5
:1095000000F0CCFD3224FFF74CBA7B4B00221A60EE
:1095100041F2042041F23022C2F20000C2F2000205
:1095200041F24C25C2F20005016813682A68734DA8
:1095300040F27016C2F20006C3EB0313306802EB70
:10954000830200F0B3FA002800F0A28041F2302A32
:1095500041F24C2E2968DFF8D0C16948C2F2000AF6
:10956000C2F2000EDAF80020DEF80030D1F1010E70
:1095700038BF4FF0000E6349C5F800E0BEF1000FA0
:1095800008BF61460CBF14250C25FEF753FFFFF7FB
:109590008BBA5D48FEF796FE4B48FEF793FEFFF749
:1095A000CFBA41F23C21C2F2000101230B6001F06D
:1095B000FDF841F23C2A0646544B554A554816F0F0
:1095C000010FC2F2000A18BF1A464FEA56010023E3
:1095D000CAF80030FEF72EFFFFF7A6BA4E48FEF796
:1095E00071FE3948FEF76EFE4FF00108FFF7EDB946
:1095F000DFF830A1504600F081FE00283FF4F9A9C1
:1096000041F23022C2F20002DAF808E013689E4507
:1096100000F0C680DAF804C0042540F2100AB969E7
:10962000F8687E69C2F2000A41F204225AF8213039
:10963000CDF808C08DE80140C2F20002386841F25E
:109640004C2A0390116006F26C7241F23026C2F28D
:109650000006C2F2000AC6F800E0CAF800C041F2F3
:10966000382A19463E683B692C48C2F2000A013389
:10967000CAF80060FEF7DEFEFFF7BBB90020014626
:109680000122F9F7BFFD322401F088F9FFF7D4B9C0
:10969000234B4CF6CD451B68CCF6CC45A5FB03050A
:1096A000AD0805EB8505AB420CBF04250125FFF78E
:1096B000FBB91C4800F096FDFFF7E2BA74DA000827
:1096C000C4DB000878DC000868C9000850DB00082B
:1096D000F0DB000850DC00082412002024DB000826
:1096E00008120020B8DA000848DA00086CDB00082D
:1096F0002812002000DB000810120020700100205A
:10970000F0DD0008C4E000085CDE000860D100085D
:10971000F0C8000810DE00086CDD0008C4DD000899
:109720004C120020843E0020D8E00008A448FEF738
:10973000C9FDA448FEF7C6FD41F2F81E4FF0000A2D
:10974000C2F2000ECBF804A08BF83CA09E499F48C3
:10975000CEF800A0CDF814A0FBF754FAFFF7F2BA48
:1097600041F24C21C2F20001D2F804E00B689E45A0
:109770007FF492AAFFF791BAFEF768FB944B0022A0
:109780001A60FFF74EB917221A60FFF7F9BB3B22A8
:109790001A606AE400221A60BDE400221A60A1E4A3
:1097A00041F24C26C2F20006DAF804C033689C4548
:1097B0007FF432AF31E7874A40F2CC1A0023C2F27D
:1097C000000A18461360FF23CAF80030F9F79AFE22
:1097D000FFF736BB7F4A40F2CC1A0023C2F2000AE0
:1097E00018461360FF23CAF80030F9F78BFEFFF725
:1097F00012BB13A800F0F6FC16E541F24C2EC2F2A3
:10980000000EDEF80030DDF850E09E457FF418AD24
:1098100017E541F2402EC2F2000E6F48CEF800303C
:10982000FEF750FD6748FEF74DFDF0E5694A40F24E
:10983000CC160023C2F2000618461360FF233360E3
:10984000F9F760FE36E66548654CFEF73BFD5D487E
:10985000FEF738FDFEF7E4BF6248FEF733FD5948D6
:10986000FEF730FDFEF7A2BF132D54D80FF2040A05
:109870005AF825F0358F00081B8F0008F78E000876
:109880002D900008D78F0008B38F0008698F00085B
:10989000CB90000853900008FF9000085B8E0008F2
:1098A000C38E0008A98E00088F8E0008758E0008F0
:1098B000DD8E0008318E0008078E0008D39800085E
:1098C000358D0008002046490422FAF7F3FDFEF723
:1098D0007EBF41F2402AC2F2000A40F2CC1EDAF802
:1098E0000030D3F1010338BF0023C2F2000E184646
:1098F000CAF800300025FF23CEF800303224F9F7F3
:1099000001FE04950225FFF719BAF7F74DFCFBF7A6
:10991000ABF9FEF728BF0026049632243546FFF740
:109920000DBA3148FEF7CEFC2648FEF7CBFCFEF719
:10993000D9BF2E48FEF7C6FC2248FEF7C3FC00F054
:1099400063F8FEF75EBF2A48FEF7BCFC1D48FEF731
:10995000B9FC00F079FB2748FEF7B4FC1948FEF784
:10996000B1FC2068FAF7CEF92348FEF7ABFC1548A6
:10997000FEF7A8FC00F07EFFFEF73BBF1F48FEF796
:10998000A1FC1048FEF79EFCFEF7A7BF1C48FEF79F
:1099900099FC0C48FEF796FCFEF79ABF1948FEF7B3
:1099A00091FC0848FEF78EFCFEF78DBF3046394625
:1099B0000422FAF799FD00287EF480AFFEF778BF05
:1099C000F4D9000868C900083CDA000830DA000859
:1099D000341200204012002020DC0008E0D80008EB
:1099E000D0010020DCD70008ACD9000894D80008CA
:1099F00024D8000844D8000870D8000880D900088E
:109A000060D900083CD9000830B5104B1B6887B0FE
:109A100013B9002007B030BDBF2069461822FAF7FD
:109A200049FD0028F5D00A486A4600231478517889
:109A300095781C50C1EB01111C18083305EB81010E
:109A40000332402B6160F1D10120E3E76004002084
:109A5000A83E002070B548F6890686B0114C6A46CB
:109A60000023C8F688061819195940681170A6FB1A
:109A700000514909C1EB0115A0EB85000833517075
:109A800090700332402BEED1074B186838B1BF20DD
:109A900018226946FAF728FD003018BF012006B0E9
:109AA00070BD00BFA83E002060040020F0B4002379
:109AB0001B4D02E00833402B22D05C5914F0800F7C
:109AC00003EB0506F6D076689642F3D1C4F3C206DE
:109AD00004F0070704F0400418B1D4F1010438BFC2
:109AE0000024002CE6D0BE420DD8B14234BF00267F
:109AF0000126B94288BF0026002EDBD0012000E0FD
:109B00000020F0BC7047B9428CBF00270127B1424A
:109B100034BF3E4647F00106002ECBD0EEE700BF33
:109B2000A83E0020704700BF70B54FF44064C4F2F7
:109B3000020404266420F7F76DFE66834FF40C7070
:109B4000F7F768FE284D26831420F7F763FE0026FA
:109B50004FF496732B60344603E004B92C682B68ED
:109B6000ABB14FF440600421C4F20200F6F77CFE72
:109B7000D6F1010338BF0023002C08BF00230028C2
:109B8000EBD0002BEBD02E682B68002BE9D13220D4
:109B9000002E18BF002C0CBF0025012515D0F7F7AB
:109BA00039FE4FF440600421C4F20200F6F75CFE77
:109BB00005467820F7F72EFE6B1E5842C6EB0404CC
:109BC00058411E2C98BF002070BDF7F723FE4FF4BC
:109BD00040600421C4F20200F6F746FE7820F7F751
:109BE00019FE284670BD00BF043E002038B54FF472
:109BF0004064C4F20204042505206583F7F70AFED9
:109C000025830A20F7F706FE29462046F6F72CFEA4
:109C100004463220F7F7FEFD621E5042504138BD27
:109C200070B5082401250026FFF7E0FF6B0000B1A6
:109C30002E43013CDDB2F7D1304670BD38B54D1E24
:109C40000446EDB239B101354519FFF7E9FF04F8D3
:109C5000010BAC42F9D138BD2DE9F0414FF440661B
:109C6000804608250124C4F2020604270AE00520E4
:109C7000F7F7D0FD502037836400F7F7CBFD013DA7
:109C8000E4B20ED0502014EA080F7783EFD1F7F733
:109C9000C1FD052037836400F7F7BCFD013DE4B248
:109CA000F0D1BDE8F08100BF38B54D1E0446EDB2DD
:109CB00039B10135451914F8010BFFF7CDFFAC425E
:109CC000F9D138BD10B50446FFF72EFF024680B922
:109CD000234603F8012B0133627003F8012B03F8CC
:109CE000012B03F8012B03F8012B03F8012B1A7049
:109CF00010BD3320FFF7B0FF20460821FFF79EFF7D
:109D0000FFF712FF012010BD70B5124B1A6882B028
:109D10000AB102B070BD012468464FF440651C6072
:109D2000C4F20205F6F796FD08202146F6F740FF3B
:109D3000042602232846694600968DF804408DF8D3
:109D400006408DF807408DF80530F6F727FD2E8385
:109D5000DFE700BF5412002000B583B06846F6F775
:109D600079FD04200121F6F723FF4FF480724FF4B0
:109D70000060002369460092C4F2020001228DF8BF
:109D800005308DF804208DF806308DF80730F6F791
:109D900005FD4EF2A000C0F60000FEF793FA4CF667
:109DA0006810C0F60000FEF78DFA03B000BD00BFDA
:109DB00010B50B4C2368012B10D04FF400604FF40A
:109DC00080710122C4F20200F6F754FD0548FEF747
:109DD00079FA0548FEF776FA0123236010BD00BF2B
:109DE000D4010020B4E0000868C9000810B50A4C8E
:109DF000236883B14FF400604FF480710022C4F2F5
:109E00000200F6F737FD0548FEF75CFA0448FEF756
:109E100059FA0023236010BDD4010020C8E00008D7
:109E200068C90008F0B583B06846FDF703FD60B36C
:109E30001A4A1B4B10681968013010609DF8052004
:109E400031B302F001021749BDF80170BDF803C03B
:109E50001A6000239DF8004018460E4602E00130CB
:109E6000782B12D0CA5C0633A242F8D100EB400234
:109E700006EB4202B2F80150BD42F0D1B2F8032025
:109E8000624503D00130782BECD1FF2003B0F0BD48
:109E900012F00102D7D001221A60F6E75C1200200E
:109EA00058120020601200202DE9F04FDFF8948155
:109EB0004E4D002783B001263C46C2462846F9F79E
:109EC0008DFE2846FEF7FEF94948FEF7FBF9684685
:109ED000FDF7B0FC04EB440908EB49090AEB070560
:109EE0004846FDF7A7FC0028FAD06A7912F0010273
:109EF000F6D1D4B399F80010134602E00133A3421F
:109F000031D018F80200884202F10602F6D103EBC4
:109F1000430C0AEB4C0CB9F80100BCF801E0864593
:109F2000ECD1B9F803E0BCF803C0F445E6D1FF2B4F
:109F300019D00022134602E00133A342D0D018F812
:109F400002C08C4502F10602F6D103EB430C0AEB8A
:109F50004C0CBCF801B08345EED1BCF803C0F4450D
:109F6000EAD1002BBCD1142E37D0731E122B3BD854
:109F7000DFE803F02F2D2B29272523211F1D1B1977
:109F8000171513110F0A31001A4D01340136063727
:109F900094E7194DF9E7194DF7E7194DF5E7194D14
:109FA000F3E7194DF1E7194DEFE7194DEDE7194DBD
:109FB000EBE7194DE9E7194DE7E7194DE5E7194DCD
:109FC000E3E7194DE1E7194DDFE7194DDDE7194DDD
:109FD000DBE7194DD9E7194DD7E71948F9F7FEFD29
:109FE000012003B0BDE8F08F004DCEE7F0E000089F
:109FF00068C90008B8E2000898E2000878E20008A2
:10A000005CE2000840E2000820E2000800E20008EC
:10A01000E4E10008C8E10008B4E10008A0E100089C
:10A020008CE1000878E100085CE1000840E10008EC
:10A0300024E1000808E1000800E10008DCE0000875
:10A04000D4E2000860120020F0B5124B186883B00B
:10A05000E8B10025104F04262C46052230466946FB
:10A06000FAF728FA9DF800C0BDF80110BDF80320EA
:10A0700007F805C004EB440307EB4303013405363E
:10A080000635142CA3F80110A3F80320E5D103B082
:10A09000F0BD00BF6004002060120020F0B5114B3D
:10A0A000186883B0E0B100250F4F04262C4604EB5E
:10A0B000440307EB43037A5DB3F801E0B3F80330E0
:10A0C0008DF800203046052269460134ADF801E0E4
:10A0D000ADF80330B6180635FAF706FA142CE6D1B7
:10A0E00003B0F0BD600400206012002010B582B003
:10A0F00004460B460092D02000222146FDF740FA8C
:10A10000D0F1010038BF002002B010BD10B582B000
:10A1100004460B460092D02000222146FDF7AEFAFD
:10A12000D0F1010038BF002002B010BD30B583B0BF
:10A13000FDF7D2F93F200DF107010122FFF7D6FF0D
:10A14000054620B301240720244B0DEB00012246D5
:10A150001C60FFF7CBFF10B39DF80730002B29D10F
:10A1600000200DF107010122FFF7C0FF0446B0B146
:10A170009DF807301A0619D503F07F0300200DF172
:10A18000070101228DF80730FFF7C0FF0EE00E2017
:10A190000DF107010122FFF7A9FF044618B90024B9
:10A1A000204603B030BD9DF807306BB90C4B01223F
:10A1B0001A60F5E7072000230DEB000122468DF819
:10A1C0000730FFF7A3FFCBE70E200DF107010122B7
:10A1D0008DF80750FFF79AFFE8E700BFE012002074
:10A1E000D81200202DE9F04F434B1B6889B01BB9F2
:10A1F000184609B0BDE8F08F836802690193C3680F
:10A2000041690293466807688069013246F26763D4
:10A21000C6F2666303926439049183FB06B901991F
:10A22000DDF80CB0019A059083FB078A83FB0BBC19
:10A2300083FB0118DDF810B00299DDF80CE0D017AF
:10A24000FD1783FB0121029A009183FB0BB3DDF81C
:10A2500010B0C5EBAA05D1174FEAEE724FEAEB7EBC
:10A2600005EB850BC0EBA800F417DDF80080A7EB29
:10A270004B0B019FC4EBA90400EB8009C1EBA801C3
:10A28000A7EB4909029F01EB8108C2EBAC02A7EBE7
:10A290004808039F04EB840A02EB820CCEEBA30375
:10A2A000A6EB4A06A7EB4C0C049F06EB041603EB47
:10A2B000830E059C8DF81960A7EB4E0E09EB001973
:10A2C00008EB01180CEB021C0BEB051701340EEB2D
:10A2D000031E002006A907228DF818708DF81A9029
:10A2E0008DF81B408DF81C808DF81DC08DF81EE088
:10A2F000FFF70CFF7DE700BFD81200202DE9F04FDB
:10A30000394B1B688BB004461BB900200BB0BDE86D
:10A31000F08F002008A90722FFF7E8FE0028F4D0FC
:10A320009DF825A09DF820709DF826809DF823902B
:10A330009DF82430CDF818904FEA1A1B4FEA171CED
:10A340000BEB8B0B4FEA1819CDF81CB00CEB8C0CF7
:10A350009DF82220CDF800C009EB890908F00F080C
:10A36000DDF81CC005930AF00F0ACDF80890CDF86F
:10A3700004809DF82150DDF81490DDF80480CDF8BC
:10A380000CA011090AEB4C0ADDF808C002F00F021C
:10A3900001EB81012E091B0909F00F0B02EB4101B2
:10A3A00008EB4C09069ADDF80080049305F00F05D0
:10A3B00007F00F0706EB860603EB830305EB460663
:10A3C00002F1FF3C07EB48070BEB43030AF1FF35B3
:10A3D00009F1640227606660A160C4F818C0E360F8
:10A3E0002561626192E700BFD812002000B50E4BD4
:10A3F0001B6883B053B1FF23C0F20203984207D811
:10A4000000220120094B1A6003B000BD1846FBE78B
:10A410000122DF200DF10701FAF74CF89DF8072023
:10A420000A2A88BF0022EDE760040020DC12002029
:10A4300000B5094B094A1B68106883B08DF80730D6
:10A4400040B1DF2001220DF10701FAF74DF800308D
:10A4500018BF012003B000BDDC1200206004002002
:10A4600041F2DC23C2F200031868704710B541F2D4
:10A47000DC24C2F200042060FFF7DAFF206810BD80
:10A4800000B50D4B1B6883B0FF200BB903B000BDB6
:10A49000112001A90222FFF729FE0028F6D09DF81D
:10A4A0000500064B9DF804201B68C0F3400040EAFD
:10A4B0004200C01AEAE700BFD8120020DC120020D8
:10A4C0000649074A074B9A42BEBF51F8040B42F8AF
:10A4D000040BF8E70448804704480047B8E4000844
:10A4E00000000020B4020020C9A50008DD0100081A
:10A4F0003349344A002301E041F8043B9142FBD345
:10A50000FEF70EF9FEE7FEE7FEE7FEE7FEE7FEE7F1
:10A51000FEE7FEE7FEE7FEE7FEE7FEE7FEE7FEE713
:10A52000FEE7FEE7FEE7FEE7FEE7FEE7FEE7FEE703
:10A53000FEE7FEE7FEE7FEE7FEE7FEE7FEE7FEE7F3
:10A54000FEE7FEE7FEE7FEE7FEE7FEE7FEE7FEE7E3
:10A55000FEE7FEE7FEE7FEE7FEE7FEE7FEE7FEE7D3
:10A56000FEE7FEE7FEE7FEE7FEE7FEE7FEE7FEE7C3
:10A57000FEE7FEE7FEE7FEE7FEE7FEE7FEE7FEE7B3
:10A58000FEE7FEE7FEE7FEE7FEE7FEE7FEE7FEE7A3
:10A59000FEE7FEE7FEE7FEE7FEE7FEE7FEE7FEE793
:10A5A000FEE7FEE7FEE7FEE7FEE7FEE7FEE7FEE783
:10A5B000FEE7FEE7FEE7FEE7FEE7FEE7FEE7000058
:10A5C000B4020020EC3E00204FF46D42CEF20002B7
:10A5D0004FF46053D2F88810C4F2020341F47001C2
:10A5E000C2F888101968002241F0010119609A60D0
:10A5F000186843F2100120F08470C2F2004120F488
:10A60000803018605960196882B021F48021196087
:10A61000DA60009201921A6842F480321A6003E014
:10A62000009AB2F5C06F09D01A6802F400320192A4
:10A63000009A01320092019A002AF1D04FF460533F
:10A64000C4F202031B6813F4003308BF019301D066
:10A6500001230193019B012B00D0FEE74FF46053CF
:10A66000C4F202034FF4E042196CC4F2000241F05C
:10A6700080511964116841F4804111609A6822F098
:10A68000F0029A609A6822F460429A609A6842F4F2
:10A6900080529A601A6822F080721A6019684FF42A
:10A6A00060528801C4F20202F8D445F20843C0F2B5
:10A6B00041735360136843F08073136011684FF463
:10A6C00060538901C4F20203F8D54FF47052C4F20A
:10A6D0000202116841F4407141F0020111601268F8
:10A6E00002F00702022A00D0FEE79A6822F0030275
:10A6F0009A609A6842F002029A609A6802F00C022C
:10A70000082AFAD14FF46D43CEF200034FF00062F5
:10A710009A6002B0704700BF4FF46053C4F2020366
:10A720009A6802F00C02042A14D0082A1CBF4FF4C5
:10A730001052C0F2F40212D04FF46053C4F202037C
:10A7400018499B68C3F30313CB5C22FA03F2164B40
:10A750001A6070474FF49052C0F27A02ECE75868E2
:10A76000596810F4800F586815BF4FF490534FF498
:10A770001053C0F27A03C0F2F40301F03F01B3FBBF
:10A78000F1F24FF46053C4F20203C0F388105B6827
:10A79000C3F30143013302FB00F25B00B2FBF3F2AF
:10A7A000CAE700BFD8010020E801002000B585B04D
:10A7B00001A802A903AAF9F76FFD10B9FF2005B09F
:10A7C00000BD029B002BF9D1024B1868039B181A9D
:10A7D000F5E700BFE412002000B50E4B1B6883B004
:10A7E00053B1FF23C0F20203984207D80022012090
:10A7F000094B1A6003B000BD1846FBE70122DF20B9
:10A800000DF10701F9F756FE9DF807200A2A88BFC7
:10A810000022EDE760040020E412002000B5094B9F
:10A82000094A1B68106883B08DF8073040B1DF20FB
:10A8300001220DF10701F9F757FE003018BF012082
:10A8400003B000BDE41200206004002041F2E423C4
:10A85000C2F200031868704710B541F2E424C2F256
:10A8600000042060FFF7DAFF206810BD0920F9F727
:10A8700085BD00BF00B5144B1B6883B02BB1AA2067
:10A8800012491022F9F716FE50B910220F4810494C
:10A8900000F040FE0F4B01221A60002003B000BD03
:10A8A000BA2001A90222F9F705FE0028EDD09DF893
:10A8B00004109DF80520074B01202D291A60EDD1C9
:10A8C00052421A600120E9E760040020F0010020F4
:10A8D000E4E20008EC01002000B5134B1B68002BDC
:10A8E00083B01ADB2B228DF804208DF805300F4B36
:10A8F0001B6813B9002003B000BDAA200C49102228
:10A90000F9F7F2FD0028F5D0BA20022201A9F9F7E3
:10A91000EBFD003018BF0120EDE75B422D228DF8E2
:10A9200004208DF80530E2E7EC01002060040020EF
:10A93000F001002040F2EC13C2F2000318687047E7
:10A9400010B5014604460A48FDF774FD04F10C03F6
:10A95000182B0AD8074B1A68A24204D01C60FFF7D4
:10A96000BBFF012010BD012010BD002010BD00BFA5
:10A97000F4E20008EC01002040F2F010C2F2000006
:10A98000704700BF014608B540F2F010C2F2000067
:10A9900000F097FDBDE80840FFF79EBF40F2F010C1
:10A9A000C2F20000FAF746B970B5284A48F280139F
:10A9B000126882B0C7F65543CB1802AE4FF46161FE
:10A9C00001FB023346F8043D0546304600F036FAF6
:10A9D0000369DA1E052A04460CD9022B2BD0092B59
:10A9E00010D18369C268D21A182A03DD53B983686B
:10A9F000022B07DC019B304603F56163019300F0F5
:10AA00001DFA044663696B6123692B61E36804F1F5
:10AA10000C00EB6007C8013102F26C72F6F760FBC4
:10AA2000A861236A2B62A368AB6063686B602368CC
:10AA30002B6002B070BD8369C268D21A182AE1DDAA
:10AA4000002BD7D18368012BD4DCDBE7EC0100209D
:10AA500046F2700048F2200108B5C4F20200C2F2CA
:10AA60000001F5F753FE60B146F2700048F2200194
:10AA7000C4F20200C2F20001F5F774FE014B00229D
:10AA80001A6008BDE81200202DE9F047DFF834E134
:10AA90000646DEF80030002BFBD1002E00F08A8045
:10AAA000464D4748770007EB060CAC444FF0FF34A7
:10AAB00015F802AC631C00EB440104F10909802283
:10AAC00012EA0A0F0CBF4FF027084FF0430801337A
:10AAD00052084B4521F8028FF2D104F1080115F814
:10AAE00003AC00EB410104F11109802212EA0A0FC4
:10AAF0000CBF4FF027084FF04308013352084B4575
:10AB000021F8028FF2D104F1100115F801AC00EB2D
:10AB1000410104F11909802212EA0A0F0CBF4FF01B
:10AB200027084FF04308013352084B4521F8028FA4
:10AB3000F2D1033518346545BAD1002200EB430346
:10AB4000114699520232602AFBD14FF480600124F1
:10AB50000021C4F20000CEF80040F6F7C5F846F236
:10AB600070000021C4F20200F5F7A4FDBB19DB0060
:10AB7000303346F270004FF6F8711940C4F202000B
:10AB8000F5F7A2FD46F2700010212246C4F2020041
:10AB9000F5F79CFD46F270002146C4F20200F5F77D
:10ABA00089FD4FF48060C4F200002146BDE8F04703
:10ABB000F6F79AB8334602483746BEE7EF12002050
:10ABC00070150020E8120020D52810B409D80C78A0
:10ABD000054A00EB4000131814544A785A708A78DA
:10ABE0009A7010BC704700BFEC120020F0B469B13D
:10ABF0000A4D01EB410700230478EC54EC18467829
:10AC0000667086780333BB42A670F5D10AB9F0BCF2
:10AC100070470846F0BCFFF737BF00BFEC120020BA
:10AC20002DE9F041644D9AB0002401A84FF400666C
:10AC3000C4F202062C60F5F70DFE04200121F5F7A1
:10AC4000B7FF022703234FF04008304601A98DF8D3
:10AC500009308DF80870CDF804808DF80A408DF821
:10AC60000B40F5F79BFD3A4606213046A6F81A80C0
:10AC7000F5F706FE03A8F6F71FF806A8F6F78AF818
:10AC800038460121F5F7A2FF4FF400100121F5F736
:10AC90008FFF4FF480606A23C4F2000003A904937D
:10ACA000ADF80C40ADF81440ADF80E40F5F7B8FF24
:10ACB0004FF4806060230126C4F2000006A9ADF8BD
:10ACC0001830ADF81A600894ADF82440F6F71AF879
:10ACD0004FF48060C4F200000821F6F765F84FF4E5
:10ACE0008060C4F200003146F5F7F0FF4FF4806059
:10ACF000C4F200003146F6F75FF84FF480604FF47D
:10AD000000713246C4F20000F6F774F80F2268466C
:10AD10008DF800208DF801408DF802408DF8036019
:10AD2000F5F796FA0BA8F5F7B3FC46F2700021464A
:10AD3000C4F20200F5F7BEFC46F27000C4F2020055
:10AD4000F5F77EFB40F23443C4F200030C934FF45A
:10AD5000006312934FF4005313934FF4A2530F93D5
:10AD60004FF4806311934FF4403315934FF02063F9
:10AD70000B9346F27000114B1494C4F202000BA91D
:10AD80001094CDF838800D93169417961894199452
:10AD90002746F5F749FC8DF82C408DF82D408DF8AD
:10ADA0002E402B68002BFCD10BA8D6210122FFF7E7
:10ADB0001DFF1AB0BDE8F081E812002070150020D8
:10ADC00000210A2200F046BC08B5074B044613B127
:10ADD0000021AFF30080054B1868836A03B19847E0
:10ADE000204601F071F800BF000000000CE30008ED
:10ADF00070B50E4B0E4DED1AAD1000241E4603E04B
:10AE000056F8242090470134AC42F9D101F05EF8A5
:10AE1000084D094BED1AAD1000241E4603E056F80C
:10AE2000242090470134AC42F9D170BDAC0200201F
:10AE3000AC020020B0020020AC02002038B5074B65
:10AE40001C68E36B05461BB9242000F00DF8E06395
:10AE5000E16B2846BDE8384000F002B864020020EB
:10AE6000002200F0C3B80000024B0146186800F051
:10AE700047BA00BF6402002010B5002302E0CC5C9A
:10AE8000C45401339342FAD110BD8218034601E045
:10AE900003F8011B9342FBD1704700002DE9F74FE7
:10AEA000064600F09FFF40F2B1739E42024640F317
:10AEB00096806FF4F663F318A6F2B2719B1040F21D
:10AEC0006D1505FB0135A6F26D716FF0630391FB03
:10AED000F3F36FF4C861ED1871184FF4C87391FB68
:10AEE000F3F16D18642196FBF1FC01FB1C6C96FBE1
:10AEF000F3F103FB1161D1F10101466006F0030695
:10AF000038BF002101960346022407261F7A4A2FE4
:10AF100011D15F69019805EB070810B9BCF1000F6A
:10AF200000D121B13B2FD4BF0027012700E00F46FD
:10AF30004744013F3FE0442F02D15F69EF193AE0F7
:10AF4000019F37B9BCF1000F0CBF89464FF00109D2
:10AF500000E089462348D3F80CA04FF0300808FBE6
:10AF600009090127A84605E009EB870B01375BF8C3
:10AF700004BCD8445745F7DB08F1040797FBF6FB00
:10AF800006FB1B7B5F691869BAF1010FB8BF4FF070
:10AF9000010A0AF1FF3AB7EB0B0748BF073700F188
:10AFA000FF3B072000FB0B7759F82A9000E0073F92
:10AFB0004F45FCDA47449869DFF82C8008FB070707
:10AFC000186A013C074443F81C7F9FD1936BD169F9
:10AFD0009942ACBF002301231360012000E0002050
:10AFE000BDE8FE8F10E30008805101002DE9F84311
:10AFF00080460C46174600F0F5FED8F800109B4A34
:10B0000091FBF2F3064602FB131104E001F5A831AF
:10B0100001F5C071013B0029F8DB4FF4616091FB41
:10B02000F0F200FB12113C20A26091FBF0F200FB59
:10B030001211626021601A1D072192FBF1F001FBE1
:10B040001022002AB8BF0732002BA26140F2B2756D
:10B050004FF4C8704FF0640CDFF81C9217DBA9079F
:10B0600004D195FBFCF20CFB125242B995FBF0F1B6
:10B0700000FB1151D1F1010138BF002100E0012195
:10B0800059F82120934218DB01359B1AE7E7013D6F
:10B09000AA0704D195FBFCF20CFB125242B995FBB6
:10B0A000F0F100FB1151D1F1010138BF002100E0A6
:10B0B000012159F821209B18E9D4A5F26C72626134
:10B0C0006B4AE3614FF0300909FB0129002222613C
:10B0D00002E001319B1A2161216959F82120934234
:10B0E000F7DA0133E360002F40F0BA8000F0A6FCED
:10B0F000604B1B681BB373689D4205D13168D8F85B
:10B100000030F26931B90CE02846FFF7C7FE00288D
:10B11000F4D110E093420CDBB26B934209DA0123C5
:10B120000BE09342FBDAB26B9342ACBF00230123E6
:10B1300003E0002301E04FF0FF33236200E02762C9
:10B14000236A2568012B0CBFF36B336A4FF46160EF
:10B1500093FBF0F200FB12333C2093FBF0F100FB79
:10B1600011336068411AA0686160EB1A821A3B2BA8
:10B170002360A26003DD013161603C3B04E0002BF1
:10B1800003DA013961603C33236063683B2B03DDE4
:10B190000132A2603C3B04E0002B03DA013AA260DA
:10B1A0003C336360A368172B1FDDE2690132E26163
:10B1B000A2690132062AC8BF0022A261E268183BD8
:10B1C0000132A3602369E26059F823108A4244DD0A
:10B1D0000133521A0C2BE26023613ED162690023D5
:10B1E000013223616261E36137E0002B35DAE26905
:10B1F000013AE261A269013A48BF0622A261E2680F
:10B200001833013AE260A3603ABB2369013B01D4E1
:10B2100023611EE00B23236163695A1E12F0030FA2
:10B22000626103F26B7305D1642293FBF2F102FBBE
:10B23000113252B94FF4C87293FBF2F102FB113391
:10B24000D3F1010338BF002300E0012303F5B673F7
:10B25000E361236959F82330E36000F0F0FB01E07B
:10B26000002323622046BDE8F88300BF805101001F
:10B2700010E30008F83D002070E3000830B5002915
:10B280003BD051F8042C0B1F1C49002AB8BF9B1857
:10B290000A6812B95A600B6030BD93420CD219682B
:10B2A0005818904203D15A588918426819605A6058
:10B2B000124A136030BD0A46516809B19942FAD961
:10B2C000146815199D420AD11B68E318D0188842EA
:10B2D000136012D108681B1813604B680CE002D988
:10B2E0000C23036030BD18681C188C4203D10C6815
:10B2F0004968001918605960536030BDF43D002062
:10B30000F8B5CD1C25F0030508350C2D38BF0C25EC
:10B31000002D064645DB8D4200D242E0234B1B68E0
:10B320001C4612E02268521B0DD40B2A02D922605F
:10B33000A4181EE0A34203D163681C4A136021E0F5
:10B3400062685A601EE023466468002CEAD123E05C
:10B350003046214600F06AF838602946304600F051
:10B3600065F8431C01461CD0C41C24F0030484422D
:10B3700001D1256006E03046611A00F057F801302F
:10B38000F7D10EE004F10B00231D20F00700C31AD3
:10B390000AD05A42E250F8BD054F3B68002BDCD181
:10B3A000D6E70C2333600020F8BD00BFF43D002039
:10B3B000F03D00201A4B10B51C68A36BD3B91820C0
:10B3C000FFF752FD43F20E33A06303804AF6CD33FC
:10B3D000438041F2342383804EF26D63C3804DF687
:10B3E000EC630381052343810B2383810122002326
:10B3F000C0E90423A46B0B49206962690A4B4143ED
:10B4000003FB0212A0FB03015118012200231218B2
:10B4100043EB0103C4E9042323F0004010BD00BF47
:10B42000640200202DF451582D7F954C38B5064C00
:10B43000002305460846236000F02CFD431C02D182
:10B44000236803B12B6038BDE83E00200EB400B580
:10B450009CB04FF40271ADF814106FF000411DABB9
:10B46000049107914FF6FF71ADF81610084953F893
:10B47000042B029006900868019302A900F0E6F9F7
:10B48000029B00221A701CB05DF804EB03B07047F9
:10B4900064020020C9B2034610F8012B12B18A429F
:10B4A000F9D102E0002918BF00231846704710F8B0
:10B4B000012B11F8013B012A28BF9A42F7D0D01A7C
:10B4C0007047034611F8012B03F8012B002AF9D12C
:10B4D0007047034613F8012B002AFBD1181A0138D4
:10B4E000704770B5A2B108E0012A03D128781B7813
:10B4F000C01A70BD013A002CF8D00B460546002A50
:10B50000F4D010F8016B1C780131B442ECD0EDE7B7
:10B51000104670BD30B50139034609E011F8015FEE
:10B5200003F8015B013A1C4615B99B18002205E09F
:10B530001C46002AF2D1F8E704F8012B9C42FBD10B
:10B5400030BD00002DE9F74F01904148D0F8009040
:10B550000846044614F8015B09EB05062046777897
:10B5600007F00807FFB2002FF3D12D2D03D114F8F7
:10B57000015B012704E02B2D04BF244614F8015B76
:10B58000002B5ED0102B08D158E02078782801D00D
:10B5900058284ED1657810230234002F0CBF6FF06D
:10B5A00000404FF00040B0FBF3FA002603FB1A08FE
:10B5B000304609EB050C9CF801C00CF0040B5FFA57
:10B5C0008BFBBBF1000F01D0303D0BE01CF0030CF6
:10B5D0001BD0BCF1010F14BF4FF0570C4FF0370CCC
:10B5E000CCEB05059D4210DAB6F1FF3F0AD050457D
:10B5F00006D801D1454503DC03FB0050012601E0DC
:10B600004FF0FF3614F8015BD3E7731C0AD1002F0B
:10B6100001990CBF6FF000404FF0004022230B60F7
:10B6200022B912E007B140427AB106B1611E116041
:10B630000BE03025002BB0D10823AEE7302DACD184
:10B64000A3E7302DA1D00A23A7E7BDE8FE8F00BFF6
:10B650006802002030B51346044A05460C461068BF
:10B6600029462246BDE83040FFF76CBF6402002047
:10B670002DE9F74F01903D48D0F800900846044668
:10B6800014F8015B09EB05062046777807F00807F8
:10B69000FFB2002FF3D12D2D03D114F8015B012748
:10B6A00004E02B2D04BF244614F8015B002B57D077
:10B6B000102B08D151E02078782801D0582847D1A4
:10B6C0006578102302344FF0FF3ABAFBF3FA03FB1C
:10B6D0000AF000266FEA0008304609EB050C9CF8DA
:10B6E00001C00CF0040B5FFA8BFBBBF1000F01D023
:10B6F000303D0BE01CF0030C1BD0BCF1010F14BF5C
:10B700004FF0570C4FF0370CCCEB05059D4210DA8B
:10B71000B6F1FF3F0AD0504506D801D1454503DCBC
:10B7200003FB0050012601E04FF0FF3614F8015BE7
:10B73000D3E7731C05D1019922230B60304622B94F
:10B7400012E007B140427AB106B1611E11600BE010
:10B750003025002BB7D10823B5E7302DB3D1AAE7A8
:10B76000302DA8D00A23AEE7BDE8FE8F6802002086
:10B7700030B51346044A05460C4610682946224651
:10B78000BDE83040FFF774BF640200202DE9F047A8
:10B790008D68AB4281460C4692461F463FD38A894C
:10B7A00012F4906F39D0266809696369C1EB060805
:10B7B00003265E43022508F1010302F4806296FB32
:10B7C000F5F6DB1912B29E4238BF1E4682B13146F1
:10B7D000FFF796FD054600B913E021694246FFF7E1
:10B7E0004BFBA38923F4906343F08003A3810CE017
:10B7F000324600F022FB054638B948462169FFF77A
:10B800003DFD0C23C9F8003018E025616661454410
:10B81000C8EB06062560A6603D46AF4200D23D4615
:10B820002A462068514600F0EFFAA3685B1BA3602C
:10B8300023685D1925600020BDE8F087A38943F0E7
:10B840004003A3814FF0FF30BDE8F0872DE9F04FB2
:10B850009DB0064603938B8903F080031BB20D460F
:10B86000144663B10B6953B94021FFF749FD2860C5
:10B87000286110B90C233360D0E040236B610023B2
:10B88000099320238DF82930DFF89C81DFF89C9103
:10B8900030238DF82A3023469A4613F8012B1AB923
:10B8A000BAEB040B0FD002E0252AF5D1F8E73046B9
:10B8B000294622465B46FFF769FF013000F0A7806A
:10B8C000099B5B4409939AF80030002B00F09F809D
:10B8D00000234FF0FF3204930793059206938DF8EF
:10B8E00053301A930AF1010A4FF0010B05E0C8EB3F
:10B8F00000000BFA00F00343049354464A482178B1
:10B90000052200F073FA0AF1010A049B0028EED127
:10B91000D90602D520228DF853201A0702D52B22F2
:10B920008DF8532022782A2A03D0079B21460A202B
:10B9300010E0039A111D12680391002A01DB07929F
:10B9400004E0524243F0020307920493013408E0FA
:10B9500000FB03230C4601312278303A092AF7D93B
:10B96000079323782E2B19D163782A2B09D1039BB7
:10B970001A1D1B6803920234002BB8BF4FF0FF332F
:10B980000BE0611C00230A2001E000FB03230C46AE
:10B9900001312278303A092AF7D9059323482178D2
:10B9A000032200F023FA40B14023C9EB000003FA60
:10B9B00000F0049B03430493013414F8011B1C485A
:10B9C0008DF82810062200F011FA88B1194B33B90E
:10B9D000039B073323F007030833039313E003AB00
:10B9E0000093304604A92A46134BAFF3008007E0CA
:10B9F00003AB0093304604A92A460F4B00F092F89F
:10BA0000431C074603D0099BDB19099343E7AB8925
:10BA100003F040031BB20BB9099801E04FF0FF306F
:10BA20001DB0BDE8F08F00BF78E300087EE300089A
:10BA300082E30008000000008DB7000870477047DF
:10BA40002DE9F04715461F468A680B69DDF820800E
:10BA50009A42A8BF13462B6091F8432006460C4635
:10BA60000AB101332B602368990602D52B68023393
:10BA70002B60236813F0060916D094F8433022682F
:10BA8000003318BF0123920616D41EE0012330466E
:10BA900039465246C047013003D14FF0FF30BDE870
:10BAA000F08709F1010901E004F1190AE1682B6846
:10BAB000CB1A9945EADBE0E7E218302182F843101F
:10BAC00094F84510023382F844103046394604F1A8
:10BAD0004302C0470130E0D023682A68E16803F0E0
:10BAE0000603042B08BFC2EB01052369A2680CBF43
:10BAF00025EAE57500259A42C4BFC3EB0203ED18A1
:10BB00004FF000091A3408E0012330463946224636
:10BB1000C0470130C1D009F10109A945F4DB00207B
:10BB2000BDE8F0872DE9FF470E7E0C9D6E2E9146F5
:10BB300080460C469A4601F1430200F0AF800FD8D0
:10BB4000632E1DD006D8002E00F0C080582E40F085
:10BB5000D0804FE0642E1CD0692E40F0CA8018E0DF
:10BB6000732E00F0B78005D86F2E2BD0702E40F0CA
:10BB7000C08043E0752E25D0782E40F0BA8041E099
:10BB80002B681A1D1B682A6001F1420781F84230B8
:10BB9000B3E021682B6811F0800F02D0191D2960D5
:10BBA00008E011F0400F03F10401296002D0B3F95D
:10BBB000005000E01D68002D45DA2D236D4284F809
:10BBC000433040E021682B6811F0800F02D0191D2E
:10BBD000296007E011F0400F03F10401296001D052
:10BBE0001D8800E01D68237E5F486F2B14BF0A2369
:10BBF000082324E081F845605B4807E00B6843F0C8
:10BC000020030B607823594884F8453021682B685D
:10BC100011F0800F03F104062E6000D003E04F0600
:10BC200001D51D8800E01D68CE0744BF41F020010A
:10BC300021601DB9236823F0200323601023002115
:10BC400084F8431001E048480A236668002EA66085
:10BC500003DB216821F00401216005B96EB104F114
:10BC60004201B5FBF3F603FB16550F46455D01F89F
:10BC700001593546002EF4D100E01746082B0AD1B1
:10BC80002368DB0707D561682369994203DC302309
:10BC900007F8013C013FD21B226133E009682B68A1
:10BCA00011F0800F05D0191D2960196863690B60B8
:10BCB0000CE011F0400F03F10401296003D0196872
:10BCC00063690B8002E061691B68196000232361CE
:10BCD000174617E02B681A1D2A601F683846FFF7C1
:10BCE000F8FB63682061984288BF23612369636021
:10BCF00005E004F1420784F8426001232361002338
:10BD000084F84330CDF800A04046214603AA4B46B4
:10BD1000FFF796FE013002D14FF0FF3021E04046A0
:10BD200049463A462369D0470130F5D02368980741
:10BD30000ED4E068039B9842B8BF184611E0012377
:10BD4000404649463246D0470130E5D0013502E051
:10BD5000002504F11906E168039BCB1A9D42EEDB36
:10BD6000E7E704B0BDE8F08789E300089AE300083C
:10BD700030B5141E9BB0054604DA8B2303604FF0E8
:10BD8000FF301DE04FF40272ADF80C2000910491D9
:10BD900001D0611E00E021464FF6FF72029105912D
:10BDA000ADF80E2028461A4669461E9BFFF74EFD49
:10BDB000431C01DA8B232B6014B1009B00221A7004
:10BDC0001BB030BD73B50093054B06460D461446B7
:10BDD000186831462A462346FFF7CAFF7CBD00BFDC
:10BDE00064020020004870476C02002010B5C9B200
:10BDF0000346821803E0047801338C4203D0934257
:10BE00001846F8D1002010BD814210B511D28C180F
:10BE1000A0420ED253428118E418CB1801E0A15C75
:10BE2000995412F1FF32FAD210BDCC5CC4540133E4
:10BE300000E000239342F8D110BDF8B50646154640
:10BE40000C4621B91146BDE8F840FFF759BA1AB9B6
:10BE5000FFF714FA2C4612E000F013F8A8420ED2B5
:10BE600030462946FFF74CFA074638B121462A46A4
:10BE7000FFF702F830462146FFF700FA3C4620461D
:10BE8000F8BD51F8040C002802DA04390B58C01828
:10BE900004387047094A136863B118186946884224
:10BEA00098BF106004D9064B0C221A604FF0FF3384
:10BEB00018467047034B1360EFE700BFFC3D0020BE
:10BEC000E83E0020F03E0020FEE700BFF8B500BFCE
:10BED000F8BC08BC9E467047F8B500BFF8BC08BC6B
:10BEE0009E46704765617374657220646174653A3B
:10BEF00020253034642D253032642D253032640DF8
:10BF00000A000000536F00004D6F000044690000FC
:10BF10004D690000446F000046720000536100004C
:10BF20005375000054750000576500005468000008
:10BF30004443463737204572726F723A204869672A
:10BF4000682070756C7365203C3D20350000000052
:10BF50004443463737204572726F723A204869670A
:10BF6000682070756C7365203E3D203235000000FE
:10BF70004443463737204572726F723A20706172BF
:10BF800069747920503120696E636F7272656374D1
:10BF9000000000004443463737204572726F723A02
:10BFA0002070617269747920503220696E636F72FB
:10BFB00072656374000000004443463737204572C1
:10BFC000726F723A207061726974792050332069FF
:10BFD0006E636F7272656374000000000000000001
:10BFE0000000000006090906000000000A040A0A11
:10BFF0001F110000110E1111110E00001209090984
:10C0000009060000040A0A0A090A000000000000EC
:10C010000000000000000000000000000000000020
:10C020000000000000000000000000000000000010
:10C030000000000000000000000000000000000000
:10C0400000000000000000000000000000000000F0
:10C0500000000000000000000000000000000000E0
:10C0600000000000000000000000000000000000D0
:10C0700000000000000000000000000000000000C0
:10C0800000000000000000000000000000000000B0
:10C0900000000000000000000000000000000000A0
:10C0A0000000000000000000000000000000000090
:10C0B0000000000000000000000000000000000080
:10C0C0000000000000000000000000000000000070
:10C0D0000000000000000000000000000000000060
:10C0E0000000000004040404000400000A0A000028
:10C0F0000000000000051F0A1F140000040E0C04BD
:10C10000060E040009150E0E15120000040A0C1587
:10C11000120D0000040400000000000003040808E1
:10C12000080403001804020202041800040A040AA6
:10C1300000000000000000040E04000000000000E9
:10C14000000404080000000E0000000000000000D1
:10C15000000400000102020404080800060909099D
:10C1600009060000040C0404040E00000C02020482
:10C17000080E00000C020C02020C000002060A0F5E
:10C18000020200000E080C02020C000006080E0954
:10C19000090600000F010204040400000609060954
:10C1A0000906000006090907010600000000040056
:10C1B0000004000000000400000404080001020C58
:10C1C0000201000000000F000F000000000804033F
:10C1D000040800000E010204000400000609131503
:10C1E00017100F0000040A0A1F110000000E0A0CAD
:10C1F0000A0E00000007080808070000000E0909E1
:10C20000090E0000000E080E080E0000000E080EB9
:10C21000080800000007080B090700000009090FC3
:10C2200009090000000E0404040E0000000E0202C2
:10C23000020C000000090A0C0A09000000080808A6
:10C24000080F000000111B151511000000090D0B4F
:10C2500009090000000E1111110E0000000E090E58
:10C2600008080000000E1111110E0201000C0A0C4A
:10C270000A09000000060804020C0000001F040464
:10C280000404000000090909090600000009090961
:10C2900006060000001115150A0A000000110A0424
:10C2A0000A11000000110A0404040000000F010636
:10C2B000080F000006040404040406001008080423
:10C2C000040202000C04040404040C00040A0A1111
:10C2D000110000000000000000001F000804000022
:10C2E0000000000000000C020E0F000008080E09FC
:10C2F000090E0000000006080806000002020E12E7
:10C30000120E00000000040E0806000003040F04D3
:10C3100004040000000007090F010E0008080A0DC0
:10C320000909000004000C040404000002000E02CD
:10C3300002020C0008080A0C0A0900000C0404049C
:10C34000040400000000151F1515000000000A0D70
:10C3500009090000000006090906000000000E0996
:10C36000090E080000000E12120E020000000A0C56
:10C37000080800000000060C020C000000040F0476
:10C3800004020000000009090B0500000000090973
:10C3900006060000000015150E0A00000000090640
:10C3A000060900000000090906061C0000000E0630
:10C3B000080E00000204040804040200040404043B
:10C3C0000404040008040402040408000000000D32
:10C3D0001200000000040A0A0A0E0000000001001A
:10C3E0000100020002000300030004000400050035
:10C3F000050006000700080009000B000D000E00F4
:10C40000100012001400170019001C001F0021006A
:10C41000240028002B002E003200360039003D0099
:10C42000420046004A004F00540059005E0063007D
:10C4300069006E0074007A00800086008C00930012
:10C440009900A000A700AE00B600BD00C500CD0059
:10C45000D500DD00E500EE00F600FF0025750000C8
:10C460004E6F6E65000000005261696E626F77006A
:10C470004661646500000000526F6C6C00000000B3
:10C480004578706C6F64650052616E646F6D00007A
:10C49000536E616B6500000054656C65747970655E
:10C4A0000000000043756265000000004D61747279
:10C4B0006978000044726F70000000005371756568
:10C4C000657A65004E6F726D616C0000436C6F633E
:10C4D0006B320000080809090A0A0B0B0C0C0D0D41
:10C4E0000E0E0F000000000000000100030A000013
:10C4F0000100040A00000100080A00000101040B09
:10C500000C000101030B0C0001010C0000000101F3
:10C51000030A0C000101040A0C000101080B0000D1
:10C520000101040B00000101030B000000000000EA
:10C5300000000100030A00000100040A00000101DC
:10C54000080000000101040B0C000101030B0C00AA
:10C5500001010C0000000101030A0C000101040AA2
:10C560000C000101090000000101040B00000101A1
:10C57000030B00000000000000000100030A00009F
:10C580000100040A00000100080A00000100050A79
:10C5900000000101030B0C0001010C00000001016F
:10C5A000030A0C000101050B00000101080B00004B
:10C5B0000101040B00000101030B0000000000005A
:10C5C00000000100030A00000100040A000001014C
:10C5D000080000000100050A00000101030B0C0027
:10C5E00001010C0000000101030A0C000101050B10
:10C5F00000000101090000000101040B000001011D
:10C60000030B000045534B4953544C46DC4E460047
:10C610005A45484E5A57414E5A4947004452454997
:10C620005649455254454C0054474E414348564F95
:10C63000524A4D0048414C42515A57D64C46500040
:10C640005A5745494E53494542454E004B44524581
:10C6500049524846DC4E4600454C464E45554E56DE
:10C660004945520057414348545A45484E52530099
:10C67000425345434853464D55485200574553533E
:10C68000490000004F5353490000000052484549FB
:10C690004E2D525548520000534348574142454E93
:10C6A0000000000000000000000200030300070477
:10C6B000010004010407020004020404020407024A
:10C6C000000B03020403060304000404050505002F
:10C6D0000405020305020405050606010406070415
:10C6E00007000307030407070408010408050409F9
:10C6F00001050908030000000D1A0F1A0E1A121A7C
:10C70000161A131A191A111A171A151A181A141AAE
:10C710000D0010000E001200160013001900110089
:10C7200017001500180014002800000054696D65FA
:10C730006F757400290D0A004F4B00004552524F8F
:10C74000520000002D2000004950414444524553FE
:10C7500053200000415020004D4F44452000000070
:10C760006170000054494D45200000004649524D7B
:10C770005741524520000000434D44200000000076
:10C780004854545020474554200000002D2D3E2091
:10C79000000000003C30643E3C30613E0D0A000069
:10C7A0003C253032783E00006361702022257322E0
:10C7B0002C22257322000000617020222573222C78
:10C7C000222573220000000074696D652022257304
:10C7D0002200000045535038323636204C4F474730
:10C7E00045520D0A0000000094D500089CD50008B1
:10C7F000A4D50008ACD50008B0D50008B4D5000811
:10C80000B8D50008BCD50008D0CE0008D8CE0008A6
:10C81000E0CE000884E10008E4CE0008F0C800087B
:10C82000F0C80008F0C80008F0C80008F0C8000808
:10C8300004000000020000000200000002000000EE
:10C8400002000000C4D50008D0D5000894D5000827
:10C850009CD50008BCD50008C8D20008CCD200087E
:10C86000D4D2000830D20008D4D50008D8D50008AA
:10C8700084D3000884D3000884D30008DCD50008E2
:10C88000DCD50008DCD5000894D50008E0D5000808
:10C8900074CC0008F0D50008BCD5000894D5000879
:10C8A000E0D5000874CC0008BCD50008FCD5000811
:10C8B00004D600080CD6000810D6000818D60008C8
:10C8C0001CD6000834D20008BCD500086163746926
:10C8D000766500002573256400000000485454501C
:10C8E0002F312E3020323030204F4B000D0A0D0AF0
:10C8F000000000003C68746D6C3E0D0A00000000F2
:10C900003C686561643E0D0A000000003C74697477
:10C910006C653E003C2F7469746C653E0D0A000026
:10C920003C2F686561643E0D0A0000003C626F6444
:10C93000793E0D0A000000003C48313E0D0A00001F
:10C940003C2F48313E0D0A003C6120687265663D0F
:10C95000222F0000223E00003C2F613E266E6273B3
:10C96000703B266E6273703B0D0A00004D61696E6C
:10C97000000000006E6574776F726B004E6574770F
:10C980006F726B0054656D706572617475726500CD
:10C990006C6472004C445200446973706C6179009D
:10C9A000616E696D6174696F6E730000416E696DCF
:10C9B0006174696F6E730000616D62696C696768AC
:10C9C00074000000416D62696C6967687400000062
:10C9D00074696D657273000054696D65727300004F
:10C9E0003C503E003C7472206267636F6C6F723D16
:10C9F000236630663066303E0D0A00003C74723E9D
:10CA00000D0A00003C74643E000000003C2F74647A
:10CA10003E0000003C696E70757420747970653D4D
:10CA20002274657874222069643D220022206E61A0
:10CA30006D653D2200000000222076616C75653D29
:10CA40002200000022206D61786C656E6774683D7D
:10CA500022000000222073697A653D220000000058
:10CA60003C74643E3C627574746F6E2074797065BA
:10CA70003D227375626D697422206E616D653D2281
:10CA8000616374696F6E222076616C75653D2273F7
:10CA900061766500223E5365743C2F627574746F35
:10CAA0006E3E00003C2F74643E0D0A003C746162CF
:10CAB0006C6520626F726465723D303E0D0A000045
:10CAC0003C2F74723E0D0A003C74683E3C666F6EEB
:10CAD0007420636F6C6F723D626C75653E00000080
:10CAE0003C2F666F6E743E3C2F74683E0D0A00004A
:10CAF0003C2F7461626C653E3C503E0D0A000000A4
:10CB00003C627574746F6E20747970653D22737524
:10CB1000626D697422206E616D653D226163746986
:10CB20006F6E222076616C75653D22003C2F627528
:10CB300074746F6E3E266E6273703B003C2F626FA2
:10CB400064793E0D0A0000003C2F68746D6C3E0D48
:10CB50000A0000003C73656C6563742069643D22C3
:10CB600000000000223E0D0A000000003C2F73650B
:10CB70006C6563743E0D0A003C6F7074696F6E20C3
:10CB800076616C75653D22002073656C6563746524
:10CB9000640000003C2F6F7074696F6E3E0D0A00D8
:10CBA000266E6273703B3C696E7075742074797088
:10CBB000653D22636865636B626F7822206E616DEC
:10CBC000653D2200222076616C75653D22616374AB
:10CBD0006976652220000000636865636B65640008
:10CBE0003C696E70757420747970653D2272616E57
:10CBF0006765222069643D220000000022206D69E3
:10CC00006E3D220022206D61783D22002220737447
:10CC1000796C653D2277696474683A0070783B00EE
:10CC200022206F6E696E7075743D22005F6F75749F
:10CC30007075742E76616C75653D00002E76616CA2
:10CC40007565223E000000003C6F7574707574209D
:10CC50006E616D653D2200005F6F757470757422A2
:10CC60003E0000003C2F6F75747075743E0000002C
:10CC70002E0D0A0044656661756C74003135000044
:10CC80003C666F726D206D6574686F643D22474528
:10CC9000542220616374696F6E3D222F00000000F2
:10CCA0003C2F666F726D3E0D0A000000436F6C6F83
:10CCB000727300003C74643E0D0A000036340000BC
:10CCC000266E6273703B266E6273703B266E6273D3
:10CCD000703B0D0A000000004C6561726E696E6762
:10CCE0002049522072656D6F746520636F6E747297
:10CCF0006F6C2E2E2E000000537769746368696E86
:10CD00006720706F776572206F6E2E2E2E000000E8
:10CD1000537769746368696E6720706F77657220F6
:10CD20006F66662E2E2E00006F66666C696E65005B
:10CD30004D696E696D756D206C656E677468206FE6
:10CD400066206B6579206973203130210000000076
:10CD500054696D657365727665722073756363657A
:10CD6000737366756C6C79206368616E6765642E99
:10CD70000000000053657474696E67206F66206E52
:10CD800065772074696D657365727665722066617A
:10CD9000696C65642E00000054696D657A6F6E657C
:10CDA000207375636365737366756C6C7920636853
:10CDB000616E6765642E000053657474696E672048
:10CDC0006F66206E65772074696D657A6F6E652079
:10CDD0006661696C65642E0047657474696E6720CE
:10CDE0006E65742074696D6500000000446973709D
:10CDF0006C6179696E672074656D706572617475B8
:10CE000072652E2E2E00000053746F726564206DC3
:10CE1000696E696D756D2076616C75650000000046
:10CE200054657374696E6720646973706C61792EE0
:10CE30002E2E0000536176696E67207365747469E5
:10CE40006E6773207065726D616E656E746C792E9D
:10CE50002E2E00006874747020706174683A202768
:10CE60002573270D0A0000006874747020706172C9
:10CE7000616D65746572733A20272573270D0A006A
:10CE80002F000000253032642E253032640000006F
:10CE90002534640025303264000000006163746949
:10CEA0006F6E00006C6561726E697200706F7765FD
:10CEB000726F6E00706F7765726F666600000000BB
:10CEC000736176656461746574696D650000000066
:10CED00079656172000000006D6F6E74680000007B
:10CEE000646179006D696E00736176657469636B66
:10CEF00065720000576F7264436C6F636B000000D3
:10CF000056657273696F6E00454550524F4D000073
:10CF1000454550524F4D2056657273696F6E000043
:10CF20005469636B65720000506F776572204F6EB5
:10CF300000000000506F776572204F6666000000A9
:10CF40004C6561726E2049522072656D6F74652068
:10CF5000636F6E74726F6C00656570726F6D64756F
:10CF60006D700000454550524F4D2064756D700046
:10CF70003C503E0D0A3C666F6E7420636F6C6F729E
:10CF80003D677265656E3E003C5052453E000000B4
:10CF90002530347800000000202000003C2F505243
:10CFA000453E0000202020002F6E6574776F726B65
:10CFB0000000000073617665776C616E0000000010
:10CFC000776C616E6D6F6465000000007373696457
:10CFD00000000000576F7264436C6F636B204E65F6
:10CFE00074776F726B0000003C423E436F6E6E655B
:10CFF0006374696E6720746F204163636573732087
:10D00000506F696E742C2074727920616761696E4B
:10D01000206C617465722E3C2F423E003C423E53B0
:10D02000746174696E672061732041636365737313
:10D0300020506F696E742C20747279206167616969
:10D040006E206C617465722E3C2F423E0000000021
:10D050007361766574696D657365727665720000DB
:10D060007361766574696D657A6F6E6500000000A6
:10D070006E657474696D6500495020616464726501
:10D080007373000045535038323636206669726D2E
:10D090007761726500000000574C414E00000000AF
:10D0A0005353494400000000266E6273703B266EA5
:10D0B0006273703B266E6273703B00004B657900B3
:10D0C00054696D65207365727665720054696D658B
:10D0D000207A6F6E652028474D54202B29000000D0
:10D0E000476574206E65742074696D6500000000EA
:10D0F0003C503E0D0A3C666F6E7420636F6C6F721D
:10D100003D7265643E3C423E000000003C2F423EC2
:10D110003C2F666F6E743E0D0A0000002F74656D23
:10D1200070657261747572650000000073617665E8
:10D1300074636F72727274630000000073617665CD
:10D1400074636F72726473313878780064697370D5
:10D150006C617974656D70657261747572650000DB
:10D160002E350000266465673B430000576F7264EC
:10D17000436C6F636B2054656D706572617475727A
:10D18000650000005254432074656D7065726174CF
:10D1900075726500445331387878000054656D70BD
:10D1A00020636F7272656374696F6E2052544320FE
:10D1B00028756E697473206F6620302E35B0432950
:10D1C0000000000054656D7020636F7272656374B7
:10D1D000696F6E204453313878782028756E6974F1
:10D1E00073206F6620302E35B04329004469737078
:10D1F0006C61792074656D7065726174757265001B
:10D200002F6C6472000000006C64726D696E000027
:10D210006C64726D61780000736176656175746F1E
:10D2200000000000576F7264436C6F636B204C44C6
:10D23000520000004D696E004D6178004175746FB9
:10D240006D61746963206272696768746E65737377
:10D2500000000000536574206173206D696E696D74
:10D26000756D2076616C7565000000005365742053
:10D270006173206D6178696D756D2076616C75657F
:10D28000000000002F646973706C61790000000079
:10D290007361766569746973000000007361766577
:10D2A00073796E63616D6269000000007361766579
:10D2B0006272696768746E65737300007361766586
:10D2C000636F6C6F727300007265640067726565EE
:10D2D0006E000000626C7565000000007361766589
:10D2E000646973706C61796D6F64650073617665F4
:10D2F00074696E74657276616C0000007465737495
:10D30000646973706C61790073617665616C6C003F
:10D31000576F7264436C6F636B20446973706C6108
:10D320007900000045532049535400005065726D48
:10D33000616E656E7420646973706C6179206F66CC
:10D340002022455320495354220000004469737041
:10D350006C6179204D6F6465000000005573652095
:10D36000646973706C617920636F6C6F7273000015
:10D370004272696768746E6573732028312D313588
:10D38000290000003000000054656D70206469734E
:10D39000706C617920696E74657276616C00000052
:10D3A0005465737420646973706C617900000000C7
:10D3B0005361766520616C6C000000002F616E691E
:10D3C0006D6174696F6E730073617665616E696D0E
:10D3D0006174696F6E00000073617665636F6C6FD6
:10D3E00072616E696D6174696F6E000064656600DC
:10D3F00073617665616E0000737025640000000043
:10D4000066617625640000007361766563616E0075
:10D4100063737025640000006364656600000000AB
:10D42000576F7264436C6F636B20416E696D6174FA
:10D43000696F6E7300000000416E696D6174696F01
:10D440006E000000436F6C6F7220416E696D6174F5
:10D45000696F6E00616E25640000000064656625DA
:10D46000640000003100000063616E25640000006C
:10D4700063646566256400002F616D62696C69678D
:10D480006874000073617665616D62696D6F6465D3
:10D490000000000073617665616D62696C6564739C
:10D4A0000000000073617665616D62696F66667386
:10D4B000657400007361766561616E00617370254B
:10D4C000640000006164656600000000576F7264CC
:10D4D000436C6F636B20416D62696C6967687400AF
:10D4E000234C4544730000004F6666736574206FDB
:10D4F00066207365636F6E64203D2030000000007D
:10D50000416D62696C69676874204D6F64650000E5
:10D5100061616E2564000000616465662564000039
:10D520002F74696D657273007361766569640000BC
:10D53000610000006F00000066256400742564002F
:10D54000576F7264436C6F636B2054696D657273BF
:10D55000000000006964256400000000612564008B
:10D560006F256400682564006D256400485454509C
:10D570002F312E3020343034204E6F7420466F759A
:10D580006E640000343034204E6F7420466F756E28
:10D59000640D0A004E616D650000000056616C75F7
:10D5A0006500000059595959000000004D4D000018
:10D5B00044440000686800006D6D000041637469B8
:10D5C0006F6E0000574C414E20436C69656E7400CD
:10D5D00041500000470000004200000036330000C8
:10D5E000446563656C65726174696F6E000000006C
:10D5F0004661766F7572697465000000536C6F74D4
:10D600000000000041637469766500004F6E000001
:10D6100046726F6D00000000546F0000486F757215
:10D6200000000000010000000F00000015000000D5
:10D63000070000000B000000070000000B000000C6
:10D64000070000000B0000000F00000014000000A5
:10D65000000000000F0000001400000000000000A7
:10D6600001000000000000000500000002000000B2
:10D670000B0000000C0000001A0000000200000077
:10D680000B000000020000000B0000000000000082
:10D69000100000001C000000280000003000000006
:10D6A0000100000001000000000000000200000076
:10D6B000050000000C000000110000002200000026
:10D6C000050000000C000000050000000C00000038
:10D6D000000000001000000010000000200000000A
:10D6E0002000000001000000010000000000000018
:10D6F00002000000050000000C0000001100000006
:10D7000022000000050000000C00000005000000E1
:10D710000C000000000000000000000000000000FD
:10D7200000000000000000000100000001000000F7
:10D730000000000003000000050000000C000000D5
:10D740000F0000001E000000050000000C0000009B
:10D75000040000000B0000000000000010000000AA
:10D760001500000025000000250000000100000059
:10D770000100000000000000322E302E37000000B3
:10D780000D0A57656C636F6D6520746F20576F725B
:10D7900064436C6F636B204C6F6767657221000098
:10D7A0002D2D2D2D2D2D2D2D2D2D2D2D2D2D2D2DA9
:10D7B0002D2D2D2D2D2D2D2D2D2D2D2D000000004D
:10D7C00056657273696F6E3A2000000072746320B0
:10D7D0006973206F6E6C696E65000000727463205F
:10D7E0006973206F66666C696E65000065657072AE
:10D7F0006F6D206973206F6E6C696E6500000000AC
:10D8000063757272656E7420656570726F6D2076D7
:10D81000657273696F6E3A203078253038780D0A5A
:10D820000000000072656164696E672069722063A0
:10D830006F6465732066726F6D20656570726F6DC1
:10D840000000000072656164696E6720646973702E
:10D850006C617920636F6E66696775726174696F58
:10D860006E2066726F6D20656570726F6D000000CE
:10D8700072656164696E672074696D65736572763F
:10D88000657220646174612066726F6D20656570D9
:10D89000726F6D0072656164696E67206E6967689A
:10D8A000742074696D6572732066726F6D20656592
:10D8B00070726F6D0000000072656164696E6720B0
:10D8C00074656D7020636F6E6669677572617469E7
:10D8D0006F6E2066726F6D20656570726F6D0000EF
:10D8E000656570726F6D206973206F66666C696E16
:10D8F000650000007570646174696E67204545506D
:10D90000524F4D20746F2076657273696F6E2030B0
:10D9100078253038780D0A0077726974696E67204F
:10D9200076657273696F6E20746F20454550524F53
:10D930004D206661696C656400000000777269744F
:10D94000696E6720495220636F64657320746F208D
:10D95000454550524F4D206661696C65640000007A
:10D9600077726974696E6720636F6E666967207489
:10D970006F20454550524F4D206661696C656400CB
:10D9800077726974696E672074696D657365727604
:10D990006572206461746120746F20454550524F58
:10D9A0004D206661696C65640000000077726974DF
:10D9B000696E67206E696768742074696D6520649C
:10D9C00061746120746F20454550524F4D2066614F
:10D9D000696C65640000000063616C6C696E6720AF
:10D9E0004952206C6561726E2066756E6374696F52
:10D9F0006E0000007573657220627574746F6E201E
:10DA0000707265737365643A20636F6E66696775DB
:10DA100072696E6720657370383236362061732004
:10DA200061636365737320706F696E74000000003A
:10DA3000776F7264636C6F636B0000003132333454
:10DA40003536373839300000636F6D6D616E643A7A
:10DA50002073657420646973706C617920636F6CE6
:10DA60006F727320746F2025642025642025640D57
:10DA70000A000000636F6D6D616E643A2073657417
:10DA800020616D62696C6967687420636F6C6F7286
:10DA90007320746F2025642025642025640D0A00FE
:10DAA000636F6D6D616E643A2073657420706F777B
:10DAB0006572202573000000636F6D6D616E643ABE
:10DAC0002073657420646973706C6179206D6F6474
:10DAD0006520746F2025640D0A000000636F6D6D72
:10DAE000616E643A2073657420616D62696C696768
:10DAF0006874206D6F646520746F2025640D0A00C2
:10DB0000636F6D6D616E643A2073657420616E6938
:10DB10006D6174696F6E206D6F646520746F202570
:10DB2000640D0A00636F6D6D616E643A20736574F5
:10DB300020636F6C6F7220616E696D6174696F6EC6
:10DB4000206D6F646520746F2025640D0A0000004D
:10DB5000636F6D6D616E643A2073686F77207465D2
:10DB60006D7065726174757265000000636F6D6D34
:10DB7000616E643A2073657420646973706C6179B6
:10DB8000206272696768746E65737320746F2025F4
:10DB9000642C2064697361626C65206175746D6FBB
:10DBA0006D61746963206272696768746E6573730E
:10DBB00020636F6E74726F6C20706572204C4452DB
:10DBC0000D0A0000636F6D6D616E643A20736574B9
:10DBD00020616D62696C6967687420627269676848
:10DBE000746E65737320746F2025640D0A00000045
:10DBF000636F6D6D616E643A20656E61626C652065
:10DC00006175746F6D6174696320627269676874AD
:10DC10006E65737320636F6E74726F6C000000002A
:10DC2000636F6D6D616E643A2064697361626C65E7
:10DC3000206175746F6D61746963206272696768D1
:10DC4000746E65737320636F6E74726F6C00000086
:10DC5000636F6D6D616E643A2073657420646973DF
:10DC6000706C617920666C61677320746F20307806
:10DC70002530327800000000636F6D6D616E643A8C
:10DC800020737461727420646973706C617920749C
:10DC900065737400636F6D6D616E643A20736574B3
:10DCA0002074696D6520746F202573202534642DE0
:10DCB000253032642D2530326420253032643A25F7
:10DCC0003032643A253032640D0A0000636F6D6DA6
:10DCD000616E643A207374617274206E657420748E
:10DCE000696D65207265717565737400636F6D6D24
:10DCF000616E643A206C6561726E20495220636FD8
:10DD000064657300636F6D6D616E643A2073617654
:10DD10006520646973706C61792073657474696ED1
:10DD200067730000636F6D6D616E643A2070726995
:10DD30006E74207469636B65723A2027257327001F
:10DD40006C64723A206F6C64206272696768746EEA
:10DD500065733A202564206E657720627269676872
:10DD6000746E6573733A2025640D0A00657370380C
:10DD7000323636206E6F772075700000657370380C
:10DD8000323636206E6F77206F6E6C696E650000DC
:10DD9000202049502025730064636637373A2025D8
:10DDA00073202534642D253032642D2530326420D3
:10DDB000253032643A253032643A253032640D0A17
:10DDC0000000000072656164207274633A2025735C
:10DDD000202534642D253032642D253032642025F1
:10DDE0003032643A253032643A253032640D0A000C
:10DDF000466F756E642054696D65723A20257320F4
:10DE0000617420253032643A253032640D0A0000F6
:10DE1000676F742074656D706572617475726520CA
:10DE200066726F6D20445331387878783A202564D3
:10DE300025730D0A00000000676F742074656D7013
:10DE4000657261747572652066726F6D20525443FD
:10DE50003A20256425730D0A000000006E6F2074BF
:10DE6000656D706572617475726520617661696C4B
:10DE700061626C6500000000757064617465206407
:10DE80006973706C6179000049524D503A20504FCF
:10DE9000574552206B65790049524D503A204F4BFF
:10DEA000206B65790000000049524D503A206465AE
:10DEB0006372656D656E7420646973706C6179203E
:10DEC0006D6F64650000000049524D503A20696E44
:10DED0006372656D656E7420646973706C6179201E
:10DEE0006D6F64650000000049524D503A20646532
:10DEF0006372656D656E7420616E696D6174696FC2
:10DF00006E206D6F6465000049524D503A20696E75
:10DF10006372656D656E7420616E696D6174696FA1
:10DF20006E206D6F6465000049524D503A20646563
:10DF30006372656D656E7420686F75720000000015
:10DF400049524D503A20696E6372656D656E74205A
:10DF5000686F75720000000049524D503A206465A8
:10DF60006372656D656E74206D696E757465000011
:10DF700049524D503A20696E6372656D656E74202A
:10DF80006D696E757465000049524D503A206465A4
:10DF90006372656D656E7420726564206272696774
:10DFA00068746E657373000049524D503A20696E73
:10DFB0006372656D656E7420726564206272696754
:10DFC00068746E657373000049524D503A20646561
:10DFD0006372656D656E7420677265656E2062722E
:10DFE000696768746E6573730000000049524D5094
:10DFF0003A20696E6372656D656E7420677265653F
:10E000006E206272696768746E6573730000000049
:10E0100049524D503A2064656372656D656E742097
:10E02000626C7565206272696768746E65737300EF
:10E0300049524D503A20696E6372656D656E742069
:10E04000626C7565206272696768746E65737300CF
:10E0500049524D503A2064656372656D656E742057
:10E060006272696768746E657373000049524D503F
:10E070003A20696E6372656D656E742062726967BD
:10E0800068746E657373000049524D503A2067659D
:10E09000742074656D70657261747572650000003E
:10E0A000706F7765725F696E697428292063616C8F
:10E0B0006C656400737769746368696E6720706F5C
:10E0C000776572206F6E0000737769746368696E9C
:10E0D0006720706F776572206F6666002020676525
:10E0E000742074656D7065726174757265000000EE
:10E0F0002020706F776572206F66662F6F6E00004C
:10E1000020206F6B00000000202064656372656D45
:10E11000656E7420646973706C6179206D6F6465DD
:10E12000000000002020696E6372656D656E7420CA
:10E13000646973706C6179206D6F64650000000024
:10E14000202064656372656D656E7420616E696D13
:10E150006174696F6E206D6F646500002020696EC8
:10E160006372656D656E7420616E696D6174696F4F
:10E170006E206D6F64650000202064656372656DBC
:10E18000656E7420686F7572000000002020696E53
:10E190006372656D656E7420686F757200000000B3
:10E1A000202064656372656D656E74206D696E759F
:10E1B000746500002020696E6372656D656E742061
:10E1C0006D696E7574650000202064656372656D0D
:10E1D000656E7420726564206272696768746E652A
:10E1E000737300002020696E6372656D656E742024
:10E1F000726564206272696768746E65737300008B
:10E20000202064656372656D656E74206772656554
:10E210006E206272696768746E6573730000000037
:10E220002020696E6372656D656E74206772656526
:10E230006E206272696768746E6573730000000017
:10E24000202064656372656D656E7420626C75650F
:10E25000206272696768746E657373002020696E4E
:10E260006372656D656E7420626C7565206272699B
:10E270006768746E65737300202064656372656DF2
:10E28000656E7420676C6F62616C2062726967688A
:10E29000746E6573730000002020696E6372656D93
:10E2A000656E7420676C6F62616C2062726967686A
:10E2B000746E6573730000002020746F67676C656F
:10E2C000206175746F206272696768746E6573731C
:10E2D0000000000020205468616E6B20796F75216A
:10E2E000000000003139322E35332E3130332E31DB
:10E2F000303300004E65772074696D657A6F6E6506
:10E300003A2025640D0A00004300000004020020AA
:10E310001F0000001C0000001F0000001E00000085
:10E320001F0000001E0000001F0000001F00000072
:10E330001E0000001F0000001E0000001F00000063
:10E340001F0000001D0000001F0000001E00000054
:10E350001F0000001E0000001F0000001F00000042
:10E360001E0000001F0000001E0000001F00000033
:10E370006D0100006E010000232D302B2000686C21
:10E380004C006566674546470030313233343536D8
:10E390003738394142434445460030313233343511
:10E3A00036373839616263646566000020202020BA
:10E3B0002020202020282828282820202020202035
:10E3C0002020202020202020202020208810101015
:10E3D000101010101010101010101010040404046D
:10E3E00004040404040410101010101010414141E2
:10E3F000414141010101010101010101010101014D
:10E4000001010101010101101010101010424242DF
:10E41000424242020202020202020202020202021C
:10E42000020202020202021010101020000000007E
:10E4300000000000000000000000000000000000DC
:10E4400000000000000000000000000000000000CC
:10E4500000000000000000000000000000000000BC
:10E4600000000000000000000000000000000000AC
:10E47000000000000000000000000000000000009C
:10E48000000000000000000000000000000000008C
:10E49000000000000000000000000000000000007C
:10E4A000000000000000000000000000000000006C
:08E4B0002C1DFF7F010000009C
:10E4B8000000000001020304010203040607080922
:10E4C80020BF000808BF000824BF000828BF0008B4
:10E4D8002CBF000818BF00081CBF0008FF00000080
:10E4E800FF000000E8030000010000003C000000FD
:10E4F80020000000200000000300000020000000B1
:10E5080060C40008891E0008040000000400000020
:10E518000000000070C40008FD1E0008080000008C
:10E52800080000000300000078C40008C1290008A2
:10E5380004000000040000000300000080C400087C
:10E548006D2700080400000004000000030000001C
:10E5580088C40008C91B000804000000040000006B
:10E568000000000090C40008512C000804000000BE
:10E57800040000000300000098C40008C126000839
:10E58800080000000800000003000000A4C4000800
:10E59800FD2400080400000004000000030000003F
:10E5A800ACC40008B92F00080600000006000000EF
:10E5B80003000000B4C400081D2300080400000084
:10E5C8000400000003000000BCC40008A5210008E6
:10E5D800080000000800000003000000C4C4000890
:10E5E800000000000000000000000000F8CE000855
:10E5F800000000000000000000000000CCC400087B
:10E6080000000000000000000000000068C40008CE
:10E6180004000000040000000100000020000000C9
:10E6280001000000050000000500000060C40008AB
:10E6380001000000010000000000000068C400089C
:10E6480004000000040000000100000016000000A3
:10E658000F000000010000000F0000007CC6000849
:10E6680084C600088CC6000898C60008FFFF000092
:10E67800FFFF0000D80E0000FF000000FF000000B0
:10E68800FFFFFFFFFF000000000000000000000087
:10E698000102030406070809007A030A01000000C2
:10E6A8003139322E35332E3130332E3130330000AC
:10E6B8000000000000000000000000000000000052
:10E6C8000000000000000000000000000000000042
:10E6D8000000000008E3000800000000000000003F
:10E6E8000000000000000000000000000000000022
:10E6F8000000000000000000000000000000000012
:10E708000000000000000000000000000000000001
:10E718000000000004020020ABE300080100000034
:10E72800000000004A000000000000000000000097
:10E7380000000000000000000000000000000000D1
:10E748004A00000000000000000000000000000077
:10E75800000000000000000000000000AD010008FB
:04E76800890100081B
:0400000508000000EF
:00000001FF
